:100000005555AAAA211900000000000000000000B8
:1000100096E400000000000000000000A21F6C0732
:100020000002100005080000890200009F02000085
:10003000B5020000CB020000E10200000000000059
:10004000000000000000000000000000E12F0000A0
:10005000E52F000000000000F7020000E72F00007D
:10006000E92F0000052D0000633000003D2D000049
:100070000330000005300000093000001730000098
:10008000293000002B3000002D3000004B300000E4
:100090004D3000006530000000000000000000004E
:1000A0006730000069300000000000000000000020
:1000B000000000006B3000006D300000512D00008A
:1000C0006F3000007D300000090300009730000011
:1000D0009930000000000000000000000000000057
:1000E0002119000000F002F800F05AF80AA090E888
:1000F000000C82448344AAF10107DA4501D100F0E3
:100100004FF8AFF2090EBAE80F0013F0010F18BF55
:10011000FB1A43F00103184714DF010034DF01002C
:100120000A444FF0000C10F8013B13F0070408BF1D
:1001300010F8014B1D1108BF10F8015B641E05D0BB
:1001400010F8016B641E01F8016BF9D113F0080F70
:100150001EBF10F8014BAD1C0C1B09D16D1E58BF02
:1001600001F801CBFAD505E014F8016B01F8016B39
:100170006D1EF9D59142D6D37047000000230024AC
:1001800000250026103A28BF78C1FBD8520728BFA7
:1001900030C148BF0B6070471FB51FBD10B510BD03
:1001A000DFF80CD0FFF7F8FF03F036F91DF050FC34
:1001B0000002100003B4FFF7F1FF03BC1DF050FC78
:1001C0000A484FF0FF0101704FF0000080F31188E2
:1001D0004FF0000080F3098805484FF002010170DC
:1001E00062B604484FF080510160704722ED00E094
:1001F0000002100004ED00E002484FF08051016061
:100200007047000004ED00E04FF0200080F31188FB
:10021000EFF3098098B112480068124909688842D2
:1002200017D0EFF309800E49096820E9F00F8860C4
:1002300000B50B48006800F0F2F85DF804EB0848E0
:1002400008490A68026000688168B1E8F00F81F32C
:1002500009884EF0040E4FF0000080F311887047BB
:100260000402100008021000EFF311804FF020018B
:1002700081F31188704700004FF0000080F311886F
:100280007047000062B6704772B6704740BA704758
:10029000C0BA7047401E0028FCDC704700BE7047A3
:1002A00040BA7047C0BA70471EF0040F0CBFEFF39E
:1002B0000880EFF309804FF0010102F0C2BD1EF08B
:1002C000040F0CBFEFF30880EFF309804FF0020139
:1002D00002F0B7BD1EF0040F0CBFEFF30880EFF380
:1002E00009804FF0030102F0ACBD1EF0040F0CBFFB
:1002F000EFF30880EFF309804FF0040102F0A1BD95
:100300001EF0040F0CBFEFF30880EFF309804FF0ED
:10031000050102F096BD4FF0000000B504F005FAAB
:100320005DF804EBFFF770BF1EF0040F0CBFEFF396
:100330000880EFF309804FF0000102F082BD000059
:10034000194910B5012008701849002008601849A3
:100350000860184908601849086000F0B9F900F011
:100360004BF900F063F8002010BD10B5114800F003
:100370002AF90F4908600D490968884207D00A48E0
:100380000078022803D1BDE81040FFF735BF10BD4B
:1003900010B5FFF7EAFF044902200870FFF710FFCD
:1003A0004FF0FF3010BD00000002100004021000EA
:1003B000080210000C0210001002100070B50D466B
:1003C0000446C1698068CC221DF045FAE169A06845
:1003D000084440384FF08071C163216A8163002175
:1003E00041630163C1628162C0E908514FF00B3182
:1003F000C1614FF00A3181614FF0093141614FF025
:10040000083101614FF00731C1604FF00631816062
:100410004FF0053141604FF00431016070BD8269D9
:100420008168914201D803F0C6B8704710B54FF407
:10043000B4714F481DF039FA002010BD70B5054663
:1004400000EBC5014A4800EB8104FFF70DFF0646AB
:10045000207828B13046FFF70FFF6FF0010070BD24
:100460000320207000206560206204F11C0000F071
:1004700083F83046FFF700FF002070BD2DE9F04102
:100480000F463B49002500EBC00001EB80042E46DF
:10049000FFF7EAFE8046206A3843206204F11C0020
:1004A000074600F090F80CE0216A026C114203D07C
:1004B00000F066F9012600E06D1C2946384600F080
:1004C00078F80028F0D1012E01D1FFF74EFF404609
:1004D000FFF7D2FE0020BDE8F08170B50D4624493B
:1004E00000EBC00001EB8004FFF7BEFE216AA943C8
:1004F0002162FFF7C1FE002070BD70B50C461C499B
:1005000000EBC00001EB800500202060FFF7ACFE8F
:10051000296A2160FFF7B0FE002070BD2DE9F0418F
:100520000D46134900EBC0001E46904601EB8004C7
:10053000FFF79AFE07460F4800680564216A2942C2
:1005400003D104F11C0100F02DF93846FFF794FEA9
:10055000FFF78AFE216A29403160B8F1010F02D10C
:10056000216AA9432162FFF787FE0020B3E700005C
:100570002C0710000402100000210160084670479B
:1005800030B50A6812B10B46C46B09E0002208605E
:10059000C0E903210BE000BF02F10C03D26812B1E5
:1005A000D56BA542F8DC1A68C0E903211860002069
:1005B00030BD0068002201E0C068521C8A4201D0B0
:1005C0000028F9D170470068704702690AB11168C4
:1005D00031B96FF00400704701F10C02C96839B1FC
:1005E0008142F9D1C9681160002101610846704754
:1005F0006FF003007047000010B54FF4C871324827
:100600001DF053F9002010BD2DE9F0418846054644
:100610002D4900EB8500174601EBC004FFF724FECF
:100620000646207830B13046FFF726FE6FF0010015
:10063000BDE8F08102202070E7611422414604F1F8
:10064000080065601DF0C2F80020206204F124005B
:10065000FFF792FF3046FFF70FFE0020E8E770B586
:10066000194900EB800001EBC004FFF7FDFD0546D2
:10067000D4E90701814205DB144804F12401006834
:1006800000F090F8206A401C20622846FFF7F4FD35
:10069000002070BD70B50C4900EB800001EBC00478
:1006A000FFF7E2FD0546206A08B1401E206204F112
:1006B0002400FFF788FF10B1606A00F011F82846A7
:1006C000FFF7DAFD002070BD94081000040210004E
:1006D00010B54FF42A7140481DF0E7F8002010BD16
:1006E00010B5044690F8380002280BD02046FFF7DA
:1006F0006CFF022084F8380038492046FFF740FF9D
:10070000FFF733FE002010BD2DE9F05F8B46064653
:10071000314900EB06109046DDE90AA911F82020C6
:100720001D461AB16FF00100BDE8F09F01EB800497
:10073000FFF79AFD074601202070C4E90165C4E96E
:100740000585C4E907A91422594604F124001DF0C7
:100750003DF8002084F8370084F838006169E060D3
:100760002061C4E90F1020460C99FFF727FEA06016
:100770002046FFF7B5FF3846FFF77EFD0020D3E7A0
:1007800010B5044690F83800022809D02046FFF73B
:100790001CFF022084F8380010492046FFF7F0FEC5
:1007A000002010BD70B5044690F838000D460228B0
:1007B0000BD12046FFF709FF032084F838002946B3
:1007C0002046FFF7DDFEFFF7D0FD002070BD044896
:1007D0000068406870470000240A10000C021000F6
:1007E00004021000F0B58446002004460C4F14E0CB
:1007F0005CF824600323DD0046FA05F280EA02601B
:100800000825002802DA87EA400000E040006D1E5B
:10081000002DF6DC5B1EEED5641C8C42E8DBF0BDDF
:100820001B0000801248804712480047FEE7FEE7A1
:10083000FEE7FEE7FEE7FEE7FEE7FEE7FEE7FEE790
:10084000FEE7FEE7FEE7FEE7FEE7FEE7FEE7FEE780
:10085000FEE7FEE7FEE7FEE7FEE7FEE7FEE7FEE770
:10086000FEE7FEE7FEE7FEE7FEE7FEE7FEE7000045
:10087000AD080000C50000001E4800684FF00051A0
:10088000002891F8210000F01C000DD0042805D0AC
:10089000082805D00C2805D096200CE011200AE08D
:1008A000252008E04B2006E0042809D0082809D0BC
:1008B0000C2809D07020401E01F82C0F08707047DA
:1008C0000C20F8E71B20F6E73720F4E770470A49C9
:1008D00093200870D0E708490B200870CCE7054842
:1008E000006818B904480078932801D000207047A8
:1008F00001207047340400222100002010B504209C
:1009000000F0B3F9052000F0B0F9062000F0ADF9D1
:10091000072000F0AAF9082000F0A7F9182000F03D
:10092000A4F9192000F0A1F91A2000F09EF9E04A7C
:1009300000201060DE4B40331860DD491839086034
:10094000DB4908310860DB49C871D94C143C206090
:10095000D74C0C3420600872D54C103C2060D44C2D
:10096000103420604872D24C0C3C2060D04C1434BF
:1009700020608872CE4C083C2060CD4C183420603A
:10098000C872CB4C283420608873241D2060C87343
:10099000241D206008740120106018600870062172
:1009A000042000F07AF90621052000F076F90621EE
:1009B000084600F072F90621072000F06EF90621C2
:1009C000082000F06AF90621182000F066F90621D7
:1009D000192000F062F904211A2000F05EF90420C9
:1009E00000F04FF9052000F04CF9062000F049F91D
:1009F000072000F046F9082000F043F9182000F025
:100A000040F9192000F03DF91A2000F03AF90420CD
:100A100000F01FF9052000F01CF9062000F019F97C
:100A2000072000F016F9082000F013F9182000F054
:100A300010F9BDE810401A2000F00BB900EB80005F
:100A40009B494000002218390A609A4A521F1070D0
:100A500001200860704796490020183908607047E7
:100A600000EB800092494000002214390A60914A4C
:100A7000121F10700120086070478D490020143942
:100A80000860704700EB800089494000002210395F
:100A90000A60884AD21E107001200860704784499D
:100AA000002010390860704700EB8000804940004A
:100AB00000220C390A607F4A921E107001200860E3
:100AC00070477B4900200C390860704700EB8000BC
:100AD00077494000002208390A60764A521E107099
:100AE000012008607047724900200839086070478B
:100AF0007149097848430A21B0FBF1F16F48491E5A
:100B000080F86010582181761121C176042280F886
:100B100060205C228276C17670476848002180F8A8
:100B200060105C2181761121C1767047604A10B552
:100B3000283214680123D10664B10024146081F8BE
:100B4000350091F83F0000BF91F83F408442FBD050
:100B5000136010BD81F83500FAE700EBC00101EB2E
:100B600000106FF0030101EB800010B55449554CA3
:100B70000978B0FBF1F0401E80B2FF280CD9010AC1
:100B80002170494200EB01206070FF20FFF7CEFF8B
:100B90002078401E207010BD002121706170BDE8DA
:100BA0001040C0B2C2E7424828300168002909D08D
:100BB00000210160C10691F83F0000BF91F83F207D
:100BC0008242FBD0704710B53E4C2178607851EAE4
:100BD000000207D051B1FF20FFF7A8FF2078401E88
:100BE000207010BDBDE810400BF07CBFFFF79EFFEA
:100BF0000020607010BD2E4A10B5303214680123F9
:100C0000590794B10024146081F8370091F83F002F
:100C100091F83F408442FBD0136091F83F0000BF41
:100C200091F83F208242FBD010BD81F83700F3E7F6
:100C30001F483030016800290AD0002101604FF0C0
:100C4000005191F83F0000BF91F83F208242FBD055
:100C5000704700F01F020121914040094FF0E0224F
:100C600002EB8000C0F80011704700F01F02012164
:100C7000914040094FF0E02202EB8000C0F8801163
:100C8000704700F01F020121914040094FF0E0221F
:100C900002EB8000C0F8801270474907090E002857
:100CA00003DA00F00F00084A00E0084A8154704758
:100CB0001C05002233000020E2021000001000207A
:100CC000E10210001402100014ED00E000E400E066
:100CD0004948012101600021016070474748012116
:100CE000016000210160704710B5002000F06BF832
:100CF000FFF7F4FFFFF7ECFF41490020086041498E
:100D0000A0200870002000F06AF8BDE81040002024
:100D100000F04DB83A4801211C3801600021016003
:100D2000704710B5002000F04EF8334901200860EC
:100D3000002000F054F8BDE81040002000F037B863
:100D40002D4901201C39086070472F4800782E4932
:100D5000491C0978401A00F03F0070472B4902787F
:100D60000A7042784A7082788A70C278CA700279B2
:100D70000A7142794A7182798A71C079C871704763
:100D800023480068417882784FF00050437A03741A
:100D9000204B1B78437443891B0A83744389C374B3
:100DA00001754275C1798175017AC175704700F08E
:100DB0001F020121914040094FF0E02202EB800028
:100DC000C0F80011704700F01F0201219140400956
:100DD0004FF0E02202EB8000C0F88011704700F075
:100DE0001F020121914040094FF0E02202EB8000F8
:100DF000C0F88012704700005C840022A00000222E
:100E00007C04002200E400E0200400200002002016
:100E10003C021000D502100010B5092000F054F873
:100E20000A2000F051F8092000F05AF80A2000F0DA
:100E300057F80521092000F05FF805210A2000F08D
:100E40005BF833487F2141707C2282700171002160
:100E500000F848192F490A684FF0010192F8C8308C
:100E6000DC070AD09C0708D590F84A40C3F38203F8
:100E700001FA03F39C4380F84A4092F81131DC07F1
:100E800021D0C3F34203012B03D0234B4FF48064E2
:100E90001C604830837802F211121478C4F34204C3
:100EA00001FA04F4A343837003791478C4F3420471
:100EB00001FA04F42343037103781278C2F3420267
:100EC00091400B43037010BD00F01F0201219140BF
:100ED00040094FF0E02202EB8000C0F8801170471B
:100EE00000F01F020121914040094FF0E02202EB87
:100EF0008000C0F8801270474907090E002803DA05
:100F000000F00F00054A00E0054A815470470000D8
:100F1000480000203C02100000E100E014ED00E079
:100F200000E400E0704710B5044602462A21002084
:100F300000F06EF9221D2B21002000F069F904F168
:100F400008022C21002000F063F904F10C020F21AB
:100F5000032000F05DF92068000E032825D304F17A
:100F600014022D21002000F053F904F110022E216B
:100F7000002000F04DF904F11C022F21002000F0A8
:100F800047F904F118023021002000F041F904F182
:100F900024023121002000F03BF904F1200232212B
:100FA000BDE81040002000F033B910BD08B507219E
:100FB0006A46084600F02CF9009808BD10B5BE4CF2
:100FC000072060700020207044F2C000608000BFE5
:100FD00000BF00BF4CF2C000608000BF00BF00BF78
:100FE0004CF2E00060800920FFF754F944F2E00081
:100FF000608000BF00BF00BF4FF48040608010BD24
:10100000F0B500252E464FF00054E02717E000BF52
:10101000883401F03F0160702170678000BF00BF1D
:1010200000BFD4F808C043F825C06680883C00BFE4
:101030006D1C521E491C3F2901D9401CC0B2002A18
:10104000E6DCF0BD2DE9F0479B4D0026AD1C0446C3
:101050002E80DFF868920121C9F880104FF4C05843
:10106000A5F8008000BF00BF00BF00BF00BF4FF465
:1010700080572F803520FFF70DF92E80FFF79EFF58
:1010800000F0DCF85C2000F0EAF823460122082199
:101090000020FFF7B5FF231D012209210020FFF7E3
:1010A000AFFF04F1080301220A210020FFF7A8FF87
:1010B00004F10C0301220B210020FFF7A1FF04F132
:1010C000100301220C210020FFF79AFF04F1140302
:1010D00001220D210020FFF793FF00F0AFF8FFF78A
:1010E0006DFF2F8000BF00BF00BF00BF00BF00BF6B
:1010F00000BF00BF00BF00BFA5F8008000BF00BF59
:1011000000BF00BF00BF4FF440602880C9F8806076
:10111000BDE8F087F0B54FF0000C059C0CB14FF026
:10112000800CC5B200264FF00057644C28E000BF89
:1011300087F889504FEAC05EBEF1000F01F03F0E04
:101140004EEA0C0E01DA4EF0400E87F888E053F8B4
:1011500026E0C7F88CE04FF0010EC4F8B0E04FF085
:10116000000EC4F8B0E0491CC9B2402902D36D1C7E
:10117000EDB20021D4F8C0E0BEF1000FFAD1761C28
:101180009642D5DBF0BD4FF0005282F88900002373
:1011900009B1802002E0C00503D5402082F8880014
:1011A00001E082F8883045480121C0F8AC10C0F851
:1011B000AC3000BFD0F8C0100029FBD17047F8B5A3
:1011C0000C4605464FF4F47600213046FFF7DBFF6E
:1011D0000020014600902B4622463046FFF79AFF3A
:1011E000F8BDF8B50C4605464FF4F87600213046B8
:1011F000FFF7C9FF00214FF4FC70FFF7C4FF002088
:10120000014600902B4622463046FFF783FFF8BD8B
:10121000294B587041F0800003F8880927480021C5
:10122000B4300160012140F8B41900BFD0F8C010FB
:101230000029FBD1D3F890001060704710B51E4C08
:101240004FF48040A41C20800420FFF723F80020E6
:10125000208000BF00BF00BF00BF00BF10BD70B541
:10126000154C2126A41C268000BF00BF00BF00BF74
:1012700000BF40F02105258000BF00BF00BF00BFB8
:1012800000BF44F22101084320800420FFF702F848
:10129000258000BF00BF00BF00BF00BF268000BF89
:1012A00000BF00BF00BF00BF0020208000BF00BF04
:1012B00000BF00BF00BF70BD8800002000100022EA
:1012C000F8B5FA4C002635466670E6602661666120
:1012D0000120A66101F004F80C2001F001F80320C0
:1012E00000F0FEFF172000F0FBFF012001F004F8E2
:1012F0000C2001F001F8032000F0FEFF172000F0A1
:10130000FBFF01F05BF86A460221E94801F0F3FCBB
:10131000E8499DF80000E84A08709DF80110117036
:10132000442802D0542800D0042601F05AFA01F0D3
:101330004EFA0521012000F0EBFF05210C2000F002
:10134000E7FF0621032000F0E3FF0621172000F04D
:10135000DFFF012000F0B8FF032000F0B5FF1720E9
:1013600000F0B2FFE570A57025713046F8BD70B58C
:10137000CE4B5889C0F38001C0F34016C0F300245F
:101380007140C0F3C0226140C0F3803551406940D4
:10139000400840EAC130588170BDD065704738B50B
:1013A0000D46009014460421684602F07FFAC349B6
:1013B0008978C90602D5072D00D1401C00996165C6
:1013C00084F8530038BD2DE9F04FBD4D0646BB4CA7
:1013D00028688BB090F83304C00718D0608840F0BC
:1013E00080006080FFF7C3FF296800F00700084411
:1013F00090F8340484F84100FFF7B9FF2968C0F37E
:101400000210084490F83404800084F840004FF043
:10141000000B84F84BB02868A44F062E90F84507BF
:101420006075387802D0062827D010E006280ED044
:1014300001208DF80000684602F0C7FC684601F004
:10144000A1F8684601F055F8684601F080FB97481E
:101450004FF002084FF0E90A06709A48042EC0F3D4
:101460000E070DD0032E26D04FF00409022E46D0D1
:10147000052E60D0062E7CD0EEE08DF800B0DAE7C5
:101480008E4A3146E06AFFF78AFF206BE065A4F8D8
:101490004C70A07880060028286890F8580703DA76
:1014A00020F0060040F0040084F8510084F85280D7
:1014B00084F84EA0D0E0814A3146E06AFFF76FFF22
:1014C000206BE0657D4804212C3002F0EFF97D4966
:1014D00001EB8000C0F30E00A4F84C00A078800659
:1014E0000028286890F8580703DA20F0060040F03A
:1014F000040084F8510084F85280ED2018E06F4A0F
:101500003146E06AFFF74BFF206BE065A4F84C70B2
:10151000A07880060028286890F8580703DA20F0A1
:10152000060040F0040084F8510084F85290E52051
:1015300084F84E0090E0A078800628D528682C34E6
:1015400000F2C9305D4A01782176C178A1764178F0
:10155000A17780782073E07F314640F00100E0778A
:101560002068FFF71CFF5848C0F30E00208428684D
:1015700000E00DE090F8580720F0060040F002006F
:1015800084F8250084F8268084F822A02C3C63E0AF
:101590004A4A3146E06AFFF702FF206BE06549489E
:1015A000F830C0F30E00A4F84C00628890060028C2
:1015B000286890F8510203DA20F0060040F0040099
:1015C00084F8510041480078012811D1296891F828
:1015D0005002C3070CD091F81011090608D53C49F8
:1015E000097829B9800703D5012184F8528002E0E7
:1015F000002184F852902868D20500F25220038816
:1016000024F8343F438863800379237143796371FD
:10161000C388E38003892381837AA372C37AE37248
:10162000037B2374A0F25220A4F1340403D490F875
:10163000932784F8462090F85F0284F84A0011B19D
:1016400084F84EA002E0E52084F84E0094F84B00A8
:1016500040F0040084F84B00286890F8FD16C90794
:10166000A1784FEA817135D0002935DB94F84B1011
:10167000490736D490F8FC06C0070DD000210120A0
:1016800003F0FEF994F84F0020F00300801C84F86A
:101690004F00A4F842B028E00121084603F0F0F919
:1016A00094F84F0040F003001DE000001802100005
:1016B00004100020D4021000D5021000CC0C100041
:1016C0003C021000009F0120F0A0012057021000F2
:1016D00085021000002904DA90F8660720F0030064
:1016E00001E090F8660784F84F00607D20F0040068
:1016F0006075F64886700BB0F548BDE8F04F01F014
:1017000052B9F4480168F24891F8002280F821208B
:1017100091F80122C2754288D20507D491F80222BD
:1017200002F00F02827591F88F27027501F20321F2
:101730000A7802F03F020276B1F801208283CA786B
:101740008277E54A0979127801F0F00141EA121135
:10175000C1777047DF48DD4A0168D27901F1D200D4
:1017600030F81220DA48428311F8F93FC3754B78FC
:10177000037689788177002101758175D64908390A
:1017800009785A2904D1D449C91F097811444183E1
:1017900070472DE9F047CE4C0546002084F84B00F9
:1017A000CC4FE12084F84E003868DFF82C93C74E08
:1017B00090F84517617590F8FD165FEAC1782146EB
:1017C000B1F802C0CB7D0CF0FF024CF0010104D057
:1017D0005FEA8C7C01D4012D0AD0DFF80083082D4C
:1017E0000DD0092D2ED0072D55D00A2D72D04BE0EB
:1017F0007371B2710A22E2756180B84911E07371A8
:10180000B2716180417D027D4B1C94F860C003FB86
:1018100002F1BCF1010F02D902FB0CF1594308EBB4
:101820004101C1F30E01A4F84C1090F8531799F838
:10183000002001F0F00102F00F021143E17790F86F
:10184000550718E0FFF786FF3968F279087D5043A5
:10185000A34A02EB4000C0F30E00A4F84C0091F83C
:10186000530799F8002000F0F00002F00F02104337
:10187000E07791F8550784F82100954A2946012020
:10188000FFF78DFD2069E06561884807607D2FD5F1
:1018900020F0040032E0427D338B017D521C5A431C
:1018A000514308EB4101C1F30E01A4F84C1090F82C
:1018B000531799F8002001F0F00102F00F021143D4
:1018C000E17790F8550784F82100814A2946E068BD
:1018D000D6E7FFE78348C0F30E00A4F84C00FFF7FB
:1018E00010FF7B4A2946606AFFF759FDA06ACAE7E4
:1018F0003A6892F8452702F0040210436075C80761
:1019000005D094F84E0040F0020084F84E0038688C
:101910004FEA817190F8FD26D20718D0002918DB14
:10192000072D04D00A2D02D0012D05D01AE014F89D
:101930004F0F20F0030008E00021012003F0A0F881
:1019400014F84F0F20F00300801C20700AE00029DB
:1019500004DA90F8660720F0030001E090F86607CB
:1019600084F84F00B570BDE8F047594800F0ACBFAF
:10197000072812D00A2810D001280ED008280CD031
:1019800009280AD0042807D0032805D0052803D049
:10199000022801D0062801D115E5FAE670472DE9A5
:1019A000F8434A4D8146012901D1002028722C7A42
:1019B0004D4E641C474FDFF818810FE0386890F8EF
:1019C000FD06C00702D098F80200800756F82420D0
:1019D000694648469047012805D0641C0B2CEDD978
:1019E0000020BDE8F8832C729DF80000F9E72DE98E
:1019F000F0410646008800283BD064223146344836
:101A000002F0D4FDFEF7E3FE304C0025314FC4E96F
:101A10000650E571386890F8FD06C0070AD0B07826
:101A2000800707D42A49088810F0760F02D040F0CA
:101A300080000880A07800281BD101212448FFF7EE
:101A4000AEFF060015D0294901200870386890F8CB
:101A5000101149070FD590F8430780070BD401F008
:101A600012F90220E07001F012F9192001F03BF99F
:101A7000A670BDE8F08165703046BDE8F04177E7BB
:101A800000207047C268120006D00088C00503D548
:101A9000082008700120704700207047C2681200BB
:101AA00006D00088000503D5092008700120704782
:101AB00000207047C268120006D00078C00703D02B
:101AC000072008700120704700207047180210009E
:101AD000CC0C10003C021000F6FF01000080012039
:101AE000009E012070A101204CDA0100DF021000ED
:101AF000426A120006D00078000703D50A20087059
:101B00000120704700207047C268120005D000789D
:101B1000000602D501200870704700207047C26A95
:101B2000120008D0026B32B10078800603D5022083
:101B300008700120704700207047C26A120006D06A
:101B40000078C00603D505200870012070470020EA
:101B50007047C26A120006D00078800703D50420BF
:101B600008700120704700207047026B32B1007886
:101B7000400703D5032008700120704700207047FC
:101B8000C26A120008D0026B32B10088400503D54A
:101B90000620087001207047002070470020087060
:101BA000012070472DE9F0410421F94801F07EFE43
:101BB0000446F7480421001D01F078FEF54F054664
:101BC000DFF8CC83B878F44EA8F12C08042801D0B3
:101BD00002280CD198F80200800602D5A200EE4936
:101BE00002E0620006EB4401EC4802F0DFFCB8784A
:101BF000032801D0022811D198F80200800603D5ED
:101C0000AA0006EB840104E005EB44006A0006EB41
:101C10004001BDE8F041E24802F0C8BC29E730B518
:101C200089B001208DF80000DE48D94DD94C0068FC
:101C3000A5F12C0590F8FD06C0070AD0A87880070A
:101C400007D4A078012804D102208DF800000AF002
:101C500052FF00F080FBD4480190CF4803902179D7
:101C600000F51C7000EB4100049000202071CF486B
:101C70000590A9686846884709B030BDF0B5C94BE2
:101C800047F6FF7201291B6803D01B7DC84C002159
:101C90001EE0C74C5B7D3C3CF9E70D18EDB2C54F2B
:101CA000EE18F6B237F815E007F1800C37F8167029
:101CB0003CF815503CF81660AEEB0505BE1B3544EC
:101CC0002DB224F81150954200DA2A46491CC9B2B7
:101CD0009942E2D3002006E034F81010891A24F863
:101CE0001010401CC0B29842F6D3F0BD2DE9F84F59
:101CF000AC4D012000902868A74C002690F8F816FB
:101D0000C90730D0A2492C3991F8487007B901278A
:101D10009F49DFF880822C3991F8471091FBF7F149
:101D20000FFA81FA98F80210042902D0032903D08F
:101D30000BE0407D460023E0007D042146009448EE
:101D400001F0B4FD944901EB800498F802000228E8
:101D50000AD005280FD0042812D0032810D002285A
:101D60000ED005280CD03DE128688B4C417D007DCC
:101D70000844460004E028688C4C3A2690F8F9A6FE
:101D8000D8F80C2091465245EDDCB9F1000F05D191
:101D900086484FF4F87194301BF087FDC64698F8DA
:101DA0000200DFF81082002108F18008A8F5AA6B74
:101DB0002BE000BF5BF8213034F911C004286344E4
:101DC0004BF8213001D003281ED1B9F1000F07D103
:101DD000784B002223F8112047F6FF7228F81120D3
:101DE000DFF8D0C134F911203CF911309A4200DCFF
:101DF0001A462CF8112034F9112038F911309A4282
:101E000000DB1A4628F81120491CB142D2DB09F147
:101E10000101CEF80C1051457DDB0023DFF89891CD
:101E2000F046CEF80C30042806D003282ED0022825
:101E300056D0052870D0D5E001210020FFF71EFF05
:101E400053482C3890F8490060B12868407D410023
:101E50005648943002F098FDC8F810007821574891
:101E60001BF001FD00204B465946D8F810200AE02F
:101E700031F820507D43AD1A24F8105051F820500D
:101E800043F82050401CB042F2DBABE00021084692
:101E9000FFF7F4FE3E482C3890F8490060B12868FE
:101EA000007D41004148943002F06EFDC8F81400F6
:101EB000802143481BF0D7FC00204B465946D8F8F8
:101EC00014200AE031F820507D43AD1A24F8105058
:101ED00051F8205043F82050401CB042F2DB81E022
:101EE0002B482C3890F84900E8B12868407D410023
:101EF0002E48943002F048FDC8F810002868017D93
:101F0000427D49000BEBC20002F03EFDC8F8140010
:101F100078212A4801E061E034E01BF0A4FC802134
:101F200027481BF0A0FC002043464A4659460EE0D5
:101F300031F820C0B3F810800CFB07FCACEB080CA8
:101F400024F810C051F820C042F820C0401CD5F839
:101F500000C09CF815C0B0EB4C0FE9DB28685B694A
:101F6000407D40000BE000BF31F820507D43ED1A6A
:101F700024F8105051F8205042F82050401CB04234
:101F8000F2DB2FE00B4A00205946F03A23E0000034
:101F9000F80C100018021000009F012048B001202A
:101FA000C0B001203C02100000800120F0A0012000
:101FB00090A7012054A6012074A3012040B1012064
:101FC000B8B1012031F8203024F8103051F8203019
:101FD00042F82030401CB042F4DB03E0FFF7C8FCBD
:101FE000002000900098BDE8F88FCF4910B58A789E
:101FF0000120092A10D1CB795B1CDCB2CB4BCC7110
:102000001B6893F8D13003F00F035B1C9C4204D291
:102010001046FFF7ADFC002010BD0022CA7110BDB4
:10202000C14910B58A780120072A0BD18B69C04CB1
:102030005B1C8B6194F86040A34204DA1046FFF702
:1020400097FC002010BD00228A6110BD70B5B74911
:1020500009684B7D097D5B1C4B43B5490C460A78EA
:1020600094F86040D2071FD0012C1DD9498849053A
:102070001AD50020AF4A14E0012109E001FB030654
:1020800032F8105032F81660491C354422F81050CE
:102090008C42F3DC32F9101091FBF4F122F81010AD
:1020A000401C9842E8D370BD047770BD2DE9F04123
:1020B00088B0FFF777FDFFF798FF00282AD0FFF7D9
:1020C000AFFF002826D09A4DA878400603D4FFF72A
:1020D0000DFE00281ED0954E934C306890F8FD06FA
:1020E000C0070BD0A878800708D4A078012805D1B4
:1020F0006079E875A07968800AF0FDFCA07808286E
:1021000001D1A079688000218948FFF748FC18B107
:10211000FFF72EFC08B0ACE487480027A7700770D3
:10212000306890F8FD06C00706D0A878800703D471
:102130000021084602F0A4FC8049A42008733068FE
:1021400090F81001400702D5E77000F08AFD607832
:1021500001282BD08DF8007001208DF81C006846F6
:10216000FFF774FF2888DFF8D881400507D530686D
:10217000407D420008EB4001404602F017FA6D48EE
:10218000019000F5F050029000F5807003902179E5
:1021900000F51C7000EB4100049069482771F8308D
:1021A000CDE90508A96868468847B3E703208DF89C
:1021B0000000D1E770B55D485F4D4FF00004016845
:1021C00091F81001420758480AD591F8431789073A
:1021D00006D4C178012908D002290FD0032903D1E0
:1021E000C470FFF71CFD2C7070BD0221C17000F09F
:1021F0004EFDBDE87040322000F075BD0321C17076
:102200008078BDE87040FFF7B3BBF0B500224D1EEB
:1022100011E0531C1F460AE030F8126030F81340FA
:10222000A64203D920F8136020F812405B1C9BB231
:102230008B42F1D3BAB2AA42EBDBF0BD2DE9FF41EC
:1022400000252E462946012002F01AFC00246F4684
:1022500000F0B2FD27F81400641CA4B2082CF7D3D8
:1022600008216846FFF7D1FF5FF0020037F8101031
:1022700019B131446D1C8EB2ADB2401C80B206283B
:10228000F4D3B6FBF5F004B0C8E438B50C46054607
:1022900001226946104600F074FD9DF80000000917
:1022A00028709DF8000000F00300207038BD08B5CC
:1022B00001F0030141EA00118DF800100122694686
:1022C000104600F091F908BD00F01F020121914075
:1022D00040094FF0E02202EB8000C0F80011704787
:1022E00000F01F020121914040094FF0E02202EB73
:1022F0008000C0F88011704700F01F02012191405A
:1023000040094FF0E02202EB8000C0F880127047D5
:102310004907090E002803DA00F00F00094A00E01F
:10232000094A815470470000180210003C02100056
:10233000CC0C100000800120DF02100000100020F3
:10234000F89F012014ED00E000E400E0FE48016881
:102350000029FCD17047FD4800220260FB481C3870
:102360000260FB48026101210161826081600260BC
:1023700001600260F449A0F574700B68002BFCD179
:10238000F4490B7B43F020030B730B7B23F04003DA
:102390000B730B7B23F080030B730B7B23F0200369
:1023A0000B73C0F8D823C0F8E023EB4802707047E5
:1023B000E548183001680029FCD1704730B5E44881
:1023C000002474300460E24880300460E048C46057
:1023D0000121C160C460046001600460DF4D202001
:1023E00028706870DB49593D0873A4200873D648EB
:1023F000183001680029FCD1FFF7ADFFD848046010
:1024000085F8344030BDF0B5D648272500784428FB
:1024100002D0542800D1182500224FF4F831CA4EBA
:10242000CC485C2724E00C465FF0000303EB000E71
:1024300011F803C05B1C8EF860C00C2BF6DB336810
:10244000002BFCD18276C77604F10C0103EB000E61
:1024500011F803C05B1C8EF860C00C2BF6DB3168F2
:102460000029FCD1511C8176C77604F13001921C01
:10247000B2EB450FD7DBF0BD2DE9F0479246089E41
:102480005B1EC6F108010022B24C01F0FF0C15469C
:10249000002189469A420BDA00EB0208875C98F823
:1024A000018027FA06F708FA0CF847EA080703E064
:1024B00007D1875C27FA06F701EB040888F86070FB
:1024C00003E001EB040888F8609001F1010102F1DA
:1024D00001020C29DEDB9C490F68002FFCD10AEBBE
:1024E0000501A1765C21E1766D1C022DD0DBBDE8F3
:1024F000F08778B500259C4E00950446006A1123AC
:1025000032782946FFF7B8FF00951823727800212A
:10251000606AFFF7B1FF78BD00B58BB000208DF881
:102520000000684601F051FC6846FFF7E2FF0BB07F
:1025300000BD2DE9F0470024DFF80C828549824672
:10254000254626464FF05C0900209C4206DA00EB47
:10255000010C1AF804708CF8607002E0471887F8D4
:102560006060641C401C0C28EFDB00BFD8F8000042
:102570000028FBD15019887681F81B906D1C032D23
:10258000E2DBB4E730B5784D044640691623AA78FB
:102590000021FFF7CEFFEA78A069BDE83040202394
:1025A0000021C6E700B58BB000208DF8000068461A
:1025B00001F00BFC6846FFF7E5FFB8E7F0B5002433
:1025C000644D05E0165D6719641C87F8606064B2AD
:1025D0009C42F7DB5C4A1468002CFCD1A9761843B6
:1025E00040F01000E876F0BD70B50023594C05E0CE
:1025F000CD5C1E195B1C86F860505BB29342F7DB22
:1026000051490B68002BFCD1A07642F01000E07617
:1026100070BD30B5554C07220220216801F242718D
:10262000FFF7E2FF2168022201F24A710920FFF759
:10263000DBFF2168062201F24D710B20FFF7D4FF6A
:1026400020684B494B4D90F85307097800F0F00093
:1026500001F00F0108432870012229461120FFF7DD
:10266000C3FF2168032201F257711620FFF7BCFF58
:102670003F480122401E007800F00F01206890F8CA
:102680005A0761F31F10287029461920FFF7ACFF85
:102690002168012201F25B711A20FFF7A5FF216872
:1026A000042201F25C711B20FFF79EFF30480222DA
:1026B000C01C2946007828702D48401C007868709E
:1026C0001F20FFF791FF2168022201F5EC61212014
:1026D000FFF78AFF26480222001D2946007828704D
:1026E0002348801C007868702720FFF77DFF216851
:1026F000012201F263712A20FFF776FF2168072289
:1027000001F266713D20FFF76FFF2068022290F80A
:102710006E17297090F86F07687029464420FFF7FC
:1027200063FF2168022201F5EE614620FFF75CFF9E
:102730002168082201F272714820FFF755FF2168D5
:10274000082201F27A7117E0040B00221C0C00220F
:10275000D0030022001000201A02100059000020AF
:1027600040050022D4021000380210003C02100084
:10277000F6FF0100300D10005020FFF735FF2168F3
:10278000052201F284715820FFF72EFF2268FF4DC9
:1027900092F88F072870012302F28A72FA21002032
:1027A000FFF70CFF2268012302F28C720E21C02079
:1027B000FFF704FF2268012302F28D721421C0206A
:1027C000FFF7FCFE332068740B20A87430BD10B5F1
:1027D000FFF71FFFFFF7E6FEFFF79EFEBDE8104084
:1027E00011E630B55C2562225E236424E849442862
:1027F00001D0542804D00D704A708B70CC7030BD5D
:102800003020087035204870322088703720C8701A
:1028100030BD38B50546DF4C406D00906073010A4D
:10282000A173010CE173000E2074042269462B2071
:10283000FFF7DAFE012205F153012F20FFF7D4FE46
:1028400095F85300A074E86D0090E074010A2175BA
:10285000010C6175000EA075042269463520FFF752
:10286000C3FE0098800F84F84000CB490122087015
:102870003920FFF7B9FE38BD00EBC00101EB0010B5
:102880006FF0030101EB800010B5C449C44A097818
:10289000146890FBF1F0401EC1B2012358075CB1EF
:1028A0000024146080F8341090F83F1090F83F40F6
:1028B0008C42FBD0136010BD80F83410FAE7B948A1
:1028C00001680129FCD170477CB5044600208DF8D1
:1028D00004002046FFF79DFFAC48B4F84C10401CA4
:1028E0000180217D00F8011C94F84E104173A94E1F
:1028F000A07D86F83600AC4D286890F842078DF828
:1029000000006188890503D520F012008DF80000D1
:10291000012269460220FFF767FE042204F1150137
:102920000520FFF761FE2968022201F24A710920A1
:10293000FFF75AFE022204F11A010C20FFF754FEA1
:10294000022204F11C010E20FFF74EFE052204F1C5
:102950001E011020FFF748FE286890F8FC06C0070B
:102960000AD0012201A94420FFF73EFE022204F111
:1029700042013F20FFF738FE012204F14F013D20C4
:10298000FFF732FE012204F150014420FFF72CFE34
:10299000844801680129FCD194F84E00307323204B
:1029A000FFF76AFF7CBD7EB50446FFF732FF77482C
:1029B000B4F84C10401C018094F8451000F8011C3C
:1029C00094F84E104173784D286890F842078DF8BE
:1029D00000006188890503D520F012008DF8000001
:1029E000012269460220FFF7FFFD012204F11501D3
:1029F0000520FFF7F9FD94F84B00664EC00708D09C
:102A0000286800F2957190F8950786F83600012243
:102A100006E094F8460086F83600012204F14601EB
:102A20000620FFF7E1FD012204F144010720FFF732
:102A3000DBFD012204F14A010820FFF7D5FD2868DB
:102A400090F8FD16C90734D061888A0731D494F80C
:102A50004B2052072DD4B0F80027ADF80420B0F871
:102A60006A07ADF80800090609D594F84110084432
:102A7000ADF8080094F840001044ADF804000222BC
:102A800002A94120FFF7B0FD022201A90920FFF7AA
:102A9000ABFD296891F8FC06C0071DD0012201F2A8
:102AA0006E714420FFF7A0FD022204F142013F2095
:102AB00010E090F8FC06C00707D000208DF8040055
:102AC000012201A94420FFF78FFD2968022201F2AB
:102AD0004A710920FFF788FD012204F151011720F6
:102AE000FFF782FD012204F152011820FFF77CFD5F
:102AF000022204F134011B20FFF776FD022204F1CB
:102B000036011D20FFF770FD012204F1380121205C
:102B1000FFF76AFD012204F139012220FFF764FD6D
:102B2000012204F13F012A20FFF75EFD012204F19A
:102B30004F013D20FFF758FD1A4801680129FCD1DB
:102B400094F84E0030732320FFF796FE7EBD30B51B
:102B50000446C069104D0122007800F00F011248B0
:102B6000006890F85A0761F31F1028702946192051
:102B7000FFF73AFDE0680222294600782870606875
:102B8000007868701F20FFF72FFD0FE05300002032
:102B90003802100000100020300D1000E10210007B
:102BA00040050022000B00223C021000206929464B
:102BB000022200782870A06800786870BDE8304074
:102BC000272011E58E498F4B0A6892F84D27027035
:102BD0000A68B2F85027428009681B7801F25371E5
:102BE00003F00F030A7802F0F0021A430271B1F801
:102BF0000B20C28002818A7B82720A7CC272897831
:102C00000173704710B50446014601220B20FFF7FF
:102C1000EBFC0222A11C0E20FFF7E6FC0122211D85
:102C20001120FFF7E1FC0222A11D1D20FFF7DCFCB3
:102C3000022204F108012520FFF7D6FC012204F14D
:102C40000A012220FFF7D0FC012204F10B012A2007
:102C5000FFF7CAFC04F10C010122BDE8104013206B
:102C6000C2E4694908B50420087365480122694631
:102C7000006890F8430720F008008DF8000003205A
:102C8000FFF7B2FC08BD604920200873704718B5F3
:102C90005E4C01226946207840F0F0008DF800007B
:102CA0001046FFF7A1FC5849C020087320788DF822
:102CB0000000012269461046FFF796FC18BD5449F2
:102CC000002008607047524840300168002909D050
:102CD000002101604FF0005191F83F0091F83F2032
:102CE0008242FBD070474A4900220A60494A10706C
:102CF00001200860704770B5474C2368002BFCD159
:102D00001D4603E0C6185B1C86F880508B42F9D341
:102D10002368002BFCD102E0C45CD4545B1C8B42C2
:102D2000FAD370BD10B501F01BFDFFF7CCFF3B4897
:102D3000007878B13848183801680029FCD1324849
:102D4000C078400602D5364901200870BDE8104021
:102D5000FFF7ACB933490020087010BD10B501F081
:102D6000FFFC2B4900200860BDE81040FFF722BAA5
:102D700010B501F0F5FCFFF7A6FFBDE81040FFF726
:102D800019BA214B10B59876DA76234818380468BA
:102D9000002CFCD1012083F8E0001F480468002CBF
:102DA000FCD1002005E0C41894F860400C54401C8D
:102DB00040B29042F7DB10BD08B543F6FF70ADF8A6
:102DC0000000022269463F20FFF70EFC0220ADF80A
:102DD0000000012269463D20FFF706FC0A49E02079
:102DE00008734FF41670FDF755FA022269468720E2
:102DF000FFF7C7FFFFF735FFBDF8000008BD000073
:102E00003C021000F6FF0100001000207A021000C2
:102E1000000500222D0000201C0B00221A021000C9
:102E200019021000DF0210007048006890F8F007E7
:102E3000C00605D5ED214EF6ED52084609F0CBFF50
:102E4000FEE705460E46012009F087FF694C6848F9
:102E5000C4E900062868A0606868E060A86820618E
:102E6000E86860612869A0616869E061A86920621A
:102E7000614EE869606230685F4FA062103F386859
:102E800007F10408E062D8F8000008F104092063A3
:102E9000D9F8000006F1040A6063DAF80000DFF8F0
:102EA00058B1A063ABF1340BDBF80000E063381FCE
:102EB00000682064FDF78BFC6064504800210068C6
:102EC000A0640F202A6809F060FF01210F206A68C2
:102ED00009F05BFF02210F20AA6809F056FF0321C9
:102EE0000F20EA6809F051FF0C210F202A6909F030
:102EF0004CFF0E210F206A6909F047FF0F21084699
:102F0000AA6909F042FF20210F20EA6909F03DFF7C
:102F1000326821210F2009F038FF3A6822210F2062
:102F200009F033FFD8F8002023210F2009F02DFFEE
:102F3000D9F8002024210F2009F027FFDAF800201B
:102F400025210F2009F021FFDBF8002026210F208A
:102F500009F01BFF381F026827210F2009F015FF19
:102F6000FDF735FC024630210F2009F00EFFFFF778
:102F70005BFF012807D002280FD0032805D00428C2
:102F800005D004210AE0012108E0032106E0002128
:102F9000032009F0E2FEFFF747FF0221032009F0BA
:102FA000DCBE10B504460146042009F0D6FE012C13
:102FB00001D1FFF739FF10BD0146082009F0CDBE51
:102FC0000146062009F0C9BE10B504460146072097
:102FD00009F0C3FE012C03D0022C01D0032C01D137
:102FE000FFF722FF10BD0320EEE700003C021000B7
:102FF000AF0550FA5800012038ED00E088021000BB
:1030000001F0AEBB704770472C4810B5016821F045
:103010000401016001F0A4FBBDE8104019F020B9E3
:103020007047704701F09CBB10B501F099FBBDE8FB
:1030300010400AF015B910B501F092FBBDE8104040
:103040004FF0005001F0B0BD7047704710B501F06F
:1030500087FB1B480078012803D0BDE8104009F029
:103060005DBDBDE8104002F075BB704710B501F0C2
:1030700077FBBDE810404FF0805001F095BD7047E0
:10308000704770477047704770477047704710B57A
:1030900001F066FBBDE81040FDF795BD10B501F0ED
:1030A0005FFB07480078012801D102F02DFB05499C
:1030B0000020086010BD70477047000010ED00E070
:1030C000DE0210004805002210B55821E4481AF02D
:1030D000CAFBE348E349E44A01808280E349418036
:1030E000E34BC380E34C0481E34C4481E34C848193
:1030F000E34CC481E34C0482E34C4482E34C84827D
:10310000E34CC482E34C0483E34C4483E34C848368
:10311000E34CC483E34C0484E34C4484E34C848454
:10312000E34CC484E34C0485E34C4486E34C84863E
:10313000E34CC486E34C0487C38741878287E24916
:10314000A0F84010E1490968B1F86220A0F84220D7
:10315000B1F8C621A0F84420B1F8A120A0F846207B
:10316000B1F8F021A0F84820B1F85421A0F84A2085
:10317000B1F85221A0F84C200022A0F84E20D44AE9
:103180001288A0F850204A7DA0F852200A7DA0F8AD
:103190005420D04AA0F85620CB4891F84E274280C0
:1031A000B1F85C17C180018110BD10B5FDF7FEFEBE
:1031B00000EB104081B2C84801220378C748442B75
:1031C00004D1382902D00021017010BD027010BD59
:1031D0002DE9F047FDF7EAFE00EB104087B2BE484C
:1031E0001C261D2290F80080BD4D1E24BD481F23C3
:1031F000B6494FF0170C4FF00F09B8F1440F0AD140
:10320000382F08D02A70047043700968032081F8B1
:10321000E801BDE8F08785F800C00470467083704F
:10322000C270096881F8E891F3E7AF481322B0490A
:103230000378AE48552B02D0027019200CE0A34B46
:103240001B6893F81131DB0702D0A74A521C127891
:103250000270A548801C0078087070472DE9F0477F
:10326000FF222821A3481AF0F6FAA248FDF75BFED8
:10327000DFF880920E240126D9F80410072545F2C4
:10328000AA58414503D0D9F8081041453BD1D9F897
:103290000000D9F80820070E424506D1032F01D1BE
:1032A000C0F30136C0F3032502E00120FFF788FEDA
:1032B000D9F80410414504D199F8000000F01F042A
:1032C00002E00220FFF77CFE032F22D1D9F8143050
:1032D0004146894A48468B4201D1036900E0874B49
:1032E0001360C369864A8B4201D1836900E0854B34
:1032F0001360436A844A434502D1D9F8200000E0B4
:103300008248106005E00120FFF75AFE0220FFF717
:1033100057FE6E48016891F8F007400702D591F812
:10332000F20704E006F003002A0740EA126091F871
:10333000DA26D20711D0B9F80C2093B243450CD04D
:10334000694A921F1278C52A07D120F0F002664818
:10335000401F0078000742EA106091F8411720F002
:103360000C00C1F3C00240EAC200C1F3800140EA90
:10337000810167480170674880F8601001218176FB
:103380001121C1766448017864F30401017040E7BB
:1033900070B5FDF79CFAFDF7A7FC4C4D2868007846
:1033A000A52802D00120FFF7FCFD4FF008500124B2
:1033B000C0F898432868594A90F8271101F0010194
:1033C000116090F82701111DC0F340000860FDF75F
:1033D000A9FDFDF793FAFDF773FF042801D1FFF76C
:1033E000C8FDFDF7CDFCFDF717FD4A48802180F8A8
:1033F0006010042181761121C176FFF72FFFFFF7BE
:1034000014FF46486C380460FFF7E2FEFFF7CDFE7C
:1034100042480C38046070BD41F6211010B54107D8
:103420004881FFF7B5FFFFF74FFE3D495F20086079
:103430003C49002008603D483B49016001F50860B7
:103440003B4908603B4800F0D2FEFCF71DFF00F04E
:1034500073F8FCF717FFFCF79BFF012010BD00007D
:10346000000001200080012018D8012098D0012000
:10347000A8000120009F0120C82A0120042B012060
:10348000402C01207C2C0120B0310120EC310120A6
:1034900074130120B0130120442B0120802B012044
:1034A0002C32012068320120D01701200C18012095
:1034B0005417012090170120BC2A012080D0012040
:1034C0008CD0012068130120D82610003C02100087
:1034D000FC021000BC1A0120D4021000D602100019
:1034E00066021000B2021000F2FF0100E2021000BA
:1034F000E10210005C291000EC02100040A5AE02B1
:10350000F002100000879303F402100000366E01F1
:103510007A02100000100020200000208804002201
:103520003C2C0120D0021000C014100094021000A6
:1035300098021000C02510007FB5FCF701FF254D53
:10354000002400BF05EB441000F11002017F4CCABB
:10355000CDE90261CDE900230FC8FDF7D5F810B120
:103560000220FFF731FD641C082CEBDB1A4D002410
:1035700004EB440005EB8001091D55F8200006C945
:10358000FDF742F810B10220FFF71EFD641C082C65
:10359000EEDB114D0024603505EBC400416855F8A1
:1035A0003400FCF74BFF10B10220FFF70DFD641C47
:1035B000072CF1DB7FBD4068FFF715BD38B50C4621
:1035C000054669462846FCF798FF00992142F8D144
:1035D00038BD00007CDA01007CDB0100F0B500247E
:1035E0005F1E26E02546661C08E000BF30F915C0C6
:1035F00030F916E0F44500DB3546761C9E42F5DBDB
:1036000030F8146030F815C020F814C020F81560A8
:1036100031F8146031F815C021F814C021F8156094
:1036200032F8146032F815C022F814C022F8156080
:10363000641CBC42D6DBF0BD01EB8010801001EBB6
:1036400041014900182291FBF2F300EB400000F524
:10365000F83002FB1311006820F07F40C84000F0F2
:103660003F0070472DE9F04F87B0074600200090DB
:10367000019002900390049005900690FA4801256D
:10368000F84E804628E002241EE0087D04FB00502E
:1036900036F91000B84216DD032304AA02A96846D1
:1036A000FFF79CFFD8F80000BDF90010007D04FB77
:1036B000005036F91000814205DAADF80000ADF88F
:1036C0000850ADF81040641CD8F8001040464A7D00
:1036D000521EA242D9DC6D1C0168097D491EA94217
:1036E000D1DC00240DF1080BB246C1465FF00005A5
:1036F00004A83BF914C030F91430D9F80000017D5A
:10370000504603FB01C63AF91660BE4235DDD74E7E
:1037100076571E4406FB01C2731C03FB01C130F83F
:1037200012203AF811006146101A0FFA80F8701E44
:10373000FFF782FF069061463046FFF77DFF0146A6
:103740000698401A002807D0D9F800000EDAB0F821
:103750009C1341450FDB1CE0D9F80000B0F898132A
:103760004A42424515DAB0F89C1302E0B0F89803DB
:10377000414241450DDD012006906D1CEDB2022D48
:10378000B6D3641CE4B2032CB0D3069807B0BDE8EE
:10379000F08F0020FAE7F0B5054600204FEA254CEF
:1037A0004FEA2146BCEB060400D564429C421FDA76
:1037B0004FEA2247BCEB070400D564429C4217DA6B
:1037C000F41B00D564429C4212DA2DB20CB2291BC4
:1037D00000D5494299420BDA12B2A91A00D54942E2
:1037E000994205DAA11A00D54942994200DA01202E
:1037F000F0BD2DE9F0479246012547F6F872564292
:103800009946AC460024089F17E000BF30F81430FA
:1038100031F81480A8EB03031BB29A4200DD1A466C
:103820009E4200DA1E46002B02DA4FF0000502E04D
:1038300001DD4FF0000C04F10104BC42E6DB55EA67
:103840000C0306D0012D01D02DB108E0BCF1010F11
:1038500005D1002203E0BCF1010F00D13246002562
:103860002C462B4611E000BF30F8136031F813C02E
:103870001644ACEB060636B24E4505DAC9F1000C2B
:10388000664501DD3544641C5B1CBB42ECDB95FBEB
:10389000F4F10A44002105E030F8113013442AF80D
:1038A0001130491CB942F7DBBDE8F08770B503461B
:1038B000002002466E4C09E09D5C521C05F00F068C
:1038C00004EB1515A65D2D78304428448A42F3DBBD
:1038D00070BD884200D308467047884200DB084626
:1038E0007047884200D808467047884200DC084686
:1038F0007047884200D30846904200D31046704774
:103900002DE9F047D0F810C00568046A85FB0C1259
:10391000A1FB041242694368914683FB02628269FB
:10392000E246A6FB02677618D0E9021781FB07C8BA
:10393000C069ACFB00C81CEB060682FB0A2CA2FB8C
:10394000011280FB0902A0FB0502401884FB07124C
:10395000A1FB03120818301A4FEAE071A4E7F0B592
:103960000025059F14E000240EE000BF05FB03F6D0
:1039700000EB860C01EB86065CF824C09CFBF7FC90
:1039800046F824C0641C64B29C42EFDB6D1C6DB22F
:103990009542E8DBF0BDF0B50025059F14E000245A
:1039A0000EE000BF05FB03F600EB860C01EB86067C
:1039B0005CF824C00CFB07FC46F824C0641C64B20D
:1039C0009C42EFDB6D1C6DB29542E8DBF0BDF0B5BB
:1039D0000025059F17E0002411E000BF05FB07F656
:1039E00000EB860C01EB860E5CF824C05EF824E048
:1039F00002EB8606F44446F824C0641C64B2BC4260
:103A0000ECDB6D1C6DB29D42E5DBF0BDF0B5002531
:103A1000059F17E0002411E005FB07F600EB860C7C
:103A200001EB860E5CF824C05EF824E002EB86060B
:103A3000ACEB0E0C46F824C0641C64B2BC42EBDB59
:103A40006D1C6DB29D42E5DBF0BD2DE9F04F814666
:103A500009A88A46B0E822400020DDF834B08A4246
:103A600029D094E6400D10003C0210000B0310001A
:103A700014DC010000241BE0002116E000FB02FC26
:103A800001FB05F800FB0BF609EB8C0C0EEB860630
:103A900003EB88085CF821C056F8247058F824809D
:103AA000491C0CFB087746F824709142E6DB641C45
:103AB000AC42E1DB401C5045DCDB68E62DE9F0431D
:103AC000914600230024224600EBC30609EB830540
:103AD00001EB820856F822C055F8247058F824806B
:103AE000521C0CFB087745F82470022AF0DB5B1CA3
:103AF000022BE7DBBDE8F0832DE9F043914600247B
:103B0000002200EBC40609EBC405002301EBC30847
:103B100056F823C055F8227058F822805B1C0CFB25
:103B200008775BB245F82270022BEFDB521C52B2D1
:103B3000022AEADB641C64B2022CE1DBDAE72DE93D
:103B4000F04389B0044600680090606801902069E5
:103B500002906068039020690490A0690590206934
:103B60000690A0690790E06908900D466846FFF747
:103B7000C7FE8046A0680190E068049060690790E5
:103B800089466846FFF7BCFE064660680190A0685B
:103B9000029020690490E0680590A0690790606930
:103BA00008900F466846FFF7ABFEC5E90401C5E97A
:103BB0000267C5E9008909B09CE72DE9FF4F4FF086
:103BC000000A89B09B465746D146D04656465546D0
:103BD00054462021684619F068FE0B9810E00999B8
:103BE000824431F9102000FB00F102FB0166884499
:103BF000414302FB009901FB004417440D44401C63
:103C00005845ECDD0B99ABEB0100401CCDE9000AF7
:103C1000CDE90654CDE90486CDE9027968460A99D2
:103C2000FFF78DFF0DB0B2E5FB480068017B427BDA
:103C300041EA0221827BC07B41EA024141EA006005
:103C400040007047F44800680179427941EA022156
:103C50008279C07941EA024141EA0060704700B5CB
:103C6000FFF7E2FF4008400000BDF8B50E460446ED
:103C7000FFF7F5FF0090FFF7D7FF054604216846E0
:103C8000FFF714FE04EB400700240099204623466A
:103C90004FF0010C0CFA03F20A4207D02A4204D07A
:103CA00037F8102026F81420641C401C5B1C1E2BC7
:103CB000F0DBF8BDC6E7FCB50E460746FFF7CFFFC1
:103CC0000190FFF7BFFF0090FFF7BCFF05460421FE
:103CD00001A8FFF7EBFD044604216846FFF7E6FD67
:103CE00000EB440007EB4007002000990446034620
:103CF0004FF0010C0CFA03F20A4207D02A4204D01A
:103D000037F8142026F81020401C641C5B1C202B64
:103D1000F0DBFCBDC0490020096891F8E81119B139
:103D2000BE480178012088404000704730B5BA494C
:103D30000020096891F8E81100290DD0B749B84B67
:103D4000012409781D2908D000215D5C04FA05F2E0
:103D50001043491C0429F8DB30BD00229D5C04FAA5
:103D600005F10843521C022AF8DB30BD70B5AB4A9E
:103D700012781D2A08D082880A8002884A80C28868
:103D80008A804088C88070BD0022A34C012303FABA
:103D900002F6256895F8E851354203D030F8125004
:103DA00021F81250521C062AF1DB70BD00B5FFF756
:103DB0003BFF40F0010000BD44E79A4A520102EB8C
:103DC000810101F10851086070470178012916D07E
:103DD00095494160491C81609449416193492C3166
:103DE00081619149891CC160491C0161491FC16100
:103DF0008E496C3101628D498D31416270478A492B
:103E000010394160491C81608849BD314161874951
:103E1000E931816184490E39C160491C0161491F42
:103E2000C1618349016282492131E6E7F0B5074665
:103E30000598884201DD1846F0BDB84201DA104607
:103E4000F0BD9E1AC01B4643CD1B00D10125724C0C
:103E500096FBF5F02468104400B294F8F1470E2C5C
:103E6000EED1A446734CA4F800C04FEA264CA4F847
:103E700002C0A6802E14E68025816781A181E2819F
:103E800023826082F0BDF0B507460598884201DDC7
:103E90001846F0BDB84201DA1046F0BD9E1AC01BAC
:103EA0004643CD1B00D101255B4C96FBF5F0246801
:103EB000104400B294F8F1470E2CEED1A4465D4CAC
:103EC000A4F800C04FEA264CA4F802C0A6802E1425
:103ED000E68025816781A181E28123826082F0BD35
:103EE00030B5002304465242184615B209E000BF1F
:103EF00034F91320AA4203DA002A00DA52421044AD
:103F00005B1C8B42F4DB30BD01EB8010801010B5E0
:103F100001EB41014900182391FBF3F403FB141357
:103F200000EB400000F5F8303F2401689C40A143BD
:103F30009A400A430270110A4170110C817010BD41
:103F40002DE9F04F8B4682460026FFF72FFF814672
:103F5000FFF778FE07464FF0270C00254FF00108C9
:103F600008FA05F111EA090F13D0002408FA04F049
:103F700038420AD0BBF1010F10D01AF806202146B2
:103F80002846FFF7C1FF761CB6B2641CA4B2202CF1
:103F9000ECD36D1CADB26545E2DB62E521462846F7
:103FA000FFF74AFB0AF80600EDE71F4915390880BC
:103FB00070471D481538B0F9000070472DE9FF4FD4
:103FC0000027864681B04FF0FF093E46BC46481C9C
:103FD00062D0501C60D0881E012800DC0120C4B2D1
:103FE0000D4801F1020805682B7D981E404501DD52
:103FF000881C00E0981E00F0FF0B901E012800DCDA
:104000000120C0B20090687D02F10208851E45457E
:1040100012DD901C11E000003C021000660210004E
:10402000B20210003C2C0120F7FF010040F8010013
:1040300069F9010018D80120801E00F0FF0A17E07E
:10404000009D11E005FB034080B21EF8000084448F
:104050001FFA8CFCB84200D90746814500D9814639
:10406000761C6D1CF6B2EDB25545EBD9641CE4B27A
:104070005C45E5D953430EEB0100185CBCEB000135
:1040800001D5C1F10001A6F1010691FBF6F1411A3B
:1040900000D5494204980170A7EB0900C0B205B0F1
:1040A000DFE430B5FB4A0346F9481468B0F9000074
:1040B000B4F8342194F8464704F00F04641C02FB62
:1040C000040562439D4207DAA2EB60029A1A92B29B
:1040D00092FBF0F0084409E0141A9C4208DD02EB60
:1040E0006002D21A92B292FBF0F0081AC0B230BD50
:1040F000084630BD2DE9FC4F8B4682460026DFF88E
:1041000098C3E44CDFF89493DFF8948317E001251B
:104110000FE0007D002205FB00618FB2391A38F9EB
:10412000170019F80110FFF7BCFF6D1C0CF8070011
:10413000EDB22068417DA942EBD2761CF6B2206830
:10414000007DB042E3D820684FFA8AF24FFA8BF133
:10415000007D6B46604416460D46FFF72FFF07466D
:1041600001AB32462946CD48FFF728FF01462068BB
:1041700090F8582407EB9210884207D39DF800006E
:104180009DF8041000EB9210884202D20120BDE895
:10419000FC8F0020FBE7821002EB42020A4400EB96
:1041A00040004000182190FBF1F301FB130110685F
:1041B00020F07F40C84000F03F007047831003EBC1
:1041C000430310B51A4400EB40004000182390FB55
:1041D000F3F403FB14033F2410689C40A043994070
:1041E00001431170080A5070080C907010BD2DE941
:1041F000F14F82B04FF0000B7821029819F055FB77
:10420000FFF7D4FD4FEA5008FFF71CFDDC4681465E
:1042100066464FF0010A00BF0AFA06F111EA090FDB
:1042200025D000240AFA0CF001272546CDF800001D
:104230000AFA05F010EA080F14D031462846FFF7B5
:10424000FBF9A04208D00299009A51F827101143B7
:10425000029A42F8271003E00BF101011FFA81FBDB
:1042600004467F1C6D1C272DE2DB0CF1010C761C33
:10427000202ED1DB5846BDE8FE8F2DE9F04F834656
:10428000844800242246D0F800A001219AF8145056
:10429000A5F1010621E003200123DFF808E203FA7B
:1042A00001F99AF8157015E05EF820C01CEA090FB4
:1042B0000FD0A0F1010300FB051C03FB05183BF91F
:1042C0001CC03BF91830BCEB030300D55B421C4417
:1042D000521C401C8742E7DC491C8E42DBDC02B9E1
:1042E000012294FBF2F058E62DE9FF4F85B0002142
:1042F00003910291019100916649012B0C6894F899
:10430000775005F00F0700D10027667D94F87A30CA
:10431000C7F1100BB34200D21E46002304930123C1
:1043200081E000BF4FF00009C84603241FE05D494B
:1043300051F824C0012199401CEA010F04FB05310A
:1043400030F911C0A4F1010101FB053130F9111060
:10435000ACEB010106D0002900DA4942DDF818C0B3
:10436000A1EB0C01002900DA49428944641CB442E3
:10437000DDDB31469EF815A01FE04A4C54F821C001
:1043800001249C401CEA040F01FB053430F914C0E1
:10439000A1F1010404FB053430F91440ACEB040432
:1043A00006D0002C00DA6442DDF818C0A4EB0C043F
:1043B000002C00DA6442A044491C8A45DDDC0499E3
:1043C000012910D10199B1EB090101D5C1F1000119
:1043D000039C214403910099B1EB080100D54942A7
:1043E000029C21440291CDE900899EF87B109942FC
:1043F00016D11168039D79430BFB0511CC1701EB16
:104400001471091111609168029D79430BFB05112C
:10441000CC1701EB147109119160002103910291F5
:1044200001215B1C04911B49D1F800E09EF8145057
:10443000691E99423FF776AF5068039978430BFBAA
:104440000100C11700EB117000115060D068029B91
:1044500078430BFB0300C11700EB11700011D06013
:1044600009B09AE530B5044600200222A1F101010D
:104470000BE000BF04EB420534F9123035F9025C61
:104480005B1B00D55B421844521C8A42F2DB30BDF4
:10449000E2FF01003C02100090AB0120D0A70120F8
:1044A000400D1000C025100070B50020FE4C0146E4
:1044B000FE4A1268537D0BE034F91150B2F8506493
:1044C000B54203DBB2F85264B54200DD0120491C5D
:1044D0008B42F1DC70BDF0B5F44C0020034624683B
:1044E00001460246F04E677D06E000BF36F91350E4
:1044F000954200DD2A465B1C9F42F7DC0023EC4E10
:10450000277D05E036F913508D4200DD29465B1CFE
:104510009F42F7DCB4F84E348B4201DB934200DA61
:104520000120F0BD2DE9F14FE049002318460C6849
:1045300094F84914267DC1F3C001B4F865B4B4F809
:1045400067A4A6EB010926E0657D0322DFF864E39A
:10455000DFF86483A5F1010519E000BF5EF822C011
:10456000012707FA01F71CEA070F0ED102FB061715
:1045700038F917C0A2F1010707FB061738F91770C1
:10458000BCEB070700D57F423B44521CD2B2954298
:10459000E4DC491CC9B28945D6DC00999B450B6017
:1045A00002D2534500D20120BDE8F88F04E000BFDD
:1045B00011F8013B00F8013B521EF9D270477CB55F
:1045C0000D460446FFF74BFB0090FFF73BFB0190C5
:1045D00000980421400800906846FFF767F90646F6
:1045E000042101A8FFF762F93044820021462846E1
:1045F000FFF7DCFF7CBD0B46AC4909684A7D097DAD
:10460000521C4A43014652001846CFE72DE9F041BB
:104610000446642119F049F90025A44E25806580DF
:10462000306890F8940700F0010045EA401060807F
:10463000A560FFF7BBFBE060FFF704FB9F4F206125
:104640009F497888608309785A2904D19C49491C7C
:10465000097808446083306800F24670C27A817A33
:1046600002F03F0241EA0221A1834178E17590F80E
:10467000491021750178A17581782176017BA17798
:104680008F49407B083100F0F000097801F00F01FC
:104690000843E077FFF73EFB6062FFF747FBA0624D
:1046A000FFF7DDFAE062FFF7CDFA20632C34F888DB
:1046B0002081E081306800F5E96090F848102176AB
:1046C00090F84A10617690F84B10A17610F84E1CC5
:1046D000E17601212177657790F84920A277C28A97
:1046E00062812282027E2273427E6273827EA27483
:1046F000C27EE274827F84F823206575257510F8E8
:10470000562C2C3CA0F5E960D2070BD090F8F306AC
:1047100000F00F0084F86000608840F480606080E2
:10472000BDE8F08184F86010FAE710B50446FBF7A5
:10473000ABFD012C0BD15D48006890F8100180079B
:1047400005D5FCF7CCF838B1FCF7C5F804E0FCF768
:10475000C6F808B9FCF7BBF8BDE81040FBF792BDFE
:104760000020E2E7514B10B51A68947E640704D527
:10477000D28A0468A2EB040202601A68947EA4073D
:1047800003D5128B0C68121B0A600268002A00DA3B
:10479000002202601C68E48AA24200DD2246026018
:1047A0000A68002A00DA00220A601C68248BA242F0
:1047B00000DD22460A601B689B7EDB0702D003688F
:1047C0000B60026010BDF0B5384D002301242D6848
:1047D00095F8E85104FA03F635420AD031F913602E
:1047E00030F91370F61B32F91370BE4201DD01205F
:1047F000F0BD5B1C062BEDDB0020F0BDF0B5002505
:104800002C46059E0AE000BF31F9147030F914C03F
:10481000A7EB0C07974200DD6D1C641C9C42F3D390
:10482000B54201D30120F0BD0020F0BD2DE9F043D9
:104830009946DDE90787002423460DE031F913503E
:1048400030F9136005EB020C664503DAA5EB0905A8
:10485000AE4200DC641C5B1CBB42EFDB444502D96A
:104860000120BDE8F0830020FBE72DE9F04F8A46E8
:10487000DDE90997012547F6F8714E429346AC46AB
:10488000002424E030F814803AF81420A2EB080247
:1048900012B2914200DD1146964200DA1646002A15
:1048A00010DA4FF0000510E0442B01203C0210000C
:1048B000802B0120C025100098D00120D8261000A0
:1048C000EEFF010001DD4FF0000C04F10104BC42D9
:1048D000D8DB55EA0C0206D0012D01D02DB108E03D
:1048E000BCF1010F05D1002112E0BCF1010F00D194
:1048F0003146002905DD03EB0902B1EB420FF2DC82
:1049000006E005DA03EB09025242B1EB420FEADBA3
:1049100000252C462A4610E030F812603AF812C002
:104920000E44ACEB060636B29E4205DAC9F1000C25
:10493000664501DD3544641C521CBA42ECDB95FB34
:10494000F4F20A44002105E030F8113013442BF84A
:104950001130491CB942F7DBC5E4F0B5064600202A
:1049600004460546521C059F0AE000BF36F911C0F7
:104970009C4504DDA44502DD64460D460120491C2A
:104980009142F3DB3D60F0BD30B50268002513466F
:104990000AE000BF50F82540944201DD224602E0C3
:1049A0009C4200DA23466D1C8D42F3DBD01800EBED
:1049B000D07040106BE570B5B14B1B685C7D1B7D02
:1049C000641C5C43002307E032F8135030F8136096
:1049D000AD1B21F813505B1CA342F5DB70BD70B515
:1049E000A74B1C68247D611A10E0012409E02D7D8D
:1049F00004FB0515641C30F9156096FBF2F620F8EF
:104A000015601D686E7DA642F1DA491C1C68247D84
:104A10008C42EADC70BD9B49012008604FF4707144
:104A2000994818F020BF2DE9F041064615460F467B
:104A3000302801D1FFF7EFFF924C20682844401C3A
:104A4000B0F5707F01D2206801E0012020608E491E
:104A500008700E542DB10844401C2A463946FFF711
:104A6000A5FD20682844401C206059E687480021A5
:104A7000012201704270817070478448007870474D
:104A800030B57F4A126892F8FD26D3070BD0D506C1
:104A90007F4A4FF000034FF0010407D5151F28602F
:104AA000012901D11360F2E41460F0E4784D083D6F
:104AB00028600129F8D0F5E72DE9F84F704C002661
:104AC0004FF00057206890F8FD06450997F851000F
:104AD00000D101250720FBF7C2FDFBF778FEDFF8C8
:104AE000AC81C8F8080020684FF0010490F8FD067A
:104AF000C00603D5062087F8510001E087F8514031
:104B000000210120FFF7BCFF4FF41670FBF7C2FB3A
:104B10004FF0E02A4FF480594FF0000BCAF8809212
:104B20004FF040514446D8F80800FBF7D6FCDFF8B8
:104B30006481012088F80000E8B2FBF7B5FFCAF8ED
:104B400000916B4600224FF04051A068FBF7E6FC55
:104B50004FF04051A068FBF7C0FC0098C00000D5A2
:104B600001262078B04202D1607801280BD197F855
:104B700051009EB140EA0522DD20A16808F005F948
:104B800084F801B0267000210846FFF779FF88F805
:104B900000B00720FBF77EFD207805E540EA0521FF
:104BA000092008F0DAF8EBE710B504463A484FF46C
:104BB00080510160FBF785FF344821468068BDE8DD
:104BC0001040FBF75BBC70B52D48006890F8D01022
:104BD000CA0732491CD090F8D12002F00F02531CB2
:104BE0000A2B01D90A2200E0521C00F1D204002352
:104BF0004D8804E034F81360B5420CD05B1C93423E
:104C0000F8DBB0F84E274A80B0F8E8200A8002E0CE
:104C1000B0F84E274A8090F88023D2071DD090F834
:104C2000812302F00F02531C0A2B01D90A2200E053
:104C3000521C00F282350023CC8804E035F8136062
:104C4000B44209D05B1C9342F8DBB0F85C27CA8001
:104C50000A81B0F8AC03888070BDB0F85C07C880EA
:104C6000088170BD03004FF0000006D00B785B1E7A
:104C700013F0FF030B7001D101200A707047000090
:104C80003C02100040021000280801200803100018
:104C9000280A0022DF02100080E100E0D826100080
:104CA00010B501462022F948FFF780FCBDE810400E
:104CB0004FF400610120FBF7E1BB2DE9F0419AB010
:104CC00080460D4614466846FFF7A0FCE0074FF00B
:104CD000010701D0ADF80070A00705D5BDF80000B0
:104CE00040F00800ADF80000600608D5E849002053
:104CF0000870BDF8000040F48060ADF80000600767
:104D000033D5E44E306890F8FD06C0070DD0FFF7AC
:104D1000D3FE0621012805D0BDF8020040F00200B4
:104D2000ADF80200ADF8001005E0BDF8000040F05D
:104D30000600ADF80000A00711D1BDF8000040F05A
:104D40000100ADF80000306800F2211041788DF8C4
:104D5000171001788DF81E1080788DF82200CE484B
:104D60000088800501D58DF84970CC49ADF81A80CE
:104D7000ADF83A50ADF83450097840465A2905D17B
:104D8000C649491C09780844ADF81A00AFF2EF0093
:104D9000BE4D03244FF4006602906846FCF727FEE0
:104DA00019AB002231460120FBF7B8FB3146012048
:104DB000FBF793FB2878002804D0FEF7DAF8641E8E
:104DC000002CEADC1AB0BDE8F0812DE9F041B14ACF
:104DD000002421461268254610F4D17F04D092F8B1
:104DE000221004254FEA111110F0050F05D092F89A
:104DF000213045F001054FEA1314C00604D592F89E
:104E0000210045F0020504098C4200DA0C46641CBE
:104E1000002DD8D00026A24F05E0F98878882A46D0
:104E2000FFF74BFF761CA642F7DBCCE72DE9F047F6
:104E3000824698480068457D017D90F821006D1CF0
:104E400000F00F074D437F1C4FF48851954818F030
:104E50002CFD0024DFF84882DFF83092914E18E0F4
:104E6000B8F8061001225046FFF727FF8E49D9F8FF
:104E7000040006F00AFD8C49002007E056F82020C7
:104E800031F910301A4446F82020401CA842F5DBC6
:104E9000641CBC42E4DBBDE8F0872DE9F35FDFF87A
:104EA000F4818B46D8F80000457D017D90F8210003
:104EB0006D1C00F00F074D437F1C4FF4885179485B
:104EC00018F0F3FC0026774CDFF8D491DFF8BCA192
:104ED00019E000BFB9F8061001220098FFF7EDFEB7
:104EE0007149DAF8040006F0D0FC6F49002007E0B1
:104EF00054F8202031F910301A4444F82020401C86
:104F0000A842F5DB761CBE42E4DBD8F8000090F83E
:104F1000210000F00F01491C002006E054F8202079
:104F200092FBF1F22BF81020401CA842F6DBBDE802
:104F3000FC9F2DE9F34F574D87B08B462868182109
:104F400090F8210000F00F077F1C684618F0ADFCB8
:104F500000266C46DFF84891DFF830A1DFF84C817D
:104F600019E000BFB9F8061002220798FFF7A5FE66
:104F70004E49DAF81000FEF7F9FE00204FEA08016A
:104F800054F8202031F910301A4444F82020401CF5
:104F90000628F5DB761CBE42E4DB2868444E90F818
:104FA000210000F00F01491C002001222B6802FAA9
:104FB00000F793F8E8313B4207D054F8203093FBD8
:104FC000F1F32BF8103026F81030401C0628EDDBEA
:104FD00009B0BDE8F08F2DE9F74F2E4D84B0914612
:104FE000286830F83B1F039140880290FEF737FE97
:104FF0000090FEF75FFE019004216846FEF756FC24
:105000008046042101A8FEF751FC40444600286870
:10501000B10090F8220000F00F04641C214818F041
:1050200044FC296891F8F102C20706D0800704D435
:1050300091F8F202044406F025F80027DFF864B086
:10504000AA4644E01648042205994088FFF735FE39
:10505000DAF800100D4891F89417C568C90704D014
:1050600041692A46284606F0B9F8DAF8000090F8B7
:10507000F102C10707D0800705D40E49284606F083
:105080001DF818B30B4D002059461DE06047100075
:10509000570210003C02100050021000EEFF010009
:1050A000D8261000C0141000400D1000BC2A0120AA
:1050B00080D0012050AF012051F8202035F9103068
:1050C0001A4441F82020401CB042F5DB7F1CA74267
:1050D000B8DBDAF80010FD4C504691F8221001F0D0
:1050E0000F0303F101034FF000011CE05BF82120E6
:1050F000056892FBF3F295F8F1725FEAC77C08D07D
:10510000BF0706D595F8F2727F1C5743B5F8F32216
:10511000BA1AB1EB480F01DA039D00E0029D2A4460
:1051200024F81120491CB142E0DB049810F0220F52
:1051300009D02046D9F80010FEF797FD2046D9F88F
:105140000410FEF7B8FD07B043E72DE9F0479A4693
:10515000DF4B894600210125DE4E1C681BE000BFA5
:1051600032F8113030F81170DB1B1FB200230AE057
:10517000C3EB031C06EB8C0C5B1C3CF811801BB2D0
:10518000B8442CF8118094F880C305EB9C1C9C4516
:10519000EEDC491C09B2637D8B42E1DC0020CE4A83
:1051A00019E000BF3AF8103039F81010591A0BB254
:1051B000002108E002EB8116491C36F8107009B294
:1051C0001F4426F8107094F8806305EB96168E4203
:1051D000F0DC401C00B2217D8142E3DC5BE62DE97E
:1051E000FE4F00258246BA4C2F46DFF8E882DFF8F2
:1051F000E892012612E000BF00EB4500C5EB051266
:10520000B0F8B11308EB8200009009EB8510CDE9EE
:1052100001076A465046FFF7DEFE6D1C206890F8D5
:10522000801306EB9111A942E6DC90F85011C907F2
:1052300010D090F8911109060CD5407DA549420087
:10524000A648FFF7B3F92068A349007D4200A448AF
:10525000FFF7ACF9BDE8FE8FFEB59D4AA1490024D9
:105260001268012300F4907592F88063C98803EBFB
:10527000961306E002EB4406B6F8B163B14202D0E1
:10528000641CA342F6DCA34219DDC5B192F85001BB
:10529000C00703D192F82002C0070FD08D49C4EB9C
:1052A000041001EB80013C228F48FFF77FF98A4808
:1052B000402200EB84118D48FFF778F9FEBD0022F3
:1052C0000292894A0092894A01926A46FFF783FE58
:1052D000FEBD2DE9FC47FEF7C2FC0090FEF7EAFC9C
:1052E000019004216846FEF7E1FA0446042101A872
:1052F000FEF7DCFA764E204444003068A10090F8B6
:10530000220000F00F077F1C704818F0CEFA00252D
:10531000DFF8DCA1DFF8B491B04622E0714840220A
:10532000C1884088FFF7C9FCD8F80010DAF8186087
:1053300091F89417C90705D032463046DAF81410B0
:1053400005F04CFF0020494608E000BF51F820203E
:1053500036F910301A4441F82020401CA042F5DBF9
:105360006D1CBD42DADBD8F80000584E454690F877
:1053700022004B4600F00F00401C002107E000BF58
:1053800053F8212092FBF0F226F81120491CA1428B
:10539000F6DB58493046FEF768FC57493046FEF7C1
:1053A0008AFC286890F82010090711D5534C002179
:1053B0002160417D4F48FFF755F82168084420607F
:1053C0002868017D4C48FFF74DF8216808442060AB
:1053D000BDE8FC8770B504460020FBF740F90320C8
:1053E000FBF73DF93A4D286890F82010490701D4A1
:1053F00024F4006490F85011C90705D190F82012E8
:10540000C90701D124F0620490F88013490701D440
:1054100024F4B07490F8D010490701D424F00404A7
:1054200090F8E81109B924F0100490F8041309B9B0
:1054300024F4C07490F85002C00701D124F48064B1
:1054400060060BD52A483C2227497C38FFF7AEF886
:105450002748402225494038FFF7A8F8284900206E
:10546000401C8842FCD3200502D52046FFF7ADFC46
:1054700014F4907F02D02046FFF7B1FE194EE007EA
:105480004DD070881F49FFF708FD286890F820006C
:1054900000070AD51B48FEF7F0FE1B4901231B4AF3
:1054A000086001461748FEF71FFF286890F8490476
:1054B000C00734D01648007870BB16480078012821
:1054C00002D1204602F08AFE204626E0C0141000D9
:1054D0003C021000E814012014160120D815012008
:1054E00014170120D826100074130120B0130120D6
:1054F000604710005417012090170120EC041000A1
:1055000020A10700A8000120A002100038261000EA
:10551000780210009A03100001E002F044FFE00658
:1055200003D57088B349FFF704FD600501D5FFF787
:10553000D0FE14F0820F02D02046FFF78DFE6006E9
:1055400006D5AF49AC4BAD4AA1F13C00FFF7FDFDDC
:10555000AC4901200870AC49087007F0B9FA002086
:10556000FBF798F8BDE870400320FBF793B82DE9EE
:10557000F041A6490025A64A0968A64EB1F8B13304
:1055800083421AD291F880339C0901EB4407B7F8A3
:10559000B17387420AD9012404EB931313E000BFCF
:1055A00001EB4407B7F8B173B84201D1254602E0D8
:1055B00008D2A4F10105A5421CD191F85001C00701
:1055C00008D103E0641CA342EADCF6E791F820026C
:1055D000C0074CD0C5EB051002EB80013C22874888
:1055E000FEF7E4FF06EB8511BDE8F041402282485A
:1055F000FEF7DCBF01EB4405B5F8AF33B5F8B153A6
:10560000C01A0002EB1A90FBF3F391F85001C007A7
:1056100003D191F82002C00729D0784DC4EB0411C2
:10562000002002EB810100BF01EB400231F9107054
:1056300032F93C2CBF1A5F4302EB272225F81020D9
:10564000401C1E28F0DB6C4D002006EB841100BFCF
:1056500001EB400231F9104032F9402CA41A5C43AE
:1056600002EB242225F81020401C2028F0DBBDE8A6
:10567000F0812DE9F04168480124684E047000254E
:105680003560192000F0AAF8192000F08FF8644F57
:10569000052038724FF41670FAF7FCFD5F48443865
:1056A0000560FF21397034600460E0E770B55A4846
:1056B0005C4C01250570207F40F0040020775348A2
:1056C000006890F81101C00705D00A2000F086F8A4
:1056D0000A2000F06BF8002184F860105C22A276AA
:1056E0001120E07684F860505823A376E0764B4B87
:1056F000443B19604A4EFF213170042184F8601048
:10570000A276E0761D6070BD70B544480024443830
:105710000460434D08352E79192000F053F8C6F186
:10572000FB002978C0B2491CB0FBF1F03E4908707B
:1057300039490C703549096891F81111C90702D02F
:10574000BDE87040B2E7384A5521921E11703749C2
:10575000087070BD10B5334C207F40F004002077F6
:105760002A48006890F81101C00702D00A2000F012
:1057700029F82B490A7B294B0020443B186084F808
:1057800060005C23A3761123E3760978891A89B235
:105790004FF4FA42B2FBF1F1234A0909521E11708B
:1057A0005521521E11701C49087010BD00F01F02D7
:1057B0000121914040094FF0E02202EB8000C0F847
:1057C0000011704700F01F020121914040094FF085
:1057D000E02202EB8000C0F88011704700F01F0249
:1057E0000121914040094FF0E02202EB8000C0F817
:1057F0008012704768130120B01301207413012038
:105800002047100056021000C80210003C02100091
:10581000E814012014160120DE02100048050022C1
:105820002E00002000100020F4FF0100E102100013
:1058300010B501462022FC48FEF7B8FE8021BDE8E5
:1058400010400120FAF71ABE30B59BB004466846F6
:10585000FEF7DCFE0021012C02D0022C02D008E071
:10586000012000E00820ADF800008DF816108DF83A
:105870001410BDF80200AFF2470140F4A670EA4DE3
:105880000291ADF8020003246846FCF7B0F819ABAA
:10589000002280210120FAF741FE80210120FAF741
:1058A0001CFE2878002804D0FDF763FB641E002C42
:1058B000EADC1BB030BD2DE9FC5F4FF0000BFEF7BA
:1058C00029FA0446FEF732FAD84907460020086054
:1058D00048608860D6494FEA5409804608604860AD
:1058E00088604FF0010A0220FFF7AEFFCE48002487
:1058F00026460069CDF800000AFA06F010EA090F02
:1059000038D000250AFA05F1394230D0C9490AFADF
:1059100004F0096891F8E811014228D02946304680
:10592000FDF78AFEC349C14A096832F91430B1F85B
:105930000AC2B3EB0C01009B33F91430A3EB0C0C3F
:1059400000D54942BCF1000F01DACCF1000C6145F1
:1059500004DBB74922F8143021F814003F2805D29F
:10596000401CC2B229463046FEF7CEFA641C6D1CBC
:10597000202DC7DB761C272EBEDBFCF744FD08F18B
:105980000108B8F1400FAEDB012000900220FFF7C4
:105990005BFFD0460026DFF89CA2354608FA05F0EA
:1059A00010EA090F1ED0002408FA04F1394216D07B
:1059B000DAF8001008FA06F091F8E81101420ED06A
:1059C0009B48214610F81600019002462846FEF733
:1059D0009BFA01983F2801D300200090761C641C9C
:1059E000202CE1DB6D1C272DD8DB009810B9052099
:1059F000FDF7E2FAFCF707FD0220FFF725FF8A48D2
:105A00008D490069FEF7B2F9DAF800408A4D0020AE
:105A100094F8E831424600BF02FA00F10B421CD074
:105A200035F91010002902DC4BF0020005E040F6C9
:105A3000FF76B14203DB4BF00100834610E0B4F87F
:105A40000A72B4F8BE6107EB060C8C4505DABF1B81
:105A50008F4202DD0EB14BF0040B401C0628DBDB4D
:105A60005846BDE8FC9F2DE9F05F72490A6892F83C
:105A7000300105067148037803F00F0407D492F84B
:105A80003E1121F00F0121430170BDE8F09F002578
:105A9000DFF894A1834604702E4601278946022030
:105AA000FFF7D2FE6449DAF81000FEF75FF9D9F883
:105AB0000020614B002092F8E81100BF07FA00FCBB
:105AC00011EA0C0F05D033F910C0B2F80882C445B2
:105AD000DBDB401C0628F1DB0F2D08D26D1CEDB27C
:105AE00044EA0510761C8BF80000102ED7DBBDE8C9
:105AF000F05F0420FDF760BAF0B54B4900204D6817
:105B00004C490A68537D117D5B1C01FB03F41CE0CA
:105B100035F91130002B02DC40F0200014E040F693
:105B2000FF76B34202DB40F010000DE0B2F83471B2
:105B3000B2F8BE6107EB060C9C4505DABF1B9F421D
:105B400002DD0EB140F04000491C8C42E0DCF0BDAB
:105B50002DE9FF5F00200090FEF728F90446FEF7CC
:105B60002BF907464FEA540B4FF4F061344817F015
:105B70007AFE2D484FF027098021203017F095FE3E
:105B8000002002900120FFF75FFE2748D0F804A014
:105B900028480068047D0120002503907FE0012053
:105BA00000FA05F111EA0B0F78D00026012000FA67
:105BB00006F818EA070F67D01B48203050F8250078
:105BC00010EA080F5FD131462846FDF735FD0190F8
:105BD00018483AF914200068B0F834118A4246DCBB
:105BE000174830F91430581AA2EB010100D5404291
:105BF000002900DA4942884224DC01983146401EDF
:105C0000C0B2024601902846FEF77EF90C483AF9E8
:105C1000141030F91400401A01D5C0F100000099A9
:105C20000844009017E000008047100080D0012059
:105C30008CD001203C021000BC2A0120F6FF01009C
:105C400098D00120B949981A00D54042009B1844C9
:105C5000009021F81420B649019821F81400B548A5
:105C600050F8251041EA080140F825100BE0019892
:105C70003146401CC2B22846FEF746F9AB483AF816
:105C8000141020F81410641C761C202E8EDBA948FA
:105C900050F82500B84201D0002003906D1C4D45FE
:105CA000FFF67DAF039838B9FCF7ADFB0298401CB6
:105CB00002904028FFF666AF9F484FF0010A00258A
:105CC0000068067D1DE0012101FA05F010EA0B0FC6
:105CD00016D000240120A04038420ED0944821461E
:105CE00010F81600804602462846FEF70DF9B8F176
:105CF0003F0F01D34FF0000A761C641C202CE9DB17
:105D00006D1C4D45DFDBBAF1000F02D10320FDF71A
:105D100053F9FCF778FB0120FFF796FDFFF7ECFE47
:105D2000854D06462868017D427D90F8460751431F
:105D3000009A00F00F00B2FBF1F400FB04420021D6
:105D4000192007F022F8286890F8460700F00F00A5
:105D500000FB044000B2FEF728F9FEF72AF90246DC
:105D60000021202007F011F8304604B08DE62DE91F
:105D7000F05F714A116891F83001C4076F480378E9
:105D800003F0F00516D0057000264B7D0C7DDFF882
:105D9000A4A15B1CB046AAF1200A914604FB03F7BC
:105DA00083460120FFF750FD2046DAF80420D9F899
:105DB00000100EE091F83E1101F00F01294301702F
:105DC00063E600BF32F91030B1F832C16345F7DB4A
:105DD000401C8742F6DC0F2E0AD2761CF6B245EA4A
:105DE000060108F101088BF80010B8F1100FD8DB9C
:105DF000BDE8F05F0220FDF7DFB82DE9F05F002578
:105E000081468A464FF001082C46012803D0BAF19A
:105E1000010F3BD008E0BAF1010F24D0FDF7C6FF17
:105E20000546FDF7C9FF044600274FF0010B00BFF0
:105E30000BFA07F129420DD05FF000060BFA06F0CD
:105E4000204204D0002231463846FEF75DF8761C29
:105E5000202EF3DB7F1C272FEADBFCF7D4FAB9F105
:105E6000010F08D00DE04FF404614FF4F83017F043
:105E70001CFDFCF7C8FAFFF77AFFFFF769FE48EA56
:105E800000682D4CBAF1010F07D010E0FDF742FF7A
:105E90000543FDF74BFF2043C5E7206890F8E80174
:105EA00028B1FFF7E0FDFFF706FD48EA0048234868
:105EB0002268401D017892F8FB2701F0F00102F002
:105EC0000F0211430170B9F1010F04D04046BDE843
:105ED000F05F07F042B81A48FEF789F9404607F02C
:105EE0003CF8012000F01AFDBDE8F05F002000F052
:105EF00015BD02461821012000FA01F3134201D119
:105F0000491EF9D5491C88401043704710B54FF41D
:105F1000805421460B4817F0A6FC2246BDE81040ED
:105F20004FF4F8310748FEF741BB000098D001203C
:105F300018D80120A04710003C021000F6FF010015
:105F4000C0251000BC1A01202DE9F04F0020FF4DA4
:105F500004460246012140F6FF7BFD4BD5F8149024
:105F60006E681B6801FA02F737421CD039F914A099
:105F7000BAF1000F02DC40F0200013E0DA4502DB4A
:105F800040F010000EE0B3F836C1B3F84171E646B8
:105F90000CEB0708D04503DBAEEB070CD44501DD65
:105FA00040F04000641C521C202ADBD30024AF695F
:105FB000AE68224601FA02F535421AD037F914507C
:105FC000002D02DC40F0200012E05D4502DB40F0D5
:105FD00010000DE0B3F83A81B3F8439108EB090CD7
:105FE000AC4503DBA8EB090CAC4501DD40F04000FB
:105FF000641C521C202ADDD3BDE8F08F10B5014689
:106000002022D448FEF7D2FA8021BDE810400120BA
:10601000FAF734BA30B59BB004466846FEF7F6FA94
:10602000207801284AD0CA48016891F8FC06800708
:1060300005D5B1F85C07ADF83400ADF83A0091F839
:10604000FD064FF00604C00709D0FEF735FD012814
:1060500005D0BDF8020040F00200ADF80200ADF836
:10606000004000208DF846008DF84500B748416893
:1060700049000B9180680C90BDF80200AFF28301DB
:1060800040F4A670B34D0291ADF8020003246846B7
:10609000FBF7ADFC19AB002280210120FAF73EFA94
:1060A00080210120FAF719FA2878002804D0FCF79B
:1060B00060FF641E002CEADC1BB030BD4FF4806032
:1060C000ADF80000CDE72DE9F84F0446006A212124
:1060D00017F0C9FB3021606A17F0C5FB2046FCF7BA
:1060E00036FD2046FCF705FA0420DFF86082DFF871
:1060F00060A203254FF0000900902046FFF78AFFB9
:10610000E8072CD04FF0000B5F465E460120D8F820
:106110000410B04008421AD03046216AFEF73BF81E
:10612000D8F8141031F91720DAF80010B1F8451139
:106130008A420BDA00994FF0010B0844C1B23F29A3
:1061400000D93F213046226AFEF738F87F1C761CC2
:10615000202EDBD3BBF1000F01D125F00105A807EC
:106160002CD54FF0000B5F465E460120D8F8081092
:10617000B04008421AD03046616AFEF70CF8D8F8F1
:10618000181031F91720DAF80010B1F847118A42D7
:106190000BDA00994FF0010B0844C1B23F2900D936
:1061A0003F213046626AFEF709F87F1C761C202EDC
:1061B000DBD3BBF1000F01D125F0020555B120461C
:1061C000FCF7C5FC2046FCF794F909F10109B9F187
:1061D000640F92DB03254FF000092046FFF71AFFFA
:1061E000E80729D04FF0000B5F465E460120D8F843
:1061F0000410B040084217D03046216AFDF7CBFFAB
:10620000D8F8141031F91720DAF80010B1F8451158
:106210008A4208DD38B1401EC1B24FF0010B304652
:10622000226AFDF7CBFF7F1C761C202EDED3BBF14C
:10623000000F01D125F00105A80729D54FF0000B6B
:106240005F465E460120D8F80810B040084217D0DB
:106250003046616AFDF79FFFD8F8181031F9172012
:10626000DAF80010B1F847118A4208DD38B1401E53
:10627000C1B24FF0010B3046626AFDF79FFF7F1CF1
:10628000761C202EDED3BBF1000F01D125F00205D4
:10629000002D0AD02046FCF75AFC2046FCF729F9CD
:1062A00009F10109B9F1640F97DBBDE8F88F2DE919
:1062B000F04106460020F16908702121306A17F08C
:1062C000D2FA3021706A17F0CEFA3046FCF711F995
:1062D0003046FCF73CFC1D4D00273046FFF79AFE88
:1062E000D5E904320024204606E000BF32F9101040
:1062F000A14200DD0C46401C9842F7DB0020EB6811
:10630000AA6905E032F91010A14200DD0C46401CDC
:106310009842F7DB002C0BDCF06901780F2904D8D8
:10632000491C01703046FCF712FC7F1C202FD4DB87
:1063300040F6FE70844208DDF1690878401E08705E
:106340003046BDE8F041FCF702BC05E01403100044
:106350003C02100020481000BDE8F0812DE9F05FFC
:1063600004464068FD4A00250778A068D4F81480E8
:10637000D2F804C090F800902E462946012000BFB4
:1063800000FA01F313EA0C0F04D018F80130AB4205
:1063900000D91D46491C2029F2D3A369D2F808C0B0
:1063A0000021904600FA01F212EA0C0F03D05A5C69
:1063B000B24200D91646491C2029F3D3E068E849C7
:1063C000057020690670086890F8FD06C20708D0BD
:1063D0008B46800705D5FEF750FB012801D12078B8
:1063E00060B1E81906EB0901FF2288427DD2081A44
:1063F0002844FF286ED8E168087073E0DBF80000DD
:1064000000F5EB604279017902F03F0201EB0228CE
:10641000C2798179007802F03F0201EB022A40063E
:1064200009D508EB0A0105EB410006EB41023844AF
:1064300002EB090109E007EB450208EB0A0102EB58
:10644000410009EB460202EB4101FDF74AFADBF895
:1064500000100246B1F8FE36934201D2A1F8FE26A2
:1064600091F8FD26520731D591F85827520614D5D8
:106470004FEA48025342CAF1000203EB420291F88C
:10648000FE16E3681144C91B1970DBF8000090F890
:10649000FE061118A1EB090016E0B1F8FE3608EB74
:1064A0000A01CA19524203EB4202E368C2F34702EF
:1064B0001A70DBF80000B0F8FE2601EB090040423C
:1064C00002EB4000C0F3470021690870BDE8F09F6F
:1064D0000BE0FFE7E0680270D8F8001041F080019F
:1064E000C8F8001020690670F0E7814211D2401A06
:1064F0003044FF2802D82169087007E02069027043
:10650000D8F8001041F08001C8F80010E06805706C
:10651000DCE7E0680570E5E72DE9F041044600217D
:1065200045698E488E4B01224FEA010C476802FAFA
:1065300001F63E420AD01F686E5C97F84A71BE426F
:1065400002D9F61B6E5401E005F801C0491C202950
:10655000ECD3D4F818500021876802FA01F63E42C5
:106560000AD01F686E5C97F84A71BE4202D9F61BCA
:106570006E5401E005F801C0491C2029ECD32046E7
:10658000FFF7ECFE2046BDE8F041FBF7FBBF2DE92D
:10659000F14F2C210098D0E90565304617F063F9DA
:1065A0004021284617F05FF90098FFF7D7FE0098C2
:1065B000FCF7CDFA0098FBF7E5FF0324DFF8A0B164
:1065C0004FF0040A00270098FFF724FDA00752D0DF
:1065D0004FF0000961484B4649460122D0F804803B
:1065E00002FA01FC1CEA080F16D0D0F814C03CF9DE
:1065F0001380DBF800C0BCF838C1E0450BDA16F8B0
:1066000001C04FF00109D444BCF1FF0F01DD4FF090
:10661000FF0C06F801C05B1C491C2029DED3B9F130
:10662000000F01D124F001044FF0000C63466146D5
:106630004FEA0209D0F8088009FA01F212EA080FBD
:1066400011D0826932F91380DBF80020B2F83C21C6
:10665000904507DA6A5C4FF0010C5244FF2A00DDD6
:10666000FF226A545B1C491C2029E3D3BCF1000FB4
:1066700001D124F002045CB10098FFF76FFE00988E
:10668000FCF765FA0098FBF77DFF7F1C642F9ADB0F
:10669000032400270098FFF7BDFCE00728D04FF047
:1066A000000CDFF8B890614660464FF0010A00BF69
:1066B000D9F804800AFA00F212EA080F10D0D9F8CB
:1066C000142032F91130DBF80020B2F8382193425F
:1066D00005DD325C1AB1521E4FF0010C3254491CD8
:1066E000401C2028E4D3BCF1000F01D124F00104A8
:1066F000A00724D50022DFF86490114610464FF021
:10670000010A00BFD9F808800AFA00F313EA080F5B
:106710000FD0D9F8183033F911C0DBF80030B3F8D6
:106720003C319C4504DD2B5C13B101225B1E2B54D4
:10673000491C401C2028E5D30AB924F00204002C8F
:106740000BD00098FFF70AFE0098FCF700FA0098BB
:10675000FBF718FF7F1C642F9CDBA6E514031000D9
:106760003C021000F0B4C64B00210C461E6896F89F
:10677000302192070BD5426896F8496101211578BE
:10678000B54203D9A5EB0605157000E014701D682D
:1067900095F8302152070BD5826895F8495141F0A0
:1067A00002011378AB4202D95B1B137000E0147036
:1067B000002901D0F0BCD1E5F0BC70472DE9F047CD
:1067C000AF4E0446002531682F4691F8300182070C
:1067D000606802D50125077003E0227891F83F1127
:1067E0000170306890F83011490704D5A06845F071
:1067F0000205077004E02178A16890F84001087054
:10680000002D6FD02C21606917F02DF84021A06970
:1068100017F029F8E06921210770206A17F023F8A2
:106820003021606A17F01FF8E168FF2008702169C5
:1068300008702046FBF7A6FE2046FBF75AFE2046CE
:10684000FCF785F94FF01009DFF83882CA460027B7
:106850002046FFF7DFFBE80726D0D8E90423002015
:10686000014605E033F911C0844500DD6046491C4E
:106870009142F7DB3168B1F83621824206DA60686E
:106880004FF001090178491E01700DE0B1F84B117C
:10689000814207DB616808784844FF2800DDFF205B
:1068A000087001E025F00105A8072AD5002001465F
:1068B000D8F818C0D8F80C3006E000BF3CF9112019
:1068C000824200DD1046491C9942F7DB3168B1F87D
:1068D0003A21824207DAA0684FF0010A0178491E86
:1068E00001700EE018E0B1F84B11814207DBA1689E
:1068F00008785044FF2800DDFF20087001E025F0F3
:106900000205002D08D02046FFF728FD2046FCF7A1
:106910001EF97F1C202F9BDBBDE8F0872DE9F0419D
:10692000DFF864818AB0012188F8001005468DF8EF
:1069300000006846FDF749FA524C00262660FDF734
:106940008EF96060FDF7B6F9A06060680421400828
:106950006060201DFCF7AAFF2061042104F10800FB
:10696000FCF7A4FFE0606846FFF754FB4748012DA1
:106970004ED0C0686061A061D4E9040101EB400120
:106980006161E16801EB4000A16901EB4000A06199
:106990006846FFF713FF6846FFF7E4FE384F386894
:1069A00090F83001800605D56846FFF7F0FD68468F
:1069B000FFF7B2FD386890F83001000702D568464D
:1069C000FFF775FC386890F83001C00602D56846BC
:1069D000FFF779FB6846FCF7BAF86846FFF71AFB41
:1069E000FFF7B2FA014620680843206028493A6858
:1069F000012D0B7892F8FB2763F303020A7009D08C
:106A000040F0020006F0A9FA88F800600AB09CE4A1
:106A10008069AFE740F00E00F4E72DE9F041184C33
:106A2000206890F8FC06800729D5FEF745F8012874
:106A300025D12068A04600F25C7004888178C07877
:106A400000F03F0001EB00251148801E0778801EF2
:106A50000678FBF7F3FBD8F80010B1F8723791F81D
:106A60000F26B1F8FE162344414391FBF2F02B446C
:106A700033443B440749C01A2044C880088164E479
:106A80003C02100014031000850210002048100082
:106A9000FBFF0100D826100010B501462022A748B0
:106AA000FDF784FD8021BDE810400120F9F7E6BC28
:106AB000F0B5A34E05460C4630689BB090F8B10087
:106AC00000F00F01491C4FF0FF308840C743684673
:106AD000FDF79CFD0120ADF80000ADF802403068E4
:106AE00010F8F91F8DF8171044F00501ADF80210E9
:106AF0000397ADF81A50AFF25F01029141788DF81B
:106B0000181080788DF81E008E4800785A2805D11C
:106B10008C48401C00782844ADF81A00874D0324A7
:106B20006846FAF764FF19AB002280210120F9F7CB
:106B3000F5FC80210120F9F7D0FC2878002804D04A
:106B4000FCF717FA641E002CEADC1BB0F0BD2DE93F
:106B5000FC5FDFF8ECB14FF0000AD146DBF8000033
:106B6000564600F57070017890F8018080780190A9
:106B70004FF00850D0F88C0100B9012600208CB2EB
:106B8000009037E0DBF8000090F8CD0300EB8000C8
:106B90004700002524E020460099FFF789FF674859
:106BA00040680FF03AF80146DBF8000090F8F82052
:106BB00012F00F0000D1012012094A43B2FBF0F09D
:106BC0001FFA80F9012E09D1BAF5707F06D25E4A0C
:106BD0000AF1010022F81A901FFA80FA6D1CADB27A
:106BE000BD42D8D94A462146302006F0FFF9019827
:106BF000204484B24445C5DDBDE8FC9F2DE9FF5F1C
:106C00004FF6FF764FF0000A93460F468046344613
:106C10005546DFF82C911BE038F815005146FFF778
:106C200047FF464840680EF0F8FFD9F8001091F889
:106C3000F82012F00F0100D1012112094243B2FBEA
:106C4000F1F080B2A04202D238F8156004466D1C03
:106C5000BD42E1DBABF8006003980480BDE8FF9F14
:106C60002DE9F041364E05468846306888B090F8E8
:106C7000D12002F00F01C2F30214491C641C0A293E
:106C800000DD0A21022C00DD0224D23006AB05AA69
:106C9000FFF7B4FF326892F8D00080071BD5BDF82B
:106CA00014600121E632ADF8006000204FF4803C12
:106CB0006F4607E013563344634502D227F811307C
:106CC000491C401CA042F5DB002904DD06AB05AAE7
:106CD0003846FFF793FFBDF814002880BDF8181060
:106CE000A8F8001008B0BDE8F0817CB50020F9F7E5
:106CF000B6FC164C01A968466588FFF7B1FF10483D
:106D00000068B0F8E810BDF80400814201D9218084
:106D100000E02080BDF8000060800020F9F7BAFC98
:106D20000B49012008700B4908700B490870BDF829
:106D300000202946092006F036F97CBD40481000A5
:106D40003C021000EEFF010018D80120D8261000E8
:106D500056021000C8021000D80210002DE9F047BA
:106D600006460078FE4D00B1287020223146FD48CD
:106D7000FDF71CFCFC4C206890F89417CA07F949F1
:106D800001D04A6900E0CA68F64B417D686820334B
:106D9000414300201AE000BF97F8F1C25FEACC78C7
:106DA0000DD05FEA8C7C0AD597F8F27232F810C0E9
:106DB0007F1C0CFB07FC0F1823F817C005E001EB44
:106DC000000C32F8107023F81C70401C276897F8EC
:106DD00015C08445E0DC686800F1010068607F7DD3
:106DE00007FB00FC4FF000001EE000BF91F8F182AD
:106DF000C1465FEAC8780FD05FEA89780CD507EB07
:106E0000000891F8F21232F81880491C08FB01F8CA
:106E10000CEB000123F8118039180CEB000832F854
:106E2000111023F81810401C216891F81580804536
:106E3000DCDC6B684FF0010803F101036B6091F833
:106E4000B10008EB101291F8F102C70705D08707CF
:106E500003D491F8F2723A44D2B2934227DA91F80D
:106E6000FD06C00719D0FDF708FE012815D12168DD
:106E7000A88891F8B91380B201F00F01B0FBF1F2CC
:106E800001FB1201B74864380029418802D041F063
:106E9000020101E021F002014180307808B1FCF7E5
:106EA00068F8BDE8F047AF486438FAF7A0BDC207FC
:106EB0002FD080072DD4B1F8F3A2002522E0417D28
:106EC000A8486943203000EB41018946002014E0C6
:106ED00093F8F232012231F910605B1C06E000BF2A
:106EE00002FB070C521C31F91CC066449342F7DCCC
:106EF000A6EB0A0229F81020401C23685F7D874218
:106F0000E6DC6D1C206890F8B11008EB1111A94265
:106F1000D5DCBDE8F04780210120F9F7AFBA2DE9B3
:106F2000FF4FDFF840B24FF6FF74002681B08A466B
:106F3000A046ABF1640BB1466DE08A486438FDF7BA
:106F400065FB894D286890F8FD06C00708D0FDF75D
:106F5000B3FD28B9BBF8021041F00201ABF80210F2
:106F6000296891F89407C00701D0102200E002229E
:106F7000ABF80020019830F81620ABF83420BBF8AD
:106F8000022042F00402ABF80220AFF22F2201F2FD
:106F9000C931CBF808200A788BF84420CA788BF8DE
:106FA00046204A788BF84A206D4D89788BF8381046
:106FB0000327C5F8049000BF6A4885F8009064383C
:106FC000FAF715FD6B46002280210120F9F7A6FA99
:106FD00080210120F9F781FA287820B1FBF7C9FF59
:106FE0007F1E002FE8DC5F48203003F0B2F95E49D5
:106FF000096891F8C82312F00F0100D1012112098C
:10700000424390B2B0FBF1F0A04203D20199044692
:1070100031F81680761C56458FDB0398A0F8008067
:107020000498048005B0BDE8F08F2DE9F0414E4D85
:107030000646884628688CB000F2823C00F29637FB
:1070400090F8810300F00F01C0F30214491C641C86
:107050000A2900DD0A21022C00DD02240AAB09AA5C
:107060006046FFF75CFF286890F8800380071AD518
:10707000BDF824300121ADF8003000204FF4803CF1
:107080006D4607E03A561A44624502D225F81120AF
:10709000491C401CA042F5DB012904DD0AAB09AA0A
:1070A0002846FFF73CFFBDF824003080BDF82810CB
:1070B000A8F800100CB0BDE8F0817CB50020F9F70D
:1070C000CEFA2A4C01A96846E588FFF7AEFF2648AC
:1070D0000168BDF80400B1F8AC23824201D9A28056
:1070E00000E0A080BDF80000E0802081854205D04E
:1070F00091F88013490701D5FEF739FA1C490120A0
:1071000008701C4908701C49002008601B49087061
:10711000F9F7C0FABDF8002029460A2005F043FF20
:107120007CBD2DE9F843DFF840800E4CD8F8000014
:10713000643C00F2C3300588468807794EE0094870
:107140006438FDF763FAD8F8000090F8FD06C00730
:1071500017D0FDF7B1FCA0B9608840F002000FE045
:1071600030031000C44810003C021000D826100064
:1071700056021000C8021000580410004C04100001
:107180006080D8F8000090F89407C00701D0102064
:1071900000E002202080A586608840F00400608026
:1071A000AFF24740A0600F48002141600E48FAF757
:1071B0001EFC6B46002280210120F9F7AFF98021E7
:1071C0000120F9F78AF90848843003F0C2F8024632
:1071D0002946312005F00AFFE81985B2B542AEDD37
:1071E000BDE8F88330031000604810002DE9F0413D
:1071F000174604460D46002609E0E00703D0314655
:10720000384605F008FE761C6D084FEA340454EA4F
:107210000500F2D1BDE8F08130B5034600204FF003
:10722000FF32012505FA00F40C4202D0521C9A42AA
:1072300003D0401C2028F5D3002030BDF0B50E4609
:107240000125074605FA06F2FE4C0F2FD4E915106A
:1072500065D2DFE807F064434B0810646419212904
:10726000323A54585C003046FFF7D6FF8540A06A9A
:107270000543A56253E001463046FFF7CDFF854048
:10728000206C054325644AE03046FFF7C5FF854082
:10729000E06A0543E56242E03046FFF7BDFF854006
:1072A000206B054325633AE001463046FFF7B4FF03
:1072B0008540A06C0543A56431E03046FFF7ACFF84
:1072C0008540606B0543656329E001463046FFF762
:1072D000A3FF8540E06C0543E56420E03046FFF7FE
:1072E0009BFF8540606A0543656218E001463046B1
:1072F000FFF792FF8540E06B0543E5630FE0A06B6D
:107300000243A2630BE0206D0243226507E00146C1
:107310003046FFF781FF8540606C05436564206857
:10732000401C2060F0BD10B501462022C648FDF784
:107330003DF98021BDE810400120F9F79FB810B554
:10734000FCF780FC0446FCF7F1FC204310BD10B5AF
:10735000FCF76AFC4408FCF7DDFC44EA50004000FE
:1073600010BD2DE9F047894605464FF0FF34FFF781
:10737000E6FFB44F024600207B6801464FF0010C47
:107380000CFA01F6164200D0641CAC4206D1B9F1E9
:10739000010F09D022EA06000B462021491C2029B2
:1073A000EED37B60BDE8F0873046F5E72DE9F04786
:1073B000894605464FF0FF34FFF7C9FFA14F02464B
:1073C0000020D7F8043001464FF0010C0CFA01F60A
:1073D000164200D0641CAC4206D1B9F1010F08D0AE
:1073E00022EA06000B461E21491C1E29EED97B60AD
:1073F000D8E73046F6E72DE9F34F9FB004466846DC
:10740000FDF704F919A8FBF7DDFBFFF7A0FF8D4E90
:1074100040087065FFF793FFDFF830928C4D4FF016
:107420000C0809F1010A4FF01F0BB065012C0DD0BB
:107430000627022C2ED0032C32D0042C35D0052C5C
:107440003CD0062C5AD0082C71D08AE0FCF7AEFC58
:107450000390FCF7B1FC04900120ADF80000ADF8FA
:107460001A8099F800005A2804D19AF800000C30CC
:10747000ADF81A0040208DF8170095208DF81E00F9
:107480003C20ADF81C0003988DF818B040087065DA
:10749000049865E0FFF75BFF0B90FFF750FF14E0E7
:1074A000FFF74DFF01210C9003E0FFF748FF00219B
:1074B0000C902098FFF77AFF0B9007E0FFF747FF4B
:1074C0000B9001212098FFF74CFF0C90ADF8007055
:1074D000286800F55A7081788DF84410C1788DF8CD
:1074E0004A1001788DF8381041788DF83E10818867
:1074F000ADF834100089ADF83A0032E0FFF727FF0D
:107500000B90FFF71CFF0C90ADF80070286800F29C
:10751000613081788DF84410C1788DF84A10017877
:107520008DF8381040788DF83E001AE0FFE708200B
:10753000ADF80000ADF81A8099F800005A2804D17F
:107540009AF800000C30ADF81A0040208DF81700B2
:1075500095208DF81E008DF818B0099870650A986E
:10756000B0650020BDF802108DF8140021F0300144
:107570008DF846008DF8160041F04A018DF845005F
:10758000ADF80210AFF2612103260291012C12D056
:10759000092C23D00A2C21D08DF86E008DF87000B4
:1075A0008DF86F00022C10D0032C0ED0042C0CD0C0
:1075B000052C0AD012E0296891F84D178DF8680063
:1075C00041F003018DF86410E6E72868B0F86E1307
:1075D000ADF86A10B0F87203ADF86C0019A8FBF7AB
:1075E00011FB194C6846FAF702FA1DAB0022802104
:1075F0000120F8F793FF80210120F8F76EFF207833
:10760000002804D0FBF7B5FC761E002EEADC21B082
:10761000BDE8F08F2DE9FC5F00210120FFF7EBFEB4
:1076200009484768FCF7C2FB0190FCF7C5FB0090D6
:10763000042101A8FCF73AF9064604216846FCF744
:1076400035F907E03803100064501000EEFF010028
:107650003C021000844600200546DFF838B5DFF80C
:1076600038A5009054E000BF4FF00008C1465C46CA
:107670002846DBF85810FFF7CFFD0146012088406F
:10768000A16C084243D1012432E000BF04FB0C513D
:10769000DAF8000037F9112090F86703B2EB001F09
:1076A00025DA08F10108B9F1000F00D1A146721ED8
:1076B00094421CD1B8F1010F19D1ACF101029542ED
:1076C00004D1611E0120FFF7B9FD0EE007EB410177
:1076D000B1F90220B2EB001F05DB35B131F9021C14
:1076E000B1EB001F01DA002000E002208046641C9C
:1076F000B442CBDBA6EB0901414508D8294602205C
:10770000FFF79CFD01200099A840084300906D1CE4
:107710006545A9DB01253AE04FF0000844462CE01E
:10772000DBF84030DBF8482000201A4311D0D9465E
:107730002046DBF85810FFF76FFD01460120884016
:10774000D9F84810084203D1D9F84010084000D0B9
:10775000012005FB0C4137F91120DAF8001091F8EF
:107760006713B2EB011F07DA30B901200099A0407E
:10777000084201D108F10108641C6445D0DBB8F16E
:10778000000F03D0691E0120FFF758FD6D1CB542A4
:10779000C2DBBDE8FC9F2DE9F041FE4C0020054610
:1077A000FE4FDFF8F483A0611EE029460520FFF7B5
:1077B00022FE21690120FE6800EB410C36F91C1005
:1077C000D8F8000090F87703B1EB001F03D92946E1
:1077D0000E20FFF733FD36F91C00A169884202DD57
:1077E00036F91C00A0616D1C60698542DDD311E58E
:1077F0002DE9F0470026374631460820FFF7FBFD0C
:10780000E648E54D0021D0F810C02868012400F5B5
:10781000F57990F8E82100BF04FA01F31A4208D084
:107820003CF9113090F87D83B3EB081F00DA761C29
:107830007F1C491C0629EFDBBE420BD190F8E611F4
:10784000C90790F8E91101D00D2000E00C20BDE837
:10785000F047F3E4002E1CD00026286804FA06F254
:1078600090F8E811114211D03CF9161090F87D23E0
:10787000B1EB021F0ADA90F8E60119F80610C0070A
:1078800001D00C2000E00D20FFF7D8FC761C062E5E
:10789000E3DB87E52DE9F04100210620FFF7ABFD92
:1078A000BE480025BC4EBB4CC7680EE0E06831689E
:1078B000284437F9100091F86513B0EB011F03DD80
:1078C00029460A20FFF7BAFC6D1C20698542EDDBD2
:1078D00000250EE0A0683168284437F9100091F8BF
:1078E0006613B0EB011F03DD29460B20FFF7A6FC52
:1078F0006D1C60698542EDDB8CE42DE9F041A54CFF
:1079000000200646206237E031460420FFF773FD71
:10791000A2480025C7682BE0FFF711FD0146284665
:10792000FFF77AFC014601208840216C08421ED1F5
:107930009949A0682844096807EB400030F9040C15
:1079400091F87813B0EB011F07D931460820FFF7F3
:1079500075FC29460920FFF771FCA068216A2844BC
:1079600007EB400030F9040C884200DD20626D1CFA
:1079700060698542D0D3761C20698642C4D349E42D
:107980002DE9F041834C00200546844FDFF8088242
:10799000E0611AE029460320FFF72DFDFE68B6F9E5
:1079A0000210D8F8000090F87603B1EB001F03D95D
:1079B00029460720FFF742FCB6F90200E169884238
:1079C00002DDB6F90200E0616D1C20698542E1D359
:1079D00020E42DE9F04100210220FFF70CFD6F4863
:1079E0006D4D6C4CC768286890F86003000713D58C
:1079F00000260EE0E0682968304437F9100091F85D
:107A00007413B0EB011F03D931460320FFF716FCB6
:107A1000761C20698642EDDB286890F86003C0067A
:107A200013D500260EE0A0682968304437F910000D
:107A300091F87513B0EB011F03D931460420FFF70D
:107A4000FDFB761C60698642EDDBD0E62DE9FC414A
:107A50000020F8F704FE4FF4F83040F6FB7115F003
:107A600002FFFAF7D6FDFAF79DFDFAF7CCFC494C78
:107A700000202060FFF76BFC0090FFF760FC019096
:107A800004216846FBF712FF0546042101A8FBF715
:107A90000DFF014600EB4500C4E90205C4E90451AD
:107AA0003D4D286890F86003010701D4C00601D558
:107AB000FFF78FFF286890F86003800601D5FFF775
:107AC0005FFF286890F86003000601D5FFF715FFF7
:107AD000286890F86003C00701D0FFF7DBFE286834
:107AE00090F86013490704D590F8E80108B1FFF752
:107AF0007FFE286890F86003400601D5FFF74BFE33
:107B0000286890F86003800701D5FFF783FD20689F
:107B1000002862D0D4E90A359D43E562606AD4E961
:107B20000F179843A8436062666CB943B143E163A1
:107B3000A26B216D9A43AA43256BB943AA43A26362
:107B4000A26CB1439143AB43A362216501220021A2
:107B5000FFF74CFB02220021E06BFFF747FB0322FB
:107B60000021A06AFFF742FB04220021206CFFF7EE
:107B70003DFB07220021E06AFFF738FB08220021C5
:107B8000206BFFF733FB09220021A06CFFF72EFBCF
:107B90000A2205E0380310003C0210006450100077
:107BA0000021606BFFF722FB0B220021E06CFFF746
:107BB0001DFB0C220021A06BFFF718FB0D220021FA
:107BC000206DFFF713FB0E220021606CFFF70EFB08
:107BD0000020F8F75FFDBDE8FC810021084605F0B4
:107BE0001AF9F5E7F0B5FE490B6893F802120A0995
:107BF000002100B90022002093F8E851F94E012439
:107C000004FA00F73D4206D036F91070B3F84AC3C3
:107C1000674500DD491C401C0628F1DB0023F248C3
:107C2000002908DD0169914202D2491C016103E08B
:107C300003610120F0BD03610020F0BD70B5E8498B
:107C4000002209684C7D0B7D651C5D43194603E0ED
:107C500030F91160491C3244A942F9DB5C4392FBC4
:107C6000F4F000B270BD2DE9F04F95B000220D92F6
:107C70000020DE4C0892139215461292D84B1090B9
:107C8000DB4A0392610C1E6820468B461496D94647
:107C900082460222777D23E00123561E36B20F96DC
:107CA000149E96F814C0E646ACF1010C15E000BF36
:107CB00002FB0E36DFF83C8338F916608E4208DC92
:107CC000DDF83C80CDF834800FFA83F83146CDF8EA
:107CD0002080864200DB30465B1C9C45E8DC521C61
:107CE0009742D9DC401A00B2BD4E0021149009E041
:107CF000039830F91100484500DA8146504500DD0F
:107D00008246491CB942F3DB0121BB48FCF718F954
:107D10003168087D00EB4002B74800EB8200827BAF
:107D2000037C1A444FEA5202C2734A7D087D96468C
:107D3000A2F101024FF00103059229E00122A0F116
:107D4000010621E003FB002CAB4F17F80C806744C1
:107D50007F78B8EB070701D4BC4601E0C7F1000CFF
:107D600091F8588408F00308C4450CDDDDF848C0DC
:107D7000002F0CF1010CCDF848C000DA7F42DDF88D
:107D80004CC067441397521C9642DBDC059A5B1C7F
:107D90009A42D3DCB1F86E32149A934237DA0EF17C
:107DA000010646430346954F0AE000BF37F913200A
:107DB0001544A24200DD14465A4500DA93465B1C86
:107DC000B342F3DB0EFB00F295FBF2F0B1F8D136D3
:107DD00000B2534503DCB1F8CF364B4501DA002041
:107DE00014E091F85824C2F38303129A934204DA00
:107DF00091F8592413998A4204DB221AA0EB0B0054
:107E0000824204DA08990D98FCF774F910901098E2
:107E100015B0BDE8F08F70B5010071484FF0000655
:107E2000006890F85A5400D1002590F849040006E3
:107E300009D56D4C607B30B9FFF715FF0146002076
:107E4000012902D0E070304670BDE178A94202D22B
:107E5000491CE170F7E7E0700126F4E710B5012056
:107E6000FFF7D9FF0446012815D1654840F6050201
:107E70000168114301605C4900200122C8728872C8
:107E80000A7388735F48016841F4006101609102E0
:107E90001046F8F7F3FA204610BD2DE9F041010035
:107EA0004F48564F4FF000060068027D437D90F822
:107EB000545403FB02F3B0F84C4407EB420732463C
:107EC00000D10025002106E037F911C0A44501DDED
:107ED000521C02E0491C9942F6DB90F84904400626
:107EE00012D5414C607B78B90027002A0BDDFCF7E6
:107EF000F2FA40B1A078A84202D2401CA07003E080
:107F0000A770012600E0A7703046BDE8F08110B5EB
:107F10000120FFF7C2FF0446012816D1384840F679
:107F200005020168114301602F490120C872002039
:107F30008872087388733348016841F400610160F6
:107F40004FF480610120F8F799FA204610BD2DE921
:107F5000F0432349DFF898C000260C68BCF90030D4
:107F60008146B4F8981647F6FF75324630468B4284
:107F700000DD0122677D0CEB470333F9023C8B42A5
:107F800001DD42F00202DFF8608098F808108A42B2
:107F900018D1BAB10223BF1E09E000BF3CF913108B
:107FA000A94200DA0D46B14200DD0E465B1C9F423D
:107FB000F4DCB4F89A16B14204DDB4F89C16A94278
:107FC00000DA012088F80820B9F1010F07D1012853
:107FD0001CD094F8971601F07F0188F8091013E07F
:107FE0003C021000BC2A0120940310000080FFFF17
:107FF00054170120A8000120D0A70120400D100037
:10800000480210004C021000BDE8F08398F80910F7
:108010000029E4D0491E88F809100020DFE72DE987
:10802000F84F0446FE480025016891F8462791F86C
:108030006A9491F869A402F00F02072A02D947F660
:10804000FF7603E0521CC2EB023216B291F815C063
:10805000087DB1F84CB4B1F84A240092F14A0027E7
:1080600002EB400E0CFB00FC3B463A460CB9B9460D
:10807000CA46002010E000BF3EF910405C4500DD1C
:108080007F1CDDF80080444500DA5B1CB44200D060
:108090000CB9521C92B2401C6045EDDB91F864C4EF
:1080A000DF4E0020E04C94450AD26278521CD2B2D6
:1080B00062704A4505D9607020700120BDE8F88FD4
:1080C00060709F4227DD2278524503D202F10102FF
:1080D000227027E02070607091F84904400716D59F
:1080E000D248FCF71FFA05000ED1306890F8491409
:1080F000C90617D5CD49B0F8BC010968884211D925
:108100005846FBF7AFFA0546012D01D00AE00125DC
:10811000607B10B106E0207004E0FCF7C5F901288F
:1081200000D100252846C9E72DE9F05FBE4C0026A6
:10813000BB4FE079BE4DDFF8FC824FF0010A40F6FC
:1081400005094FF4806B01281ED1386890F8E811BA
:10815000D1B190F8FC01000616D50120FFF742FDD1
:10816000012811D105F08EF8286840EA090028603E
:1081700084F806A0D8F80010012041F40061C8F886
:1081800000105946F8F77AF96079012823D1FFF7F2
:1081900046FF0646386890F89706000605D5012088
:1081A000FFF7D5FE08B1012601E0012E13D12868A2
:1081B00040EA0900286084F80AA000202073E072D9
:1081C000A073D8F80010012041F40061C8F8001035
:1081D0005946F8F753F93046BDE8F09F2DE9F047CE
:1081E0000024954E954FDFF840920125A0460121CD
:1081F0000020FDF702FE70889149FCF79AFE3D7061
:108200000020FFF7EFFC10B1022C07D008E040F28D
:10821000C11004F0A2FE13F062FF07E089F80780A6
:108220000020FAF7C9FE641C032CE0DB89F8068005
:10823000BDE8F0872DE9FF4F7949002422460D68FB
:108240007849A0462E7DA14601EB460103917D4968
:1082500002917D49019195F8C27647F6FF710B4670
:10826000A34607F07F0A009708B94FF0000A687D1F
:108270000027864600FB06FC09E0039830F917004A
:10828000984200DA0346A04200DD04467F1C6745A1
:10829000F3DBF446002709E0029830F91700884222
:1082A00000DA0146904200DD02467F1C6745F3DBA1
:1082B000002709E0019830F91700884200DA0146EA
:1082C000904200DD02467F1CB742F3DBB5F8C306DF
:1082D000A04209DDB5F8C506984205DAB5F8C7062B
:1082E000904201DA4FF00109B5F8C906904209DD64
:1082F000B5F8CB06884205DAB5F8CD06A04201DA1A
:108300004FF00108009800060AD54748817B39B92B
:108310000021B9F1010F06D0B8F1010F03D00171AE
:10832000584604B075E50279524502D2521C0271DA
:10833000F6E701714FF0010BF2E770B538480268BB
:1083400092F8460700F00F00072802D947F6FF739E
:1083500003E0401CC0EB003003B2107D547D314976
:10836000444301EB40050021084607E035F9106061
:108370009E4200D00EB9491C89B2401CA042F5DBD8
:1083800092F86434002228488B4209D24178491C73
:1083900011F0FF01417004D042700270012070BDE5
:1083A0004270002070BD2DE9F0471F4C0027A07AD5
:1083B00001280BD0E07A012808D0607B012805D085
:1083C000207B012802D0A07B012875D10026DFF890
:1083D00050804FF6FF7AB146607B0025012802D11C
:1083E000FFF7ABFF0546A07A012804D11DB9002094
:1083F000FFF715FE0546E07A01280AD1D8F80000FB
:1084000090F84904400604D51DB90020FFF745FD4A
:108410000546207B01281CD1DDB9002016E00000B4
:108420003C021000400D100094031000A402100044
:10843000480210004C021000D82610008C041000D6
:1084400068130120442B0120802B0120FFF7E3FC5F
:108450000546A07B012804D11DB90020FFF7EAFEE4
:108460000546D8F8000090F89706000603D50020CE
:10847000FFF76DFD00B905B3012700213846FDF770
:10848000BCFC294829494088FCF707FDFCF721FF7F
:108490002020FCF7A4FE0220FCF7DEFE761C032E53
:1084A0009ADB84F805905246DD21992004F06DFC9A
:1084B0000020FAF781FD0EE015E0C12040EA072018
:1084C00004F04BFD012F06D15246CC21992004F037
:1084D0005CFC13F004FE84F80A9084F80B9084F896
:1084E0000D9084F80E90A3E610B50120FFF7A2FED0
:1084F0000446012816D10E4840F6050201681143D2
:1085000001600C490020C8728872087301208873CA
:108510000948016841F4006101604FF48061012065
:10852000F7F7ACFF204610BDD8261000A8000120A8
:1085300048021000940310004C02100008B5DFF848
:108540001492854E0127DFF81482854D002430787F
:1085500080B10128FBD16B4600224EF27D71F7F706
:10856000DDFF0098C1071DD001210846F7F7B5FFD0
:108570003470ECE701210020FBF71FFC6B46002262
:1085800002210120F7F7CAFF01210846FBF715FC7D
:1085900000988007DBD54EF27F710120F7F79DFF31
:1085A0003770D4E701071CD508210120F7F795FFA4
:1085B0000020F8F754F80620F8F751F80121084692
:1085C000FDF71BFCDFF89CA16749BAF80200FCF735
:1085D00064FCBAF802006549FCF7ABFC644807701C
:1085E0000EE0410713D504210120F7F776FF0020A4
:1085F000F8F735F80620F8F732F80020FEF78EF984
:108600000620F8F747F80020F8F744F89FE7C1067E
:108610000AD510210120F7F760FF99F80000002823
:1086200095D1FEF762FB92E781060AD52021012051
:10863000F7F753FF99F80000002888D1FEF73DFDB9
:1086400085E7C10507D54FF480710120F7F745FF95
:10865000FEF77DFA7BE7810507D54FF40071012015
:10866000F7F73BFFFEF75DFD71E7410606D54021B8
:108670000120F7F732FFFFF7E9F968E7010407D5B2
:108680004FF400410120F7F728FFFDF73FFC5EE7BC
:10869000410554D54FF480610120F7F71EFF35489E
:1086A00004602888800505D43348006890F8FC06EB
:1086B00080070AD50020F7F7D2FFF9F7BFFD7080D9
:1086C000FEF7ABF90020F7F7E5FF2C48D0F800A043
:1086D00004605046FCF77EFEB8F80000C00501D5E6
:1086E000274807705FEA8A7001D500F0B7FBAAF54A
:1086F000E061B73905D1052004F02FFCC8F800402F
:1087000012E05FEACA7008D0D8F8000040F0150007
:1087100004F023FCC8F8004019E71AF0420F05D016
:10872000286840F0060007E02C6010E75FEA4A5036
:1087300086D5286840F4806004F00FFCF4E78004DC
:1087400088D54FF400510120F7F7C7FEFCF791FFE1
:10875000FDE6000067021000A80310004C021000A4
:1087600050021000D8261000A80001206813012034
:108770008C041000680410003C0210004802100035
:108780006902100070B5FF4800240470FE480470B0
:10879000FE480470FE480470FE4804700120FE4943
:1087A000FF4D0870FD4908702C616C61AC802C7025
:1087B000FF20EC61E880FB480068B0F85211A98105
:1087C000B0F8540168813C21F74815F04CF840217D
:1087D000F64815F048F83C21F54815F044F8F448FF
:1087E00040213C3015F03FF8AC70EC70BDE87040B3
:1087F00001F018B830B50024234605E030F91350D5
:108800008D4200DD641C5B1C9342F7DBE548006889
:1088100090F86101A04201D2012030BD002030BD9E
:10882000F0B5064600200446059F0CE036F91450CA
:10883000D3F800C0AC4501DA1D603C7010B9954218
:1088400000DD0120641C8C42F0DBF0BD30B585B04A
:10885000D44C01A800902068002503ABB0F9522148
:10886000017DD448FFF7DCFF50B123689DF8040078
:1088700093F88A2102F00F01814219D81B7D14E080
:1088800002A80090206804ABB0F95421417DCA4889
:10889000FFF7C6FF68B123689DF8080093F88A21A6
:1088A00002F00F01814203D85B7D591A814200DA40
:1088B000150905B0284630BDFEB5BA4801AB5022B7
:1088C000006890F88911B0F9877101F00F060C0962
:1088D000B0F9855102A90091017DB648FFF7A0FFCC
:1088E0000198B84201DD3046FEBDA84201DA2046BB
:1088F000FEBD401B311B4843791B90FBF1F0204427
:10890000FEBD30B5AD48A74D0478286890F85101F8
:10891000800703D5FFF7D0FFA4EB0004286890F888
:108920005101400702D5FFF791FF0444002C01DA02
:10893000002402E00F2C00DD0F24204630BD30B5AE
:1089400064290DD00023642408E000BF30F91350DF
:108950004D4395FBF4F520F813505B1C9342F5DB77
:1089600030BD70B5002364250AE0CC5C642C06D0D1
:1089700030F91360664396FBF5F420F813405B1C56
:108980009342F2DB70BD2DE9F04700258946294668
:108990002F462E46A8462B460DE000BF30F913C0E7
:1089A00039F913400CFB0C660CFB047704FB0488BC
:1089B000654421445B1C9342F0DB87FB020485FB8A
:1089C000013CC71A86FB020385FB056564EB0C04BA
:1089D000B0EB060C63EB050688FB020381FB01216B
:1089E000851A63EB01086421A7FB010304FB013135
:1089F000002207FB02113346624614F0C3FE024612
:108A0000A2FB070301FB073102FB04112A46434680
:108A100014F0B8FE002C00DA4042BDE8F08730B513
:108A200047F6F873002405E030F91450AB4200DD3E
:108A30002B46641C9442F7DB002405E030F8145008
:108A4000ED1A21F81450641C9442F7DB30BD70B568
:108A500003460020024601EBD17408E003EB420616
:108A600033F91250B6F90260AD1B2844521CB2EB28
:108A7000640FF3DB621008E003EB420533F91240A8
:108A800035F9025C641B2044521C8A42F4DB70BD41
:108A9000F0B587B00746434C03A8009020689C4679
:108AA0008E461646017D002504AB0FFA8CF2704607
:108AB000FFF7B6FE01283BD102A80090206805AB65
:108AC00032B2417D3846FFF7ABFE012830D1DDE9F7
:108AD000041081424FF0640203DD504390FBF1F13A
:108AE00002E0514391FBF0F1206890F892218A4214
:108AF0001EDD9DF8081019B990F89121D20716D003
:108B0000427D521E8A4203D190F8911189070ED5F9
:108B10009DF80C1019B990F89121520707D5027DE4
:108B2000521E8A4204D190F89101000700D4012519
:108B300007B02846F0BD2DE9F04185B08046012000
:108B400001900290174C04A8009020681E468C46A5
:108B50001746017D002501AB32B26046FFF760FE8B
:108B6000064603A80090206802AB3AB2417D404619
:108B7000FFF756FE012E01D0012831D1DDE90110A9
:108B800081421DE062021000B0021000B10210002C
:108B90006302100064021000C8021000CA02100034
:108BA000AC0310003C02100054A7012090A7012044
:108BB000742D0120EC310120B0310120CB021000D6
:108BC0004FF0640203DD504390FBF1F002E05143AB
:108BD00091FBF0F0216891F89211814200DD0125AE
:108BE00005B02846BDE8F081F0B40446FF480B46C6
:108BF000802100680D4690F8680110B10146C0F56B
:108C00008075FB480089032805D22146F0BC52003C
:108C10001846FBF7CBBC00200FE000BF33F9106013
:108C200034F910704E4307FB0566F71706EB17661D
:108C300046F30F2623F81060401C9042EEDBF0BC98
:108C40007047F0B50024E94D0FE030F8146031F8BA
:108C50001470012B0CD0F61B2F6897F86D717F42B2
:108C600006EBC70620F81460641C9442EDDBF0BDEF
:108C70003E442F6897F86D71F2E72DE9FC47DC4D13
:108C800080460026288990B93C22DA49DA48FBF769
:108C90008DFC4022D949DA48FBF788FC3C21D948B1
:108CA00014F0E1FDD74840213C3014F0DCFD288968
:108CB0000127CE4C032802D2D348077013E012D903
:108CC0002168B1F86B2182420DD94B7DCA4ACD494A
:108CD000C84801F0A6FF2068CA49C94A037D3C3153
:108CE000C64801F09EFF206890F85011427D0907A8
:108CF00010D590F88D11CDE9001290F88B31C34A50
:108D0000BC494046FBF7B1FD2068BE49427DB839F9
:108D1000BE4802E0BB494046B839FFF765FF20680E
:108D2000B44A90F85011437D0907B94901D5B748B5
:108D300000E0404601F075FF2068AE4AB449437D2B
:108D4000B048B83801F06DFF206890F85011C9069E
:108D500010D5427D90F89612AD48FFF7F0FD2168DE
:108D600091F85001C00605D54A7D01F51C71A8484F
:108D7000FFF7F7FD2268B2F85411B2F86901B2F8B2
:108D80007F4101440BB229898C4201D2184403B2BD
:108D900000200446DFF87CC2DFF87492527D1CE0AC
:108DA00039F91080984515DD761C022E13D96878A4
:108DB000401C40B26870002804DD97488CF80070B1
:108DC0006C70077047F6FF70814201D2491C2981FF
:108DD000BDE8FC870026401C00B28242E0DC6C70DB
:108DE0008CF80040EEE7034610B50020024603E091
:108DF00033F91240521C20448A42F9DB10BDF0B511
:108E00007A4D0F4600262968497DFFF7ECFF04469E
:108E10002868017D3846FFF7E6FF002C00DA64423F
:108E20002A6800237249D2F89C52AC4206D8002826
:108E300000DA4042A84201D80B620DE0086A401CEB
:108E4000086292F89B22824206DC7448012602687E
:108E500042F4003202600B623046F0BD63480068A5
:108E600090F89011890606D5614901220A7090F8A0
:108E700095211209CA6190F8F102C00701D002F0F1
:108E800001B970471CB55A490020098901B9012070
:108E90001021564CCDE9001020680F236049427D17
:108EA000604801F02EFE0220009020685C49437D5E
:108EB000B0F9AE215B48FBF7A1FC012800D00020EF
:108EC0001CBD2DE9F34F002085B0824605460746BC
:108ED0000290554C401E03902078DFF83CB14FF0D3
:108EE00000084FF0010901281CD0404E306890F86E
:108EF0002010C9061DD590F825104C4802889142D3
:108F000017D2A0F800804A48016841F022010160B0
:108F10004FF480610120F7F7B1FA8BF8009007B0A9
:108F2000BDE8F08F8BF8009000F07CFC84F80080A6
:108F3000F5E70320F7F793FB3E482D4C0078012816
:108F40007ED02089012813D9306801232D49427D24
:108F50002848FFF776FE30682A490123027D3C311C
:108F60002648FFF76EFE3068334990F8FD0208701E
:108F700000202081FFF7C5FCDFF89CB0019021495B
:108F80009BF8000000903068B046B839427D019BE4
:108F9000059801F093FD9BF8000000903068194996
:108FA000019B027D7C39069801F088FD234E3078C4
:108FB0000A287BD00F2802D200F101003070D8F8C7
:108FC0000000464690F85011090745D5427D90F8BB
:108FD0008D11CDE900120B4A90F88B31B83A054952
:108FE0001046FBF742FC3068027D2AE03C0210008C
:108FF000AC031000741301206C140120B013012085
:10900000A8140120F82C012040041000B4501000D6
:10901000B031012064021000C8021000500210009C
:10902000801A0120441A0120CA02100054021000C4
:109030004802100057021000E5031000C90210009A
:1090400025E090F88E11CDE90012FF4A90F88C319E
:10905000FE491046FBF709FC3068FD4AFD49437D97
:10906000F9483C3801F0DDFD3068F84AFA49037DE3
:10907000F54801F0D6FD306890F89101000625D53D
:10908000F549F448FFF7BBFE01281DD01EE030680B
:1090900090F85101C00605D5FFF7F4FEEF4901280D
:1090A000087004D00598FFF7E8FD04E007E084F8B5
:1090B00001808BF800900320F7F7ECFA2FE70D20E2
:1090C00003F04BFF142079E7012002900320F7F70B
:1090D000E1FA3068DFF88883B34690F89011090709
:1090E0004CD5D949427D5E464031DA48FFF797FCBE
:1090F0003068D549427D403100F57470FFF743FC7C
:1091000060613068417DD0484030FFF7A0FCA0612D
:1091100063698646322B1CDDCB48DBF800204030EB
:10912000B0F90060B2F854118E4207DD92F815C014
:1091300000EB4C0C3CF902CC8C4509DC49428E42D8
:1091400007DA527D00EB420030F9020C884200DA67
:109150000125DBF8000090F8941199420EDAB0F87E
:10916000AC2172450ADA90F89001400600D501273B
:10917000D8F8001041F48051C8F80010DBF8000066
:109180005E4690F85011C9061AD5427D90F89612A5
:10919000B048FFF7D4FB3068027D90F8E012AE488B
:1091A000FFF7CDFB3068427D90F89712AD48FFF78E
:1091B000C6FB3068027D90F8E112AB48FFF7BFFBB9
:1091C000306890F89011890710D5B0F85231B0F896
:1091D0005421A1499F48FFF75BFC012806D1D8F82C
:1091E0000010012741F40051C8F80010306890F8D1
:1091F000911189060AD5B0F85231B0F85421964938
:109200009448FFF798FC012800D10127306890F8B6
:109210009111490617D5B0F95421417D8D4801F0CF
:109220001DFD02280DD870B13068417D894801F0DC
:1092300029FD02463068417D864801F00FFD022875
:1092400001D901273D46316891F89001820705D484
:10925000000703D491F8910180060BD5012F09D1A5
:10926000B4F9040000280ADB401E00B2A0800028E8
:1092700005DCBA4691F8950100F00F00A08091F846
:109280005001C0061AD54A7D01F51C717148FFF7DF
:1092900068FB316870480A7D01F52871FFF761FBB2
:1092A000316870484A7D01F52171FFF75AFB31683A
:1092B0006D480A7D01F53071FFF753FB306890F877
:1092C0005011090611D5CDF80090437D4F46674AED
:1092D0006749604801F07BFC00973068634A654944
:1092E000037D5D4801F073FC0CE0407D594942006C
:1092F0005F48FBF75BF930685749007D42005D48E5
:10930000FBF754F9306890F89111C90627D503A9E5
:109310000091427DB0F8AC31521E00214D48FBF760
:109320001CFB012815D10399012904DB3068427D1B
:10933000921E8A420EDAE0880125401E00B2E080CB
:1093400000280CDAD8F80010AA4641F48051C8F879
:109350000010306890F8950100F00F00E080306850
:1093600090F85111C9070CD0B0F95E21417D4048F9
:1093700001F065FC3068B0F95E21017D3D4801F0E7
:109380005EFC306890F85011490713D5CDF8009075
:10939000364A437D4F460A3A3749354801F017FCB3
:1093A00000973068314A3549037D0A3A314801F067
:1093B0000EFC0CE0407D2E4942002F48FBF7F6F8EA
:1093C00030682C49007D42002C48FBF7EFF83068EC
:1093D00090F8911189060FD5B0F85231B0F85421A8
:1093E00026492548FFF7A7FB012805D1D8F800102A
:1093F00041F48041C8F80010306890F89111490696
:109400001BD5B0F95421417D1B4801F027FC0228EF
:109410000DD890B13068417D174801F033FC024609
:109420003068417D144801F019FC022805D9D8F8AC
:10943000001041F40041C8F80010114F0B23387898
:1094400000903068427D1DE07C2C0120B01301208B
:1094500074130120B4501000F0501000630210008B
:109460005002100054A7012090A70120DA03100039
:10947000305110006C511000B0310120EC3101204E
:10948000C8021000D349D44801F018FB3878009086
:109490003068D0490B23027D3C31D04801F00EFBEF
:1094A00032682378B2F85211B2F85401012B04D07B
:1094B000CB4B1B78012B09D010E0B2F8983103B1E7
:1094C0001946B2F89A314BB1184607E092F8573175
:1094D000C91A92F8563189B2C01A80B2C14B1B78B2
:1094E0003BB192F8A331184492F8A43180B21944E8
:1094F00089B20FB20FFA80FC0097A781A4F80AC0C6
:10950000B346527D6146B848FFF774F90646DBF86A
:1095100000003946027DB548FFF76CF90746B448AC
:1095200061460670B3480770DBF80000427DA94829
:10953000FFF760F901281AD0A07820B1401EA07072
:10954000AB4800260670DBF800000099027DA148B8
:109550003C30FFF74FF901281BD0E07820B1401EC6
:10956000E070A44800270770012E25D026E0DBF824
:10957000000000253C2290F8951101F00F01A18018
:1095800090F86E01A07093499748FBF70FF80126F9
:10959000D9E7DBF800000025402290F8951101F092
:1095A0000F01A18090F86F018A49E0703C318F482B
:1095B000FAF7FCFF0127D7E7012F0BD08E490020D7
:1095C00008708E490870206900281DDD401E20614A
:1095D0000DD019E0884880F8009081480078012873
:1095E00012D1DBF8000090F8970120610CE0DBF865
:1095F000000090F89001C00606D5D8F8001041F49C
:109600000061C8F8001002E0029801280CD17C48E3
:10961000016841F0220101604FF480610120F6F7FA
:109620002DFF784981F80090BAF1010F0CD17448F0
:10963000016841F0420101604FF480610120F6F7BA
:109640001DFF704981F80090DBF800005E4690F83D
:109650009011890624D52178012921D1E1690029B9
:1096600015DD427DB0F954115F48FFF7C3F8074696
:109670003068027DB0F952115C48FFF7BBF807B1C2
:1096800000B94DB1306890F895010009E0615A4881
:109690000078012807D017E0E069401EE061F6D1AC
:1096A00000202070F3E73068B4F9041090F89501B9
:1096B00000F00F00884207D1002D7FF439AC4B49F0
:1096C000494800F035FD2AE400F00FFB27E42DE9BE
:1096D000FC4188460746FFF714F94A4E05464A4CB6
:1096E0003078009020682B464849427D384601F08A
:1096F000E5F930780090206844492B46027D3C31E2
:10970000404601F0DBF9206890F85011090719D59F
:10971000427D90F88D11CDE900123C4A90F88B31D2
:109720003B491046FBF7A1F82068027D90F88E11A6
:10973000CDE90012354A90F88C313C32354910465B
:10974000FBF793F82068324A3349437D2F4801F0F4
:1097500068FA20682F4A3149037D2C483C3001F0DB
:1097600060FA206890F85111C9070CD0B0F95E2159
:10977000417D294801F063FA2068B0F95E21017D3E
:10978000264801F05CFA206890F85011490711D57D
:1097900001250095437D224A13491F4801F017FA1D
:1097A000009520681E4A1149037D1C4801F00FFAFC
:1097B000BDE8FC81407D184942000B48FAF7F6FEEF
:1097C00020681649007D02B04200BDE8F04107481C
:1097D000FAF7ECBE742D012054A7012090A70120B8
:1097E000AC0210006E021000B0310120EC310120FB
:1097F000B0021000B10210006202100064021000FA
:1098000048021000C80210003C021000402C012049
:1098100074130120B0130120305110006C5110005E
:10982000D0031000F9490020FA4A0870F849C860CE
:1098300008618880C88008701070F74A48701070FE
:10984000887008814881704730B5F44A0024126856
:10985000937EDD0792F882310BD0834217DC158BA3
:10986000EB1A834213DB92F8830188420FDCD28A21
:109870000AE083420BDCD58AEB1A834207DB92F8BD
:109880008301884203DC128B101A884200DA01241B
:10989000204630BD2DE9FE4314460D460646072BF3
:1098A00009D0DB48092BB0F9041006D03180C188FB
:1098B000298000781070BDE8FE833288ADF8022060
:1098C0002A88ADF800202778ADF806108146C088B8
:1098D000ADF8040001AA694602A810F024FC02A811
:1098E00010F019FCDFF834830346D8F800C09CF868
:1098F0007401BCF8762100F00F01BCF878C10009B2
:1099000052430CFB0CFC93420BDD634501DB084624
:1099100007E09B1A411A4B43ACEB020193FBF1F1B8
:10992000401ABDF90230C0F11001B9F904C04B432F
:1099300000FB0C3343F30F133380BDF900304B436E
:10994000B9F9061000FB013040F30F102880D8F859
:109950000000102199F8002090F87501A1EB10117A
:109960007943000900FB0210C0F307102070A2E742
:109970005FF0000200EB82035B6840F82230521C6B
:10998000052AF7DB416170472DE9F04F002793B0BE
:1099900080463E463D46FFF7EBFF002158F8210088
:1099A0000744484300FB0155491C06440629F5DBE2
:1099B000974C0997143460680A90A068CDE90B06AB
:1099C00020690D906069CDE90E05E0691090206A6C
:1099D000119009A8F9F794FF834603912068CDE917
:1099E0000907A0680B90E068CDE90C0660690E904D
:1099F000A069CDE90F05206A119009A8F9F780FF49
:109A00008146206809906068CDE90A07E0680C90FB
:109A10002069CDE90D06A0690F90E069CDE9100538
:109A20008A4609A8F9F76CFF0326A9FB06570A46E0
:109A30000AFB06710926A0FB0637002409FB041463
:109A400002FB0672002100FB0120EA184441039941
:109A500012EB0B0061414FF47562002313F092FE8C
:109A6000C8F80C0013B0BDE8F08F30B56B4A012484
:109A70001268937EDD0792F87A310BD0834217DCAF
:109A8000158BEB1A834213DB92F87B0188420FDCC3
:109A9000D28A0AE083420BDCD58AEB1A834207DBC9
:109AA00092F87B01884203DC128B101A884200DA9C
:109AB0000024204630BD2DE9F047DFF860910546CF
:109AC000534CD9F800008AB00E4690F870019A46BF
:109AD00017464FF00008C00728D0082D26D094F96B
:109AE0000200062819DB11463046FFF7BEFF0028AA
:109AF0004B48314609D0FFF747FF06B24848394680
:109B00001830FFF741FF07B210E0FFF731FF44487C
:109B100039461830FFF72CFF08E0401C404940B29E
:109B2000A07041F82060183141F82070ADF8006055
:109B3000ADF804708DF814A02B4605AA01A968465B
:109B4000FFF7A8FE072D2DD0092D2BD1D9F8001035
:109B500091F87001400725D5B4F90420BDF9000043
:109B6000101A00D5404291F87C3198420EDAB4F9CF
:109B70000630BDF90400181A00D5404291F87D6105
:109B8000B04203DAADF80020ADF8043022789DF839
:109B90001400101A00D5404291F87E11884201DA73
:109BA0008DF81420D9F800004E464FF0000790F8C9
:109BB000700100060FD5082D0DD0BDF90410BDF9B8
:109BC0000000FFF741FE8046012804D1306890F87C
:109BD0007111C9070DD0BDF90010A180BDF9042095
:109BE000E2809DF814C084F800C0B8F1010F2FD0B6
:109BF00066E0072D18D00B49097831B390F8A6011B
:109C0000401CE06000200AB0BDE8F087AC02100004
:109C1000E403100062021000640210003C02100015
:109C2000845010006E021000FE490F7090F89001F1
:109C3000C007E7D0FC48016841F0220101604FF401
:109C400080610120F6F71AFCDCE790F87301D7E792
:109C5000306890F87131DB0732D0837EDB0790F8F3
:109C6000823113D08B4201DDADF80030018BC91A6F
:109C7000BDF90030994201DAADF8001090F8831177
:109C8000914201DDADF80410C08A12E08B4201DD83
:109C9000ADF80030C18AC91ABDF90030994201DA25
:109CA000ADF8001090F88311914201DDADF8041079
:109CB000008B401ABDF90410884201DAADF80400A7
:109CC0000397BDF800000297ADF80E008DF808501C
:109CD000BDF80400ADF80C008DF80AC08DF80B70CB
:109CE00002A802F08DFF01208DE7D04810B5017861
:109CF000CF48006849B190F9A611CA480278CD480A
:109D0000012A05D0002101610DE090F97311F4E7FB
:109D1000C268521CC2608A4208D300231A46194600
:109D20000820FFF7C8FEBDE810407BE510BDF0B588
:109D30000746DDF814E037F912404FF0FF30744564
:109D400001DA002400E01046012517E0561B07D475
:109D500037F916C0F44503DDA44501DD30466446FD
:109D60005619A1F1010C664507DC37F916C0F44518
:109D700003DDA44501DD304664466D1C9D42E5DDF2
:109D8000F0BDAB490A68B2F8641181420DDAB2F84D
:109D90006621824201DCFF207047401A521AC0EB54
:109DA000002090FBF2F00028F6DC01207047F0B5AF
:109DB00000240125A1F101060BE0571B02D430F964
:109DC00017703C445719B74202DC30F917703C4415
:109DD0006D1C9D42F1DD012A02DB891E8A4200DDF5
:109DE000640030F912002044F0BD2DE9F047904D99
:109DF00014469A462E6830F91420814602FB04F07E
:109E00000123A1F1010196F862C117E0E51A08D417
:109E100039F91570B6F85E81474502DB07FB05008E
:109E20003A44E5188D4208DC39F91570B6F85E81C0
:109E3000474502DB07FB05003A445B1CB3EB1C1FE4
:109E4000E4DD4A4380FB0A01D31713F09BFC00B208
:109E5000DAE62DE9F05F8B46D0E900159146002245
:109E600080689A4613464FF48034814202DD0246F0
:109E70000B4602E001DA0A460346A0EB01014FF46B
:109E8000803CA1FB0C084FEAE17707FB0C874FF001
:109E900000062B44C2F1000201FB067103EB4202F3
:109EA0004FEAE27313F06EFC4FF48036A9FB063CD8
:109EB0004FEAE97505FB06C51B18A3FB0A06002738
:109EC00009FB07524A4102FB0A614FEAEA7503FBAC
:109ED000051122463B4613F055FC5A464FEAEB73F8
:109EE00013F050FC00B2BDE8F09F2DE9F04F93B0A5
:109EF0000C46824617469946002518210CA81C9E40
:109F000013F0D3FC00200290039004902EB948482F
:109F1000006890F8620100F00F06BA1B07EB060319
:109F200000D50022661EB34200DD631E0CA9504618
:109F3000F9F743FE4FB1B7422FD13D48006890F882
:109F40005101800613D54D466BE03948006890F802
:109F50005101800665D4BAF904000290BAF90000F4
:109F60000390BAF902004B46012204900DE00AEB7F
:109F700044007F1C30F9061D0291B0F904100391D2
:109F8000B0F902004B463AB20490611E02A8FFF7F6
:109F900060FF99FBF6F1451A43E0DDE910B1B1F13C
:109FA00000084BDADDE90C2352EA030046D0DDE974
:109FB0000E0105910890002940DB1D48056895F8C1
:109FC0005001400611D55846414613F0DBFB0028EE
:109FD00000DA404295F86311884206DA4B463A4669
:109FE00021465046FFF701FF1AE01BEB0B01A1FBD6
:109FF000062448EB080000FB0640F31701FB0303AF
:10A00000089805994542A5FB0907002464EB010463
:10A0100004FB09714FEAE97605FB061113F0B2FB68
:10A02000054609E0AC021000480210006E02100064
:10A030003C021000E403100028B213E5B8F1000F51
:10A04000CCDADDE90C010843C8D00F980028C5DB45
:10A05000E7E738B5AA4D049C2D6895F85051AD0638
:10A0600003D50094FFF741FF01E0FFF7BEFE00B209
:10A0700038BD2DE9F04700249A46CE1E814623467E
:10A08000A44627462546022A03DBB24201DC1046DD
:10A09000BAE50020491E07E039F91080B8F1000F39
:10A0A00001DDC4447F1C401C8842F5DB9CFBF7F7B4
:10A0B000022A12DA10460DE039F91060BE4203DAC6
:10A0C0003CB90446002304E01CB19E4201DD334646
:10A0D0000546401C8842EFDB14E0B24212DD104618
:10A0E0000EE000BF39F91010B94203DA3CB904465A
:10A0F000002304E01CB1994201DD0B460546401ED9
:10A100000228EFDC534500DA154628467CE530B5D9
:10A11000044630F911300020491C06E034F9115092
:10A120009D4201DD2B460846491C9142F6DB30BDBD
:10A130002DE9F34F724C85B0226892F88451567D18
:10A1400005F00F035F4206EB470606F0FF0B167D96
:10A150002A09554200EB430006EB45050590EDB298
:10A1600001EB420001952A4600210690FFF7CFFF40
:10A1700005465A4600210598FFF7C9FF06462068A4
:10A18000604F90F87001800607D5B7F900302A4675
:10A1900001990698FFF76DFF05462068DFF868A172
:10A1A00090F87001C00607D5BAF90030324659461A
:10A1B0000598FFF75EFF0646DFF85091DFF8508103
:10A1C00099F80000012828D1206890F86001010763
:10A1D00023D0010921D0B7F90010009100F00F033E
:10A1E000B8F9082001990698FFF7A1FD0746BAF9CA
:10A1F000000000902068B8F90A20594690F86001E4
:10A2000003090598FFF793FD002F01DB002802DA10
:10A21000FFF76BFD01E03D4606462FB232B2A8F8CB
:10A220000870A8F80A200026009620685946B0F960
:10A2300018300598FFF70DFF0096039020683A4606
:10A240000199B0F916300698FFF703FF02902068D5
:10A2500090F87001800704D5032203A902A806F034
:10A260007DFD03A902A8FAF77DFA01232A46019988
:10A270000698FFF79CFDFFF784FDC3B225480078E0
:10A280000028206810D090F9A51198F801204046C8
:10A29000521E52B288F80120002A08DB226892F888
:10A2A000FC22114449B204E090F97211EDE7FF225B
:10A2B000427099F8004005690CB96D1C05618D422A
:10A2C00019D340F2FF110161C8F80C6044B1039842
:10A2D00002B2029801B20920FFF7EDFB48B10AE093
:10A2E000012089F80000039802B2029801B2072009
:10A2F000F2E7FFF7FAFC07B00120BDE8F08F00009D
:10A300003C021000B8031000B6031000AC021000AD
:10A31000E40310006E021000E448E54A0068B0F85B
:10A32000AC139180E34990F8B00308817047E1498C
:10A330000020DE4A8880C880C86048801268DE4BF2
:10A3400092F85C2112091A7008610870DB490870E4
:10A3500070472DE9F043A1B0814602AF782138461D
:10A3600013F0A3FAD1480123016891F8B1204C7D84
:10A3700091F8A01103EB1216890715D50025804628
:10A3800010E000BFD8F8001005FB04F009EB400016
:10A390004A7D91F88B31CDE9003249460246FAF701
:10A3A00064FA6D1CB542EDDB002010E000FB04F206
:10A3B000002109E002EB010C57F8215039F91C305B
:10A3C0002B4447F82130491CA142F3DB401CB0422A
:10A3D000ECDB002007E000BF57F8201091FBF6F1FE
:10A3E00047F82010401CA042F6DB00200121A4F118
:10A3F000010517E04FF0000C63460BE003FB041867
:10A4000039F9182057F82180B2EB080200D55242E2
:10A4100094445B1CB342F1DB9CFBF6F2824200DD0C
:10A420001046491CA942E5DBB0F5803F04DB4FF63E
:10A43000FF7021B0BDE8F08380B2FAE730B59B49E8
:10A440009D4B096891F85021920725D59B4A1278B7
:10A450004AB191F8A74104F00F022509B1F8A841CB
:10A46000B1F8AA1107E001F5AC710C7904F00F0204
:10A4700025090C884988A04201DC1A7030BD884249
:10A4800001DB1D7030BD001BAD1A6843091B90FB3A
:10A49000F1F01044187030BD91F85C0100F00F002D
:10A4A000F8E72DE9F041814D814A2E6896F8801336
:10A4B000B6F8AC33C9073DD096F8AF4304B90124D0
:10A4C000918896F8AEC3CF1A07FB0CF797FBF4F40C
:10A4D000B6F8AA730F442744764CB8420ADD00262A
:10A4E00020210120E660F5F7C9FFE680286890F892
:10A4F000B00306E0814202D9704D2D7825B196F85F
:10A50000B0032081BDE8F0816D4D2D78002DF9D18B
:10A51000B4F90850002D01DD6D1E25812489002C21
:10A52000F0D1891E814200DA01468B4200DD1946D6
:10A530009180E7E79380E5E75C4A10B51468002155
:10A54000B4F8A121824204D294F8B000800700D56B
:10A5500001215848594B0278914211D11978914202
:10A560000AD0574C2478224307D00169491E016163
:10A57000002901DC0078187010BD01700169F7E74F
:10A5800039B194F8B22002610170002AF4DC19702C
:10A5900010BD94F8B320F6E7444910B5096891F866
:10A5A000B010CA06434918D5464A14780A46D388DB
:10A5B000C3EB03125200012C05D0C41A002C0CDC92
:10A5C0003F4C247824B102EB4000C0F34F1004E06C
:10A5D000C3EB83121044C0F38F10C88080B210BD4B
:10A5E00010B5FFF7B6FEFFF7D7FF324CA080FFF79C
:10A5F000A3FFA088FFF722FFA088BDE8104050E726
:10A60000F0B430490B782B494A88B3B1322A01D2D1
:10A61000521C4A80254A0125136893F8B1405B7D9E
:10A6200005EB1415CC6894FBF5F605FB1644264E95
:10A63000634306EB430700230BE0012AEAD9521ECD
:10A640004A800022CA60E5E730F813C027F813C03B
:10A650005B1CD2F800C09CF815C09C45F4DCCB68AC
:10A660005B1CCB60136893F89477FF0707D05B7D82
:10A67000641C5F00634306EB4304002307E0C868E3
:10A680000CE0FE1830F8166024F813605B1C1668A6
:10A69000767D9E42F5DCC868401CC860A84202DB9B
:10A6A000F0BC09489CE7F0BC704700003C02100079
:10A6B000D82610001C041000CB0210006E021000FF
:10A6C0006202100057021000F02D0120E049002026
:10A6D000C86088604860DF490870704710B5002383
:10A6E0000BE000BF30F91340002C00DA64428C42CA
:10A6F00001DD012010BD5B1C1BB29342F2DB002088
:10A7000010BD70B5D44CD54AD5492068437DD54895
:10A7100000F087FA2068D44AD449037DD44800F079
:10A7200080FA2068427DB0F99812CD48FFF7D6FF35
:10A7300005462068027DB0F99812CC48FFF7CEFF9D
:10A740000022C349012803D0012D01D04A6070BD09
:10A750004868401C4860236893F89A328342F6DCCC
:10A76000C448036843F480330360C3484A60016807
:10A7700041F022010160BDE870404FF4806101208A
:10A78000F5F77CBE70B50546002003460CE000BF1F
:10A7900035F9134031F91360A41B00D5644224B28B
:10A7A000A04200DA20465B1C9342F1DB70BD2DE92C
:10A7B000FF4FA94E8146B9F1010F306808D0AF4D67
:10A7C000AF4B047D0020DFF888B24FF0010A64E04F
:10A7D000AC4DAD4B447DF5E735F8101033F91070F2
:10A7E000DFF8A8C2C91B0AB29CF800C00021BCF166
:10A7F000010F05D0002A08DADBF80C2012B116E0B0
:10A80000114614E0029949420DE0DBF808C0BCF1A2
:10A81000000F0CD10199DDF80CC009B2624506DDCC
:10A820000D998A4201DD09B201E00FFA8CF107EBC4
:10A83000010223F81020376897F8802352072BD5A0
:10A84000B9F1010F4FF0000202D0DFF824E21DE061
:10A85000DFF810E20AE000BFC2EB02180EEB880C32
:10A86000521C3CF8108088442CF8108097F88083A4
:10A870000AEB981C9445EFDC0EE000BF0EEB821C47
:10A88000521C3CF8108088442CF8108097F8808384
:10A890000AEB981C9445F1DC401CA0429CDBBDE80F
:10A8A000FF8F2DE9F84F6C4D694C00262A684FF058
:10A8B000010A92F82300527D00F00F0774480178D6
:10A8C00001293FD0804600913B466E49714800F017
:10A8D000F5F898F800000090286868493B46027D2A
:10A8E0006D4800BF00F0EAF86C48007840077DD55D
:10A8F0006B480078B8B3A660E660286890F82C1022
:10A90000B0F82F90B0F833700C0901F00F08427DB9
:10A910005D496448FFF736FF844628685849027D40
:10A920006148FFF72FFF29684A4AB1F85431BCEB60
:10A93000530F04DCB1F85211B0EB510F45DD82F832
:10A9400000A043E02680D0463B464E494E48CDF815
:10A9500000A000F0B3F8CDF8008028683B464749D6
:10A96000027D4748BEE7FFE7A168491CA16028684F
:10A9700090F82A20B1EB121F00DDA660E16802F01A
:10A980000F02491CE1608A4200DAE66090F8242058
:10A9900011090FD090F8383021888B420AD9491C10
:10A9A000218090F82B1012090C09544301F00F017B
:10A9B000514304E090F82B100C0901F00F01884678
:10A9C000B0F82D90B0F83170A1E716704B464246B2
:10A9D000214601200097FFF7EAFE4B4642462146FA
:10A9E00000200097FFF7E3FE286800E00AE090F8F7
:10A9F0009111090606D590F88003400702D5BDE8FD
:10AA0000F84F7EE6BDE8F88F134810B5006890F85F
:10AA10002000C1071AD025490978002916D12449F8
:10AA2000097809B1800611D52248007800280DD197
:10AA300021480078002809D10320F5F710FEFFF720
:10AA400030FFBDE810400320F5F724BE10BD000024
:10AA500030041000D70210003C021000D81501206D
:10AA6000B4501000E814012014170120F050100019
:10AA70001416012050021000480210002C1401206E
:10AA8000B0130120F01301207413012040041000C2
:10AA9000C8021000C82A0120042B01204404100021
:10AAA00057021000402C01207C2C01205D02100078
:10AAB000620210006702100065021000F0B40C463C
:10AAC00001460498C3F11006012801D0002014E0CB
:10AAD0002046F0BC5200F9F769BD00BF34F91050B0
:10AAE00031F910705D4307FB0655EF1705EB17753D
:10AAF00045F30F1524F81050401C9042EEDBF0BCDB
:10AB00007047F0B40C460146DDE90460F51A0128EF
:10AB100001D0002010E02046F0BC5200F9F746BDFD
:10AB200034F9107031F910C05F430CFB057797FBC7
:10AB3000F6F724F81070401C9042F1DBDFE72DE9B6
:10AB4000F0470026DDE908A9B446354637463446C5
:10AB50000FE000BF31F91480B8F1000F03DD464467
:10AB600005F1010503E002DAC44407F1010704F12D
:10AB700001049442EEDB96FBF5F69CFBF7F700240C
:10AB800021E06BB131F91450002D0FDD30F8145075
:10AB900035442DB220F814504D4513DD35440FE0F7
:10ABA00030F8145031F814C0654409E00ADA30F87E
:10ABB00014503D442DB220F81450554502DA3D445E
:10ABC00020F81450641C9442DBDBBDE8F0872DE9CB
:10ABD000F04391460022DDF81CC019E000252E4606
:10ABE0004FEA050402EB0407BF1E08D49F4206DAB1
:10ABF00030F9178039F9147008FB07553E44641C7E
:10AC0000052CEFDBBCF1010F06D021F81250521CCD
:10AC10009A42E3DBBDE8F08395FBF6F421F812409D
:10AC2000F5E770B5002407E032F8145030F81460EE
:10AC3000AD1B21F81450641C9C42F5DB70BD30B58F
:10AC400000231C4607E000BF30F91350954201DA9B
:10AC500020F813405B1C8B42F6DB30BD70B5054617
:10AC60000020044603460AE035F91360964204DDED
:10AC70000CB9401CC0B2641C00E000245B1C8B4279
:10AC8000F2DB70BD10B50022134603E030F913402B
:10AC90005B1C22448B42F9DB09B192FBF1F210B24A
:10ACA00010BD10B5044647F6FF70002206E000BF55
:10ACB00034F91230834200DA1846521C8A42F7DB1C
:10ACC00010BD10B504461C48002205E034F91230CE
:10ACD000834200DD1846521C8A42F7DB10BD2DE985
:10ACE000F04300252E462C46DDF81C9018E000BFEE
:10ACF00031F9147030F914C007EB0208C44505DDC2
:10AD0000BCEB070700D57F423E4408E0A7EB0208F2
:10AD1000C44504DABCEB070700D57F423D44641C00
:10AD20009C42E5DBB9F1000F00D10025B54201D20C
:10AD300001206FE700206DE70080FFFF10B5BB48E2
:10AD4000BB4A00685168414010D05060480701D5A7
:10AD5000FDF718FDB748006890F81001C00605D54A
:10AD60004021BDE810400520F5F788BB10BD10B5A7
:10AD70000446480709D5B0492046F8F776FF204633
:10AD8000BDE81040AD49F8F796BF10BD70B5A94CAD
:10AD9000206890F81001C0065BD5A948A449007846
:10ADA0000979084000F004050620F5F758FC29460B
:10ADB000A448FFF7DCFF0620F5F76CFCA2480078FA
:10ADC000400746D0680744D50420F5F748FC9B4966
:10ADD0009948FEF77CFC0420F5F75CFC2068964956
:10ADE000407D42009948F9F7E1FB2068017D407DF4
:10ADF0004A00964901EB40009049F9F7D7FB2068DB
:10AE00009349407D42009348F9F7D0FB2068017DCB
:10AE1000407D4A008F4901EB40008F49F9F7C6FB9E
:10AE20002068017D407D08444100884811F003FC02
:10AE30008A4D68802068017D407D08444100854836
:10AE400011F0F9FB2880BDE8704010210520F5F7CE
:10AE500015BB70BD2DE9F0417548794E4FF00008E3
:10AE600080F800807E4935680D427CD040680540FE
:10AE70007C480078002876D10620F5F7F0FB2946BB
:10AE80007048FFF774FF6B4C774F206890F8A01163
:10AE9000C90709D0307800060CD43878022809D0C8
:10AEA0006848FFF7ADFB05E090F85C016F4900F0E2
:10AEB0000F0008700620F5F7EDFB680709D50420A0
:10AEC000F5F7CDFB5D495C48FDF7FBFF0420F5F786
:10AED000E1FB3878022802D13068002801DAFFF758
:10AEE00093FD5948007840073AD0680738D5206864
:10AEF0005149407D42005548F9F758FB2068017DD3
:10AF0000407D4A00514901EB40004C49F9F74EFBA6
:10AF100020684F49407D42004E48F9F747FB2068C2
:10AF2000017D407D4A004B4901EB40004A49F9F759
:10AF30003DFB2068017D407D08444100434811F0FD
:10AF40007AFB464D68802068017D407D08444100C1
:10AF5000404811F070FB288010210520F5F78EFA8B
:10AF6000434981F80080BDE8F081314910B50020E7
:10AF70004860FFF7ABFBFDF705FCFFF7D8F9BDE82C
:10AF80001040FFF7C9B92A4C08B500256570FFF7D6
:10AF9000ECFF4FF6FF76607868B30128FBD16B4673
:10AFA000002255210420F5F7B9FA0098C00706D011
:10AFB00031460420F5F791FAFFF7D7FF6570009846
:10AFC000400705D504210846F5F787FAFFF742FF49
:10AFD0000098400605D540210420F5F77EFAFFF7DA
:10AFE000D5FE0098C006D6D510210420F5F775FAD5
:10AFF000FFF7A4FECFE704210020F8F7DEFE6B4642
:10B00000002202210420F5F789FA04210120F8F733
:10B01000D4FE00988007BED531460420F5F75DFACE
:10B02000FFF7A3FF01206070B5E700003C061000A9
:10B03000400410003C021000C82A0120042B01200B
:10B04000A802100050AF012028061000EC271000C5
:10B05000B031012068281000EC310120D027100009
:10B06000140200805D021000CC021000CB02100020
:10B07000C8021000FD48002141728172C172C17185
:10B0800001727047F9480021016101717047F74969
:10B0900000B50120C870FFF7F5FF5DF804EBE9E7A4
:10B0A000F2480021C16081700121C170704700B574
:10B0B000FFF7E8FFED490120C87000BD2DE9FC470E
:10B0C00089460746F8F7CBFD0090F8F7F3FD0190AD
:10B0D00004216846F8F7EAFB0446042101A8F8F7C2
:10B0E000E5FB2044E14C4600E1492069E14D704315
:10B0F00001EB400029687200B1F8F3823946F9F794
:10B1000055FA2868216990F8F202884202D101209C
:10B11000207102E02079012819D1D54F002014E0D8
:10B120002A68012137F9103092F8F222521C05E00A
:10B1300006FB010C491C37F91CC063448A42F7DC4A
:10B14000A3EB080229F81020401CB042E8DB286875
:10B1500090F8F2122069814201D3401C00E00020E7
:10B1600020612079BDE8FC872DE9FC4115460E469B
:10B170000746F8F774FD0090F8F79CFD01900098E1
:10B180000421400800906846F8F790FB044604212B
:10B1900001A8F8F78BFB00EB440C07EB440207EB2C
:10B1A0004C03014606EB440706EB4C06002006E084
:10B1B00032F810C00CFB05FC27F810C0401CA04260
:10B1C000F6DB002006E000BF33F810206A4326F8C3
:10B1D0001020401C8842F7DBBDE8FC812DE9FC47CC
:10B1E000154689460646F8F73AFD0090F8F762FDE5
:10B1F000019004216846F8F759FB0446042101A890
:10B20000F8F754FB0146304606EB440305EB4407D0
:10B21000002207E030F802CB33F8028B521CC44402
:10B2200027F802CBA242F5DB01EB440206EB8400D7
:10B2300006EB420305EB4206002207E030F8027BF2
:10B2400033F802CB521C674426F8027B8A42F5DBB6
:10B2500048462946002204E030F8023B21F8023B30
:10B26000521CA242F8DB09EB440005EB84020021EA
:10B2700005E000BF30F8023B22F8023B491CA14226
:10B28000F8DB6FE72DE9F05F7A4E00247A4F3568DE
:10B2900023464FF0010A95F81051A3465FEAC56CAA
:10B2A000724D1DD500230DE031F9138030F913C024
:10B2B000A8EB0C08904500DD641CB84501DA21F8C4
:10B2C00013C05B1CD6F800C09CF815C09C45EBDC95
:10B2D00014B185F805A001E085F805B000242346E7
:10B2E000D6F800C0B1469CF815C0ACF1020C0FE0D6
:10B2F00031F91C6030F91C80A6EB0806964200DD8F
:10B30000641CBE4202DA21F81C805B1C0CF1010CAB
:10B31000D9F80060767D6645EADC002631F916C072
:10B3200030F91680ACEB080C944500DD641CBC457C
:10B3300002DA21F816805B1C761C022EEEDB23B1AC
:10B340004E484F494088F9F7A8FD14B185F806A08A
:10B3500001E085F806B0D9F8000090F81001C006A9
:10B3600002D56879BDE8F09FA879FBE72DE9FC419B
:10B37000404D3E4C01272B6860780026B3F8AE8123
:10B380005A7D18B1207801280BD021E0E178802087
:10B39000CDE900017F233B493B48FFF7B2FBE67054
:10B3A00016E0921E3748384905E000BF31F812C058
:10B3B00020F812C0521C93F815C09445F6DC002208
:10B3C00031F8123020F81230521C022AF8DB2670B5
:10B3D0002E48007806280CD00220009028680FFA2A
:10B3E00088F22849437D2848F9F708FA6070384602
:10B3F000F2E628682349437DB0F94D212248FFF742
:10B4000041FF0027012802D0E6606670EFE7A079CF
:10B41000012809D060790128E9D160780028E6D1B7
:10B420001B4800780128E2D1E068401CE0602968F0
:10B4300091F81A11814202D20120A070607000F0D0
:10B4400041FC01210220F5F719F8D0E7F0B40B46D2
:10B450000849096891F89417C9072AD00D49096865
:10B46000490026D400EB420400211EE048041000ED
:10B47000A45210003C0210000CFEFFFFD826100062
:10B48000A8000120801A0120441A0120CC021000DB
:10B490005F0410007404100030F8025B34F8026B93
:10B4A000491C354423F8025B09B29142F4DBF0BC3D
:10B4B0007047F0BC014652001846F9F777B870B5EE
:10B4C000FA4E0025307810F0940F3FD0F84CF9492F
:10B4D0002068427DF848FFF7B9FFFFF747FF0546B0
:10B4E000012833D1206890F89407C107F34808D0A9
:10B4F0003168490005D44169C068F14AFFF76EFE22
:10B5000003E0C068EE49F9F75AF83078000607D52D
:10B510002068EB4990F893270846521CFFF724FE59
:10B520002068E84990F8F102C007E54802D0FFF72B
:10B53000C5FD01E0F9F743F8206890F8F102C00773
:10B5400004D0E1480079012800D00025284670BDCC
:10B5500070B5D74D0024286890F8E801C0B1D348F1
:10B560000078800714D5D548D8490069F8F7FEFB64
:10B57000D7480124007802280AD1D34E707838B910
:10B580002A68D44902F5F872D048F9F71CF97070AE
:10B59000204670BDF8B50746C448C54D0126007861
:10B5A0002968400702D5B1F8E72201E0B1F8E922A5
:10B5B000C748DFF824C3C44C03780220062B10D000
:10B5C0000090087D4A7D00FB02F3B1F9E9220CEB03
:10B5D000400107EB4000F9F711F9607001282BD00A
:10B5E0002FE091F8103100261B072AD50090087D26
:10B5F000497D12B200FB01F30CEB400107EB400068
:10B60000F9F7FCF8012803D00020E060607018E032
:10B610006078B0B9E068401CE060296891F81A11C0
:10B6200081420ED20120A070607000F04BFB01211E
:10B630000220F4F723FF04E0A848016841F001016B
:10B6400001603046F8BD2DE9F041994D0E460346A4
:10B6500029681446DFF870C24F7D087D07F10107A5
:10B66000024607FB04F700FB07F09D4F274417F83D
:10B67000017C8CF8077091F86110090700D510441F
:10B68000420019463046F8F791FF2868017D407D59
:10B69000401C641E6043414306EB4100BDE8F0815D
:10B6A0002DE9F84FDFF808A280460646DAF80000D8
:10B6B000DFF814920F46447D007D641C444399F8E2
:10B6C0000A10484689F80B1000254FF0010B4AE09C
:10B6D000827A844B02FB04F103EB410605FB04F183
:10B6E00008EB410100910BFA02F1C279114389F88C
:10B6F000071031460098F8F77EFFDAF8000090F85E
:10B70000611009071CD5791E8D4208D1007D4200C9
:10B71000009800EB440106EB4400F8F747FF99F866
:10B720000A0068B9DAF80000017D90F8F3064A00D3
:10B7300000096C49604301EB40003146F8F736FFE1
:10B7400099F80A104846491CC9B289F80A10DAF873
:10B75000002092F8F326B1EB121F03D3002181726F
:10B7600089F809B06D1CBD42B2D33046BDE8F88FF0
:10B770002DE9F047DFF8388106469146D8F80000F9
:10B780000D460224007D314642002846F8F70EFFA0
:10B79000B9F1010F00D1012401270CE0007D00FB6D
:10B7A00007F14200604306EB410105EB4000F8F76A
:10B7B000FDFEA41C7F1CD8F80000417D491CA1425D
:10B7C000ECD8D8F8001091F86110090721D50123B1
:10B7D000B9F1000F10D0427D017D521C03EB5203E2
:10B7E0004B434A4305EB420006EB43034A00BDE8E6
:10B7F000F0471946F8F7DABE417D027D03EB5103AD
:10B80000491C5343514306EB430305EB41005200EF
:10B81000EDE7BDE8F08770B5254E05460C4630686B
:10B820002946007D42002046F8F7C0FE3068007DC2
:10B83000420005EB400104EB4000F8F7B7FE30682A
:10B84000007D420005EB800104EB8000F8F7AEFEBE
:10B850003068417D007D491E4143420004EB4103B5
:10B8600000EB400005EB40011846F8F79FFE3068FA
:10B87000417D007D414304EB410305EBC001BDE880
:10B88000704042001846F8F791BE70B50346104864
:10B890000C460078072801D0062827D112480078E6
:10B8A000012823D01846FFF7B6FF41E074041000CA
:10B8B0003C021000441A012048B001207C571000BF
:10B8C000AC51100050AF012048041000BC2A0120E8
:10B8D000CC02100068130120A8000120F80210001B
:10B8E00024DC010040B201205F041000D848006849
:10B8F000820001D5002202E0C20004D501221846D0
:10B90000FFF736FF14E0D34AC504127F04D5114671
:10B910001846FFF7C5FE05E0800405D5CE49184658
:10B92000FFF791FE044603E001221846FFF78BFE65
:10B93000204670BD2DE9FC47C84F00263878042802
:10B9400001D0FFF797FBDFF80883C24DC44C98F88D
:10B950000000C0071BD0C3496868FFF796FFFFF7D8
:10B9600019FE0646D8F80000C10510D5216891F8E7
:10B970009417C90707D0400005D4D5E90510BA4A85
:10B98000FFF72CFC03E0B849A869F8F718FEB8F8EF
:10B99000000040040CD52068017D90F8D10000F033
:10B9A0000F00401C41434A00B048A968F8F7FEFD6B
:10B9B0003878022871D12068D8F80010B0F8AE713C
:10B9C000CA056AD590F89407C00707D0480005D487
:10B9D000D5E90510A44AFFF701FC03E0A249A869D4
:10B9E000F8F7EDFDA249A048F8F73FF9A1499E48B4
:10B9F000F8F761F9216891F85002C0074DD091F82D
:10BA00001001000649D591F850219948DFF8648269
:10BA100012071BD54A7DB1F93402CDE90002B1F914
:10BA20003232954A95499248F8F71FFF2068027D07
:10BA3000B0F93812CDE90012B0F93632904A914986
:10BA40004046F8F712FF8C48DFF834828E490978B7
:10BA5000012902D12168B1F8B07101250095216852
:10BA60003AB2A1464B7D17468449F8F7C7FE044613
:10BA7000D9F8000090F85012890707D40095037D8B
:10BA80003A4680494046F8F7B9FE0443012C04D1F8
:10BA90007E480126417801B945703046BDE8FC87F3
:10BAA000704770B56E4C7A482168027891F8C810DA
:10BAB000CB0723D08B0721D5764B1B78C1F38205AA
:10BAC000012101FA05F52B4214D00170C8B282425F
:10BAD00014D0012810D0CD2001F03FFA206890F852
:10BAE0001001C0060AD5BDE870404FF480710520F2
:10BAF000F4F7C4BC0021E8E7CC20EDE770BD2DE9E8
:10BB0000F04765494FF00009C1F80090FFF7C9FF01
:10BB100050484F4D007820B1F7F72BFAC5F8009048
:10BB200077E64F48006890F81001800701D5F7F7D5
:10BB300098F84A4C20780128F0D00620F4F78FFDC1
:10BB4000FFF7F8FE0646FFF703FD0746FFF7B7FCD1
:10BB500082460620F4F79EFD50492868DFF82C81C4
:10BB60000860012E01D0012F22D12078022801D0B7
:10BB7000032809D198F80100012805D100F0A2F8A6
:10BB800001210220F4F77AFC2078072804D0062847
:10BB900002D0022803D007E04FF4007105E02868C6
:10BBA000002801DB082100E004210320F4F766FCF3
:10BBB000BAF1010F06D12078072813D00421042000
:10BBC000F4F75CFC20780628A8D128680028A5DABC
:10BBD00098F801000028A1D10620F4F740FD3E436B
:10BBE00002D008E04021EAE72878800703D001214D
:10BBF000002001F046FF0620F4F74CFD8EE7002000
:10BC000070472DE9F0438946154909684C7D0B7D45
:10BC1000641C012117E000BF4A1C01FB03F55A43D5
:10BC200000EB450600EB420709EB4505002207E063
:10BC300036F812C037F81280C44425F812C0521CDE
:10BC40009A42F5DB491CA142E6DBBDE8F083000027
:10BC5000740410007C57100040B20120CC02100088
:10BC60003C021000400D10004C1901204C1801201E
:10BC7000442B0120802B0120B450100054170120C8
:10BC8000F0501000901701207302100048041000BB
:10BC90006F0210004B000020F8021000A8021000F4
:10BCA000FC4AFD4BA2F124010879125C1A70401C79
:10BCB000C0B20871042801D100200871704780B219
:10BCC000F4F74BBFF4F76FBF10B501462022F348DD
:10BCD000F8F76CFC0221BDE810400846F4F7CEBB33
:10BCE00070B5EF4D0446286890F8FD06C0072CD0CB
:10BCF0002078EC4E10F0060F15D0A078800712D4F3
:10BD0000F8F7DAFE012821D0608840F00200608058
:10BD1000286890F8FD06000717D520210620F4F7C3
:10BD2000ADFB01203070286890F8FD0600070CD5A7
:10BD30003078012809D1F8F7BFFE012805D110217C
:10BD40000620F4F79BFB0020307070BD2088C0F304
:10BD500041010329E7D140F006002080E3E7D04904
:10BD60004CF2030209688B7BC97B42EA034242EA38
:10BD70000161490041F00101C1607047CA49097879
:10BD8000022915D1C649096891F8101189060FD505
:10BD9000C04924390A46CB7A9269012B09D0012384
:10BDA000CB7242F000528A61C16801F05531C16026
:10BDB00070470023CB7242F080528A61BB4AC1684F
:10BDC0001140F4E72DE9F04399B005466846F8F7CD
:10BDD0001DFCB04CB648243CB64AA56101881180D0
:10BDE000B549B14EDFF8B88249880180E8074FF0C5
:10BDF00001074FF0000971D0BDF8000040F00102CA
:10BE0000ADF80020D8F8000090F8B0309B060DD5B2
:10BE100090F8D13003F00F035B1C042B06D842F4DA
:10BE20000062ADF8002045F48042A26190F8F2264D
:10BE3000D2070ED03278072A0BD0062A09D0BDF8D7
:10BE4000022022F48062ADF80220A26942F400527E
:10BE5000A26190F86120120705D5BDF8002042F4D8
:10BE60008072ADF8002090F82011DFF850C2944A9B
:10BE7000CB0701D0137833B190F80337DB0730D00C
:10BE8000C9072CD02DE0317804291CD0002D1ADBF5
:10BE900090F822118DF8171090F821118DF81E10CE
:10BEA00090F8231135E000BF8DF86070A16921F48E
:10BEB0000051A16133E0A06940F48060A061684650
:10BEC000FFF75CFF36E090F8F206800709D5002DF9
:10BED00009DBA06940F48050A0612BE051E01178AB
:10BEE00021B1002D26DA8CF8009037E0317807294F
:10BEF00003D0062901D00229E5D1002DE3DB90F81B
:10BF000005178DF8171090F804178DF81E1090F88B
:10BF100006178DF8221090F8F216C907C4D190F8D0
:10BF200061000007C7D5BDF8000020F48070ADF8AF
:10BF30000000C0E79CF8000001280FD1D8F80000ED
:10BF400090F85012C90709D090F81001000605D5E5
:10BF5000002D03DB4FF48060ADF80000E80505D547
:10BF6000BDF8000040F48060ADF80000E0780128E2
:10BF700007D03078072801D0062802D16846FFF79D
:10BF8000EEFEA80705D5BDF8000040F00800ADF8AA
:10BF9000000015F0140F20D0D8F8000090F8A01180
:10BFA000C90706D090F89417C90702D03178032941
:10BFB00007D0317802291DD007291BD0062919D0B6
:10BFC00005E0BDF8000040F01000ADF80000BDF83D
:10BFD000000040F00600ADF800006846FFF780FE64
:10BFE000AFF21B30029027726846F5F700FD19B0DA
:10BFF000BDE8F083002D01DA022910D090F8F82670
:10C00000D20703D090F8FB268DF84820BDF8002019
:10C01000062942F00202ADF8002007D020E0BDF86A
:10C02000000040F00600ADF8000019E090F802179B
:10C0300009B18DF84410BDF8021040F202221143FC
:10C0400021F02001ADF80210A16941F08041A16109
:10C0500090F8F816C90703D090F8FA068DF8480052
:10C060008DF84690A06940F08000A061B5E70C49CA
:10C07000096891F8FC20104491F85027C0F38D0016
:10C08000801A80B20C2800D20C2091F8D210401AED
:10C09000C0B2704780041000200000207C571000C0
:10C0A0003C0210000A031000CC021000ABAAAAAA9E
:10C0B000DC021000DA021000D8261000570210002F
:10C0C000720210002DE9FC47DFF8FC83D8F800006D
:10C0D00090F8DA06C0077CD0FC4EB71C30785A289E
:10C0E00001D0C52802D138785A2872D0F8F7E4FC7C
:10C0F00001286ED100242046F4F7B1FAF6F79EF835
:10C10000F34D28800020F4F7C5FAD8F800304246F5
:10C11000B3F8DC1601EB51000FFA80F828884FEADB
:10C12000510C604501DB404507DD02B00202BDE86D
:10C13000F04701218A2000F028BE914693F8DE26C0
:10C14000A8460A445A25824208D393F8DF26891A62
:10C15000814203DC0202357002214EE0DD4989890B
:10C1600089B2A1F5AA42AA3A44D00020F4F777FA9E
:10C1700001A96846F6F789F8D9F80000B8F8001068
:10C18000B0F9DC2690F8DB06511A91FBF0F09DF82F
:10C190000010084404B2002C01DA002402E00F2C45
:10C1A00000DD0F2441EA042203218A2000F0EDFD86
:10C1B000E0B28DF800009DF80410F6F778F8F6F775
:10C1C0003DF80446B8F80000042140EA04428A2001
:10C1D00000E051E000F0D9FDA8F800400020F4F79D
:10C1E00059FABA499DF80000491C0870C520307002
:10C1F000012405E00202357005218A2000F0C5FD0A
:10C20000D9F80000B44B90F8DA0680070ED5B8F8DC
:10C210000000FFF72CFF064618703D7032460621DD
:10C220008A2000F0B2FD26B1012404E0002018703D
:10C230003D70012C06D101210846F9F7DEFD0020F2
:10C24000FAF76CFB0FF04BFF012C15D1A34840F619
:10C25000B772016811430160A148016841F40051BF
:10C260000160A048016841F400110160A102BDE82D
:10C27000FC470120F4F702B9BDE8FC879A4810B5E5
:10C2800001789A4A904802299379006811D00629CA
:10C2900019D007291AD0012B1BD0022B1CD090F8E3
:10C2A000134100BF90F810315B062AD5042916D03F
:10C2B00026E090F81741022BF4D190F81531A342F3
:10C2C000F0DD1C46EEE790F81841EBE790F81941D5
:10C2D000E8E790F81441E5E790F81541E2E7937A32
:10C2E000042B02D090F81B31537292F90930002BC5
:10C2F00002DD5B1E537203E0D3690BB990F80F4166
:10C30000917204B91424F4F720FD002800DD6400C4
:10C31000204610BDF0B56C49054600200C6894F825
:10C320002070F9071BD070490A787049022A17D08B
:10C33000072A15D0062A13D094F839306C4E367877
:10C340001EB194F84944E40707D06A4C24780CB134
:10C35000BC0602D5684C2478CCB15A42CA60F0BD04
:10C36000664B1B78012B0CD0072A0DD0062A0BD068
:10C3700094F83A300E78032EE0D2761C0E70CB6023
:10C38000DCE794F83F30F5E794F85630F2E7CC68F4
:10C39000641CCC609C42E2DD0023CB6058490978E4
:10C3A00001B9012040F002002EB9072A03D0062A65
:10C3B00001D040F01400284040F00040F0BD10B51E
:10C3C0004A4B02460020484C1B690146062A02D00F
:10C3D000072A0BD00DE04B480278012A05D0062031
:10C3E0002070580704D5042003E001700720207056
:10C3F0000120454A18401170404A117010BD2DE9C6
:10C40000F04F0026DFF8E4900346B046D9F810500C
:10C4100030463746B446E907324610D03B493C4CDB
:10C420000978012909D03249097831B921780129DF
:10C4300003D038490978012901D1227001274946E2
:10C44000AC0704D52C4C2478012C00D101276C07B3
:10C4500009D5284C2478012C03D02F4C2478012CAA
:10C4600001D14FF0010C184CDFF8B0A0DFF88CB010
:10C47000DFF874902468012F06D0042B06D0032B1C
:10C480000ED0022B63D065E0CA616FE00A62C86912
:10C49000401CC86194F85D71874267DACA6160E048
:10C4A0001F4F3F78012F3FD01E4F3F78012F3BD0C9
:10C4B0009AF80070012F37D094F81071FF0749D017
:10C4C000CF79012F32D045E03C021000ECFF010093
:10C4D000AA0310005C291000EFFF010048021000C1
:10C4E0004C02100050021000CC0210005C0410003E
:10C4F0005D02100062021000650210005802100078
:10C50000670210004A041000570210006002100079
:10C51000630210004904100064021000D7021000EA
:10C52000B0021000B10210000A6213E00F6A7F1C13
:10C530000F6294F812C10CEB8C0CB7EB4C0F09D3C3
:10C540000A628BF800200120FE4E307013E0BCF12F
:10C55000010F04D0032B04D0022B0CD016E0CA61CB
:10C560000A62032789F8007017200FE0042789F872
:10C57000007003200AE0022689F80060012668079F
:10C5800003D516204FF0010800E0132099F8007041
:10C590009F4201D08AF8002094F850322840DB07EF
:10C5A0000FD094F82032DB0709D194F81A34DB0756
:10C5B00005D194F810311B0603D5022F01D140F4A8
:10C5C0008070E14B002E1E708BF8008000D10A7045
:10C5D000BDE8F08F2DE9F041DC4FDD4E01243868D5
:10C5E00090F81001C106307800D50446D94D0021DD
:10C5F0000428696108D0032806D0022804D0062840
:10C6000005D0072803D007E0FFF7F9FE01E0FFF7A8
:10C61000D6FE6969084368612869FFF77BFE69698E
:10C6200008436861307884420AD0386890F8100175
:10C63000C00605D5BDE8F04140210520F3F71EBF37
:10C64000BDE8F0817CB5C14C206890F8E602C007D7
:10C6500001D0FFF725FBFFF7BDFFBF4908680028A1
:10C6600009DDBE4A127832B9401E086003D10221AA
:10C670000620F3F703FFFFF701FE0646FFF71FFB57
:10C68000B44D40F217316869084239D0FFF71AFDFE
:10C690000020F3F7E4FF6869FFF794FB02216B4683
:10C6A00000220846F3F73AFF02210846F3F715FF88
:10C6B00001A90520F3F721FF0198A8B1F4F773FA57
:10C6C0004FF480410520F3F7D9FE4FF400556B4637
:10C6D000002229460220F3F721FF29460220F3F722
:10C6E000FCFE3046FFF7EBFA206890F8E602C00740
:10C6F00001D0FFF7D5FAFFF702FA0020F3F7CAFFDF
:10C700007CBD10B501210220F3F7E7FEBDE8104023
:10C7100098E710B54FF480610220F3F7DEFE8C48F5
:10C720000178022901D1032101708A490020C871D2
:10C7300010BD10B54FF400610220F3F7CEFE85491D
:10C740000120C87110BD2DE9F04140210220F3F70E
:10C75000C4FE7E4C0120824D824E226812E00021F0
:10C760000CE0032803DB577DBF1E874205DA00FB80
:10C77000031335F8137026F81370491C137D8B4290
:10C78000EFDC401C517D8142E9DA714801780129D2
:10C7900017D006210170FEF783FC73490120087051
:10C7A0006C490020C861086267490870206890F8E9
:10C7B0001001C00605D5BDE8F04140210520F3F782
:10C7C0005DBE3DE763490020684A486188611060AA
:10C7D000C8610862C8605C490870654908706549AD
:10C7E000087056E42DE9F041002704210220F3F7F8
:10C7F00074FE6148574E0568306990EA050420D000
:10C800002C404FF6FF7807D030B90127414602206F
:10C81000F3F763FEFFF7D6FF600701D5FEF747FC8D
:10C820004B4C356175B10321012F15D020780228BA
:10C8300007D10020444A3062F06110704C4A1070F9
:10C840002170FDE6F4F7AFF9012020704146BDE804
:10C85000F0410220F3F741BEE80702D00420207027
:10C8600000E02170BDE8F041ECE670B50446394DBA
:10C87000000705D508210220F3F72FFE0020A8713C
:10C88000E00605D510210220F3F727FE0120A8714C
:10C89000E00406D54FF480510220F3F71EFE02207B
:10C8A000A8712A48006890F81001C00605D5BDE8B7
:10C8B000704040210520F3F7E1BD70BD10B5F4F7DD
:10C8C00072F9234901200870224900204871BDE80F
:10C8D00010404FF6FF710220F3F7FFBD38B51B4C37
:10C8E00043F25D11206890F81001C00601D543F6AF
:10C8F0005D516B4600220220F3F710FE00984008BD
:10C9000004D0022269465520F8F78DF80098C0053A
:10C9100001D5FFF7D3FF009841F21801084201D07A
:10C92000FFF7A3FF0098400701D5FFF75BFF0098D2
:10C9300040063FD50748002141700549097807297D
:10C9400036D11BE04B041000570210003C021000CF
:10C95000CC0210005C041000380610005D021000CC
:10C96000400D1000A800012048041000A80210008B
:10C9700058021000490410003C061000216891F88C
:10C980001011CA064FEA017108D58078002902DB30
:10C9900002280DD007E003280AD004E0002907DAB6
:10C9A0008078012804D040210220F3F796FD01E0B1
:10C9B000FFF7C9FE206890F81001C00609D500985D
:10C9C000000501D5FFF7B5FE0098400501D5FFF73A
:10C9D000A0FE0098C00701D0FFF793FE38BD504875
:10C9E0000078504910F01F0008D007280CD0421ED4
:10C9F0000A704870421C8A70C870F2E60020087005
:10CA0000012048700222F6E70520087006204870D1
:10CA10000722F0E7444810B5012202704148002186
:10CA20002438424B0161817141618161C1610162C0
:10CA300019703F4B404C19703E4B5B8823803F4C34
:10CA40002380C2710172FF2141728272FFF7C7FF1A
:10CA5000FEF71DFBBDE810405021394810F025BFFE
:10CA600008B502210020F7F7A8F96B4600224FF421
:10CA700000710220F3F752FD02210120F7F79DF922
:10CA8000022269465620F7F7CEFF009880050AD5A6
:10CA9000FFF7C0FF4FF6FF710220F3F71EFD21499B
:10CAA00001202439487108BD1E49002024394871ED
:10CAB00097E61C4C0020243C607106E0607920B1B0
:10CAC0000128FBD1FFF70AFFF8E7FFF7C9FFF5E7F9
:10CAD000144900202439C86108621A4908701A49AB
:10CAE00008707EE610B5F4F75EF80121BDE810404D
:10CAF0000220F3F7C3BC10B50A4C243C207A01286D
:10CB000009D1F4F750F81148006890F8160100B9FF
:10CB10000120FFF7D4F80020207210BD61E600006C
:10CB20002000002080041000CC021000C902100078
:10CB3000D8021000D8261000DA021000DC02100023
:10CB40005800012057021000580210003C0210004B
:10CB500010B504460220F3F782FD2046F4F7FEF8F4
:10CB6000BDE810400220F3F795BDF4F7F7B81CB507
:10CB700000210091019102789DF8001062F30301F9
:10CB80008DF80010427862F307118DF80010428989
:10CB9000BDF8011062F30B01ADF801100289BDF878
:10CBA000021062F30F11ADF8021081798DF80410B4
:10CBB000C1798DF805100179CA099DF8061062F354
:10CBC000C7118DF80610027962F306018DF8061080
:10CBD00080788DF807006846FFF7BAFF1CBD1CB5CA
:10CBE00000200090019002208DF80000FC480068B1
:10CBF000C007400E8DF807006846FFF7A9FF1CBD6F
:10CC00001CB500210091019101788DF80010417848
:10CC10008DF80110C188C1F307118DF802108188C9
:10CC2000C1F307118DF80310017901F00F018DF8A0
:10CC30000410827941EA02118DF8041081788DF890
:10CC40000510C07800F00F008DF80600E448006879
:10CC5000C007400E8DF807006846FFF779FF1CBD3E
:10CC60001CB50021009101910E218DF800108DF866
:10CC70000200DB480068C007400E8DF807006846D8
:10CC8000FFF766FF1CBD1CB5002000900190D54841
:10CC900000684178827810208DF800004006437AC1
:10CCA0008DF80130D04B1B788DF8023043891B0A78
:10CCB0008DF8033040898DF80400C9488DF80510BF
:10CCC0008DF806200068C007400E8DF80700684602
:10CCD000FFF73EFF1CBD1CB5002000900190112005
:10CCE0008DF80000BE480068C007400E8DF80700B0
:10CCF0006846FFF72DFF1CBD2DE9FC4106460020CC
:10CD000000900190122015460C468DF800004FF05F
:10CD100008571EE0200A8DF80100C4F30B008DF8BF
:10CD20000240315C30448DF8031041788DF80410D6
:10CD300081788DF80510C0788DF80600D7F8E001ED
:10CD4000C007400E8DF807006846FFF701FF241D5D
:10CD50002D1F002DDEDCBDE8FC811CB500220092F9
:10CD600001920F228DF800208DF80100080A8DF83D
:10CD700005008DF80610402099498DF80700012024
:10CD800008606846F3F7EAFF1CBD1CB5954B1B68AD
:10CD900093F8F0379B061DD5002300930193DB2306
:10CDA0008DF800308DF801008DF80210100E8DF80E
:10CDB0000300100C8DF80400100A8DF80500884857
:10CDC0008DF806200068C007400E8DF80700684601
:10CDD000FFF7BEFE1CBD1CB5002300930193DB23AF
:10CDE0008DF800308DF801008DF80210100E8DF8CE
:10CDF0000300100C8DF80400100A8DF80500784827
:10CE00008DF806200068C007400E8DF807006846C0
:10CE1000FFF79EFE1CBD1CB50022009201920F225E
:10CE20008DF8002005228DF801208DF802006C4855
:10CE30008DF803100068C007400E8DF807006846A3
:10CE4000FFF786FE1CBD2DE9FC4104460025009538
:10CE500019208DF8000040070195417A8DF80110E6
:10CE6000614909788DF802104189090A8DF803108B
:10CE700040895C4F8DF80400594E386841788DF830
:10CE8000051080788DF806003068C007400E8DF8D8
:10CE900007006846FFF75CFE00951A2001958DF8A3
:10CEA0000000386800F5FC6001788DF801104178C9
:10CEB0008DF8021081788DF80310C0788DF8040089
:10CEC0003068C007400E8DF807006846FFF740FE47
:10CED00000951B2001958DF800006068000E8DF80C
:10CEE00001006068000C8DF80200A088000A8DF82F
:10CEF000030020798DF8040020788DF80500207B50
:10CF00008DF806003068C007400E8DF807006846AF
:10CF1000FFF71EFE00951C2001958DF80000A0680B
:10CF2000000E8DF80100A068000C8DF80200208929
:10CF3000000A8DF80300207A8DF80400207C8DF81B
:10CF40000500207D8DF806003068C007400E8DF882
:10CF500007006846FFF7FCFDFDE61CB5214909689E
:10CF600091F82911490603D400F00F010C2919D1B9
:10CF700000210091019116218DF800108DF801001B
:10CF8000010A8DF80210010C000E8DF804001448FF
:10CF90008DF803100068C007400E8DF80700684642
:10CFA000FFF7D6FD1CBD1CB500230093019316238B
:10CFB0008DF800308DF80100080A8DF80200100A83
:10CFC0008DF8040006488DF803108DF805200068E0
:10CFD000C007400E8DF807006846FFF7B9FD1CBD7D
:10CFE000E00100223C021000D60210001CB5002314
:10CFF00000938DF80000080A8DF802000193100AD2
:10D000008DF805000F488DF803108DF80620006894
:10D01000C007400E8DF807006846FFF799FDDEE770
:10D020001CB500200090019080208DF8000005487C
:10D030000068C007400E8DF807006846FFF788FDBE
:10D04000CDE70000E00100228A48006890F82A013C
:10D0500000F00700801C00EB8000C006000EF3F714
:10D0600011BD2DE9F041844D286820B30520F3F768
:10D07000F6FA00245FF00107286807FA04F6304248
:10D0800013D004EB440005EB800898F8060005284F
:10D090000BD104217948F6F709FCC1B208F106006A
:10D0A000FFF765FD2868B0432860641C0A2CE3D3B1
:10D0B0000520F3F7EFFA7148001F4068002802D0FE
:10D0C000BDE8F041C0E7BDE8F081F3F7E8BC6A498C
:10D0D00000EB400210B501EB820101248B79674916
:10D0E000091F032B4A6802D0042B04D006E08440B9
:10D0F00014434C6002E08440A2434A6004215F482C
:10D10000F6F7D4FBC0B210BD2DE9F0475B4E052009
:10D11000361F7768F3F7A3FADFF85891564D0024CD
:10D120004FF00108296808FA04F0014225D004EB09
:10D13000440205EB820A9AF80620032A09D0042A41
:10D1400007D0052A19D1D9F8002092F82921D20652
:10D1500013D481432960D9F8000090F81001C0066B
:10D1600003D547480078072807D060B2FFF7AFFF24
:10D1700001460AF10600FFF7FAFC641C0A2CD1D321
:10D180000520F3F787FAD9F8000090F82901C006C6
:10D190000CD570682FB1002808D1BDE8F047F3F72F
:10D1A0007EBC002802D0BDE8F0474DE7BDE8F0871F
:10D1B00032490020091F486080212F4810F075BBBC
:10D1C0002E4C08B5241F00252570F3F768FC207845
:10D1D00050B30128FBD100226B4607211046F3F71C
:10D1E0009DF90098400706D504210020F3F775F952
:10D1F000F3F755FC25700098800705D50221002023
:10D20000F3F76BF9FFF780FF0098C007DFD001212B
:10D210000020F3F762F91748006890F82901C0066A
:10D22000D5D5FFF71EFFD2E700210846F6F7C5FD6A
:10D2300000226B4608211046F3F770F90021012007
:10D24000F6F7BBFD00980007C1D5FFF7B1FFF3F774
:10D2500026FC0F210020F3F740F901202070B6E7EB
:10D2600010B5F3F71CFC0121BDE810400020F3F7D6
:10D2700005B900003C021000582610008804100078
:10D28000CC021000FC49002001220870FB490A7002
:10D290004870886008718870C8700C310860888098
:10D2A000F749086048608860C86008614861704755
:10D2B0002DE9F04F8B46F349002305460E681846CA
:10D2C0001A4696F8E841012101FA02F73C4204D0DF
:10D2D00035F912709F4200DD3B46521C062AF3DBF3
:10D2E00096F868224FF0640A5A4392FBFAF2E64B32
:10D2F0000FFA82F8002293F8009000BF01FA02F3BF
:10D300001C4258D0E14F3F78012F12D196F8E6C168
:10D310001CF0300F07D0B9F1040F04D03BF91270A4
:10D32000CCF3011C20E05FEA9C1702D0B9F1040F96
:10D3300016D0D74F3F78012F19D035F912703BF92D
:10D3400012C0674503DD474501DD0343D8B296F8B7
:10D350005F341B072FD5CF4B1B78012B13D02AE04E
:10D360003BF912704FEA9C1C97FBFCF704E03BF979
:10D370001270B6F81EC2674435F912C067451ADA52
:10D380000343D8B217E0531E01FA03FC14EA0C0F52
:10D3900011D01CEA000F0ED0002A0CDD96F855348F
:10D3A0005F4397FBFAF305EB420737F9027CBB4278
:10D3B00001DD20EA0C00521C062A9FDBBDE8F08F3D
:10D3C000F0B5B04BAD4F01241A6892F8FC2102F081
:10D3D0000F053A78C5F11006012A4FF0000211D16D
:10D3E0001D6804FA02F695F8E851354203D030F88A
:10D3F000125021F81250521C12B2062AF0DB002003
:10D40000387016E01F6804FA02FC97F8E87117EA12
:10D410000C0F0AD030F9127031F912C077430CFBAF
:10D42000057747F30F1721F81270521C12B2062A23
:10D43000E8DB186890F8E601000706D59248007806
:10D44000042802D1944800880880F0BDF0B500237C
:10D450008C4D012404FA03F72E6896F8E8613E42E9
:10D4600006D032F8136030F81370F61B21F8136001
:10D470005B1C1BB2062BEDDBF0BDF0B5DFF8FCC189
:10D48000034600229CF803000CF10C0583EA000619
:10D490007C480124D0F8007004FA02F030420BD02E
:10D4A000184297F8E70102D004EB101002E000F0F8
:10D4B0000F00401CA85411E015F802E0BEF1000F67
:10D4C0000CD0AEF1010E1EF0FF0E05F802E005D102
:10D4D000184202D00843C1B200E08143521C062A20
:10D4E000DADB8CF803300846F0BDF1B59DF800009A
:10D4F000002823D001216846F6F7D8F9C0B20128E8
:10D500001DD05E4A9078002818D15E4C00215C4DF9
:10D5100024680123084694F8E8610C3503FA00F406
:10D52000264205D035F910408C4201DD21461071AC
:10D53000401C0628F2DB10798340D8B2F8BD9DF874
:10D540000000F8BDF0B54F4B00252C461B682A465D
:10D55000012793F8E86100BF07FA02F31E4211D0D9
:10D5600030F91230002B01DB9C4601E0C3F1000CC6
:10D570008C4507DD002B01DD1D4403E001DAC3F11A
:10D5800000031C4402F10102062AE5DBA54201D298
:10D590000120F0BD0020F0BD2DE9FE4F00240094D5
:10D5A0000194274636490294FFF70AFF0320F3F758
:10D5B00056F83349384A0C313148FFF747FF03200A
:10D5C000F3F768F82F4D286890F81011C90626D592
:10D5D0003249098811F4405F21D0012100F5F4702F
:10D5E000F6F764F94FF6FF7606EA400124480FF09B
:10D5F00022F8DFF8AC800121A8F81A00286800F5AD
:10D60000F470F6F753F906EA40011D480C300FF0AC
:10D6100012F8A8F81800711C0520F2F72FFF2868EF
:10D62000DFF880A0144E90F8E6114FF00109490789
:10D6300051D5DFF84880DFF870B098F8011079B163
:10D64000D8F808204146521CC8F8082090F8FF017D
:10D65000000900EB8000B2EB400F3CDD8C6044E041
:10D66000B0F8FD1106480C30FFF76CFF01281DD003
:10D67000C8F808402FE00000650210008C0410007C
:10D6800080D001203C0210007202100061021000E4
:10D6900067021000730210006813012028061000B2
:10D6A000D0271000480210004C021000D8F80810D3
:10D6B00040464A1CC8F808202A6892F8FF2102F068
:10D6C0000F0303EB8303B1EB430F04DD80F80190FC
:10D6D0008460110909D0DFF810B19BF8000001281F
:10D6E00012D0296801F5F8712AE088F80140DAF8CB
:10D6F000001041F01001CAF80010DBF8001041F4EE
:10D700008011CBF800104AE028686B4600F5F871EC
:10D710004FF0640C90F8E88109FA07F218EA020F5A
:10D7200009D031F8172090F81F8302FB08F2B2FBF2
:10D73000FCF223F817207F1CFFB2062FEAD319460C
:10D740002A48FFF7B5FD2A4A1178C82902D201F10B
:10D75000010100E0C821C9B211702B6893F85F2461
:10D76000520724D59BF80020012A20D1142938D350
:10D77000204A2149012818D9C50716D082F80090FF
:10D780000D786D1CEDB20D70282D10D90C70147031
:10D79000DAF8001041F01101CAF8001034704FF4AB
:10D7A00080610120F2F76AFE1BE00C70147040B13A
:10D7B00086F8009093F8E611890703D5FFF795FEE8
:10D7C00000E034700D490978012900D100200C4C8B
:10D7D000A178FFF752FEA178884202D0A070FFF72F
:10D7E0003FFA3078BDE8FE8F730210008CD0012024
:10D7F00074021000750210007602100084021000FE
:10D800008C0410002DE9FE43E14E1023DFF88483E1
:10D810003068DFF88493457D90F814C02C4690F86A
:10D82000232004FB0CF1A3EB12140023CDE90031FB
:10D830001709012202926D1CB0F92830B0F9262098
:10D8400005FB0CF508EB4C0109EB4C00F6F7EEFF7D
:10D8500000282AD1336841464E46187D11E000BFAA
:10D8600031F910C036F910200CFB07FC02FB04C292
:10D870004FEAE27C02EB1C7242F30F1221F81020F7
:10D88000401CA842ECDB93F8200000070DD5C148EE
:10D89000F6F7F3FCC1490023C14A086003B0014612
:10D8A000BDE8F043BB48F6F71FBDBDE8FE83F0B509
:10D8B000B748016891F8E80100282CD091F82400BD
:10D8C000B84A00F00F040020C4F11007012600BF81
:10D8D00091F8E83106FA00F52B4219D0B24B32F933
:10D8E0001050B1F933C333F91030AC449C450FDB11
:10D8F000B1F935C3A5EB0C0C9C4509DC654303FB72
:10D900000753DD1703EB157343F30F1322F81030A1
:10D91000401C0628DCDBF0BD2DE9FE4F9C49086861
:10D9200090F85022D2077DD0894690F82310B0F8A5
:10D93000314301F00F059D49C5F110060978012911
:10D9400001D1B0F83E479A499A48F6F78EF99A49BC
:10D950009848F6F7B0F9D9F80000DFF854C2964FAE
:10D9600090F8211249061CD5427DB0F93412CDE958
:10D970000012B0F932324F46904A91496046F6F7AC
:10D9800074FF3868027DB0F93812CDE90012B0F9A1
:10D9900036328C4A8C498848F6F767FFDFF81CC29C
:10D9A000884FD9F800004FF00008CA46427DCDF8F4
:10D9B0000880CDE90082B0F92F2323B2994680492F
:10D9C0006046F6F733FF0446DAF800004B467E491E
:10D9D000027DCDF80880CDE90082B0F92F233846CA
:10D9E000F6F724FF54EA000149D10020704F744B30
:10D9F0005446DAF800100FE033F9102037F910C060
:10DA00006A430CFB06224FEAE27C02EB1C7242F3F3
:10DA10000F1223F81020401C4A7D8242ECDC0020CB
:10DA2000654F00E02BE0684B10E000BF33F9102099
:10DA300037F910C06A430CFB06224FEAE27C02EB86
:10DA40001C7242F30F1223F81020401C0A7D824200
:10DA5000ECDC91F82000000711D55C4D5848C5F862
:10DA60000080497DF6F7FEFC29680844286020689C
:10DA7000017D5548F6F7F6FC296808442860BDE8A2
:10DA8000FE8F2DE9F047424C80460E462068032267
:10DA90004FF4007990F85A1402EB41074C49097889
:10DAA000072936D0062934D04A49097889BB90F82D
:10DAB0004904400603D5FAF72AFA012801D05EB1DD
:10DAC00013E0206890F81001C0065FD54946BDE814
:10DAD000F0470520F2F7D2BC206890F84904C0074F
:10DAE00003D0FAF721FB0128EBD03B4D2878B84250
:10DAF00009D246B9206890F84904000603D5FAF720
:10DB0000ADF90128DDD02878B84202D200F1010039
:10DB1000287046B9206890F8C206000603D5FAF7C7
:10DB2000E3FC0128CDD0206890F82000C0072DD05C
:10DB30002A4E2B4DB8F1000F0AD02A480078002851
:10DB400024D12888C00521D50320F2F788FD0FE0F5
:10DB50000320F2F784FD2878C00701D0FFF752FEBA
:10DB60002878800701D5FFF7A2FE2888C00508D5D0
:10DB7000206890F85102000701D5307808B9FFF706
:10DB8000CBFEBDE8F0470320F2F784BDBDE8F08787
:10DB90003C021000A8000120400D1000A00210005F
:10DBA0003826100068130120BC2A012073021000DF
:10DBB000442B01204C190120802B0120B45010006F
:10DBC00054170120F050100090170120EC041000B1
:10DBD000CC021000720210009E0410001A05100002
:10DBE000A802100044021000FE490020087070478F
:10DBF00000E010460A5C8242FBD1704770B50025F8
:10DC00000E4603462C4606E019462046FFF7F0FF75
:10DC10001855641CE4B2B442F6D300220AE0985CC2
:10DC2000904203D19D546D1CEDB201E0185C9854F4
:10DC3000521CD2B2B242F2D3284670BD38B18842EB
:10DC400002D20B4601461846884200D011540846BD
:10DC500070472DE9FF4F99B001200490E248196800
:10DC60009A460068067D477D41B19AF802109AF8FD
:10DC700000905046B14205D2491C04E04FF0000923
:10DC80004D4608E0314645789AF80300CEB2B842D6
:10DC900000D2471CFFB2002007A90854401C2D28C1
:10DCA000FAD3199905EB051001EB400C681C67E0ED
:10DCB0001998E34608EB081100EB410C09F1010447
:10DCC0005AE000BF0CEB04001590006810B31CF87C
:10DCD000040000B31598002310F8010C00B10346AE
:10DCE0001BF8041021B107AA1846FFF7A7FF034647
:10DCF0001A9800280BEB04000ED0159010F8011CA8
:10DD000021B107AA1846FFF799FF034615984178F5
:10DD1000D9B91FE0E41C2EE0189010F8011C59B18D
:10DD200015981BF8042010F8010C104304D007AA22
:10DD30001846FFF783FF03461898417851B11598AC
:10DD40001BF804204078104304D007AA1846FFF7B8
:10DD500075FF034613B10CF804300CE004982D282D
:10DD600006D20CF804000498401CC0B2049002E0F3
:10DD7000401E0CF80400641CB442A3D908F1010051
:10DD80008046B84294D907A80499FFF737FF804628
:10DD900041001B980FF067FD00204FF6FF7202E074
:10DDA0004AF82020401C4045FAD33BE0199905EB86
:10DDB000051001EB400022304C4605902FE00598FD
:10DDC000011901204058A8B3487838B307AA105C5D
:10DDD00048701B991B9A0AEB800B31F81010491CF4
:10DDE00022F810109BF800102046F5F772FD8BF812
:10DDF00000009BF801102846F5F76BFD8BF8010039
:10DE00009BF802102046F5F76CFD8BF802009BF89A
:10DE100003102846F5F765FD8BF80300641CB44237
:10DE2000CDD36D1CBD42C1D3A8F101001DB0C0B25D
:10DE3000BDE8F08FFFE7E41CF0E72DE9F0439946D9
:10DE400055784FF0010C1BE005EB051300EB430682
:10DE500022360023147897780CE000BF06EB040804
:10DE600098F90180884503D10CFA04F848EA0303C5
:10DE7000641CE4B2A742F1D249F825306D1CEDB222
:10DE8000D378AB42E0D2BDE8F083F0B5554B002625
:10DE9000554D1C78A0B0012C11D11E700B78002BB1
:10DEA0005AD04B78002B57D02B688F781C7D641E7E
:10DEB000A74251D05B7DCC785B1E9C424CD00023A6
:10DEC0004FEA0D0444F823605B1C202BFAD34B78F7
:10DED00091F803C01BE000BF50F82370B7B17E0873
:10DEE00046EA47063E4354F82370374344F823700C
:10DEF00004EB8307D7F804E04EEA060EC7F804E007
:10DF0000D7F808E04EEA060EC7F808E05B1C9C450F
:10DF1000E2D2002304EB8306766840F823605B1CA2
:10DF20001E2BF7D3012A17D1087808B1401E0870BC
:10DF3000487808B1401E48702A688878127D521EC1
:10DF4000904201DA401C88702A68C878527D521EBF
:10DF5000904201DA401CC87020B0F0BD2DE9F74FA7
:10DF60004D78DFF88890DFF880B04FF0030E79E04D
:10DF700000986C1C936A50F82560DBF80000007D67
:10DF80006043D9F8004003EB400304EB40070C78F2
:10DF9000641C012014E000BF00FA04FC1CEA060F18
:10DFA0000DD003EB440A33F914803AF902CCE04473
:10DFB000BAF902C0E04498FBFEFC27F814C0641CC8
:10DFC00091F802C0A445E7DC91F800A0BAF1000F77
:10DFD0002DD000FA0AF4344214D003EB4A0434F989
:10DFE000028C05E0A00410003C0210009802100012
:10DFF00033F91AC0B4F90240C444A4449CFBFEF4B3
:10E0000027F81A40DBF800C08C789CF814C0A445AF
:10E0100000FA04F000EA060014D110B303EB440048
:10E0200033F9143030F9020C1844401017E016F0A0
:10E03000010FE7D0B3F90040B3F902C064446410A3
:10E040003C80DFE768B103EB440033F9143030F96A
:10E05000026CB0F902003344034493FBFEF027F84E
:10E0600014006D1CC878A84282DAD9F800009062CA
:10E07000BDE8FE8FF0B50025059E2C468F1E00EBF7
:10E08000410006D430F9045CCF1E02D430F9067C7E
:10E090003D448F1C974207DAB0F90440C91C9142F5
:10E0A00002DAB0F906000444281B00D540424FF4C0
:10E0B00035714843C11700EB91508012A54203DD32
:10E0C000316808443060F0BD196808441860F0BD3C
:10E0D0002DE9FF4FDFF808B407460E46DBF80000D5
:10E0E000002585B090F8A0002C46C106FD484FF4ED
:10E0F000803900EB460A29D5002105E037F81120C8
:10E1000000EB4103491C5A80B142F7D3418801809A
:10E1100030F81620AAF8022000210DE04A1C00EB7E
:10E12000420330F8122033F802CC5B88634403EBDF
:10E13000420227F81120491CB142EFD307A800235F
:10E140000090324619463846F6F707FC07994FF01B
:10E15000000800291CDCDBF8000090F8A000C006D5
:10E1600004D5E048B0F90000019001E0CDF804804A
:10E17000701E37F911C00390814224DBDBF80000E8
:10E1800090F8A000C00608D5BAF90200029006E097
:10E1900007EB410030F9020CE6E7CDF80880DBF828
:10E1A000000090F8A000000706D502A8009001AB7F
:10E1B000721E3846FFF75EFFDDE90110814207DD80
:10E1C00005460C4607E007EB4100B0F90200DDE729
:10E1D00001DA0D460446A0EB0102A2FB09064FEA54
:10E1E000E27303FB096102FB08110CEB0402C5F1A9
:10E1F000000302EB43024FEAE2730FF0C3FA079CFD
:10E20000A4FB0936E51705FB096204FB08221B186D
:10E210004A410899A3FB0105CC1702FB015103FBFE
:10E2200004114A4600230FF0ADFA039AD3170FF0FA
:10E23000A9FA00B209B0FBE52DE9FF4F044681B011
:10E240000020DFF89C920F9D064607460090D9F803
:10E25000000090F8A000000719D5207808B1401EF2
:10E260002070607808B1401E6070D9F80020A07856
:10E27000127D521E904201DA401CA070D9F80010A5
:10E28000E078497D491E884201DA401CE0709548DB
:10E29000442144380FF0E7FA002293469246607812
:10E2A00030E021782AE000BFD9F80030D5F8288086
:10E2B00093F814C0431CE64603FB0C1C08EB4C0C03
:10E2C000DDF80080BCF900C0C44502DD761CB6B2A2
:10E2D0006744944502DD62468B46824695F818C035
:10E2E000BCF1010F09D10EFB03FC7F4B0B441CF862
:10E2F000038048F080080CF80380491CA3788B4207
:10E30000D2DA401CE1788142CBDA6078D9F800108B
:10E310000FE000BF91F814C000F1010808FB0CB237
:10E32000AB6A03EB420213886E4A443A22F810307B
:10E33000401CE2788242EDDA6A48497D5246443810
:10E34000039BFFF7C5FE0E990860664844214438D8
:10E350000FF089FADFF88C812078A8F144080AF1DF
:10E360000101D9F800200AE092F814C0AB6A01FB61
:10E370000C0C03EB4C031B8828F81030401CA378CE
:10E380008342F1DA5748117D5A464438029BFFF721
:10E390009FFE04990860EF602E8105B048E5F0B556
:10E3A0004F4C059F2668D6F8105296F81842BD4289
:10E3B00002D304F00F040FE0D6F81462BE4201D875
:10E3C000240909E004F00F0CCCEB14147F1B7C43F0
:10E3D000751BB4FBF5F464441668C4F11005604382
:10E3E00006FB0500000910601868614300FB05107A
:10E3F00000091860F0BD2DE9FF4F3948964684B0FA
:10E400000D7891F80190CA7800680024897802900C
:10E41000007D2346A0465FEA050B29D1CC4625E0C6
:10E420000CF101060196DEF828604FF0000A012584
:10E43000009609E0DDE9006707FB005706EB470699
:10E440006D1CB6F90070BA44A942F3DADDE9006543
:10E45000454306EB4505B5F900506D4395FBFAF5CC
:10E4600005FB0C33641BA8440CF1010C6245D7DAA0
:10E47000451EA9422FD1CC462BE000BF0CF101066E
:10E4800001964E1E0396DEF828604FF0000A5D46A6
:10E49000009609E0DDE9006707FB005706EB470639
:10E4A0006D1CB6F90070BA44039EAE42F2DA019DCB
:10E4B00005FB0016009D05EB4605B5F900506D43C0
:10E4C00095FBFAF505FB0C3305FB0044A8440CF161
:10E4D000010C6245D2DAB9F1000F2BD15D4627E07D
:10E4E0003C021000E0571000D0A70120DEF8287091
:10E4F0004FF0000A012600970AE0771C07FB00573F
:10E50000DDF800C0761C0CEB4707B7F900C0E24409
:10E51000B242F2DA009E471906EB4706B6F90060F0
:10E52000764396FBFAF606FB05449B1BB0446D1C34
:10E53000A942DBDA029D6D7D01956D1EAA422BD1A9
:10E540005D4627E0DEF828704FF0000A4E46A2F143
:10E55000010B00970AE0771C07FB0057DDF800C0AD
:10E56000761C0CEB4707B7F900C0E244B345F2DA7A
:10E57000561C06FB0057009E06EB4706019FB6F9A6
:10E580000060764396FBFAF606FB054406FB07336C
:10E59000B0446D1CA942D5DA07980460079843601F
:10E5A0000798C0F8088008B042E42DE9F04F89B020
:10E5B0004FF00009DFF878B48646CDF81090CDF81A
:10E5C0001490CDF81890DBF8000014460F46B0F810
:10E5D0006820217E4D464E46C84609B9B0F8C8218C
:10E5E00078783BE05EF820A03878039030E0012096
:10E5F000884010EA0A0F29D0DBF80000D4F828C0C0
:10E60000029B007D01935B1C009303FB00130CEB4A
:10E610004303B3F90030934208DDDDF804C001FB89
:10E6200003660CFB03881D4409F10109237E012BBD
:10E630007AD0002B009B00FB03F0FE4B0B4410F83C
:10E6400003C07AD04CF0200C00F803C0491C0391A1
:10E65000B87803998842CADA0298401C0290F97887
:10E660008142BFDADBF8000090F8600000060BD5AD
:10E6700004AB224639467046FFF7BDFE0498059963
:10E680000644069888440544E94800230168087D4B
:10E69000CA8A401E00FB05FAA2FB060C03FB06C358
:10E6A000F11702FB01314FEAEA7B52465B460FF05D
:10E6B00069F80390DE4841464FEAE87600684FF07B
:10E6C000000C427D038B521EA3FB01080CFB018151
:10E6D0006A4303FB06114FEAE27A53460FF052F801
:10E6E00002900398002800DA0020D14E0390316890
:10E6F000C98A814200DB014602980391002800DAB2
:10E70000002002903168098B814200DA08460290AD
:10E71000E560A4F80890207E022811D0012816D0C8
:10E7200000B356E000E008E0009B5843C14B0B44A7
:10E7300010F803C04CF0800C86E74CF0400C83E7E7
:10E74000306890F88000C00643D5002210E03068A1
:10E7500090F88010C90612D590F8A0004007F4D4B4
:10E76000012205E0306890F88000800631D5022251
:10E7700002A903A802F0F2FA207E012829D130680C
:10E7800090F8A010490724D508A9CDE90014B0F9E4
:10E790001820B0F9161007AB3846FFF74DFD30686A
:10E7A00090F88000C00604D5012208A907A802F04D
:10E7B000D5FAE0680090DDE9021008AB07AAFFF780
:10E7C000EEFD08A907A8F5F7CDFF0798E0800898A7
:10E7D000A08002A903A8F5F7C5FF039801B26180E4
:10E7E000029800B22080326892F8A020520701D42B
:10E7F000E180A0801EE52DE9F84F8D4E84460C4641
:10E800003068994692460027B0F9BE56B0F9BC165A
:10E81000B0F9BA26B0F9B8360FFA8CFCB9F1010F8D
:10E8200008D1BAF1010F11D0B0F8B406024418446F
:10E8300012B203B22846CDF800C0F5F724FB85B22A
:10E84000306890F8F1070D2803D00EE0B0F8B60656
:10E85000ECE744EA044200215D20FEF796FA45EA1F
:10E86000044201215D20FEF790FA3068AC4290F836
:10E87000F10708D20D2804D1012202215D20FEF704
:10E8800084FA012706E00D2804D1002202215D2030
:10E89000FEF77BFA306890F8F1070C2806D166483D
:10E8A000B9F1010F05D08484C58407853846BDE8D9
:10E8B000F88FC48205834783F8E770B55C4D002468
:10E8C0002868B0F8BE36B0F8BC26994202D9914209
:10E8D00000D2012490F8F1070D2804D1224600212E
:10E8E0007120FEF752FA286890F8F1070C2801D140
:10E8F00051488482204670BD2DE9F04188464C493C
:10E900000446DDE9060609681F004FF0000506D041
:10E9100001280BD0B1F9AE06012E0ED011E0B1F9ED
:10E92000AA06012E0DD1B1F8AC3608E0B1F9BC034E
:10E93000012E06D1B1F8BE3301E0B1F8B036C01AED
:10E9400000B2844200DD012591F8F1373A49082BE5
:10E9500002D00C2B08D00CE008230B804C80888060
:10E96000CA800D814F8204E0012E05D0C8830C843B
:10E970004D84012D07D014E08A89521C8A81C881F8
:10E980000C824D82F5E721463846FFF796FF0128B5
:10E9900007D133463A4641462046FFF72CFF00B9DF
:10E9A00000252846BDE8F0812DE9F04F9146204A28
:10E9B0008646002348784FF0010BCE78D2F800A0AD
:10E9C0001AE000BF5EF820700A78441C8D7810E0D1
:10E9D0000BFA02FC1CEA070F0AD09AF81480D9F847
:10E9E00028C004FB08280CEB480CBCF900C06344A9
:10E9F000521C9542ECDA401C8642E3DAC9F810302A
:10EA0000BDE8F08F2DE9FC4FA2F101020B4B02EBA8
:10EA1000D27242F34F020DB20093A5EB02030FFA3C
:10EA200083FA05EB02034FF0000B1FB208E0000071
:10EA30003C021000D0A7012018D801203843012043
:10EA40004FEA2144A4EB0201224416B25A4680F850
:10EA50003A2080F83B20FF4A09B2D946136893F860
:10EA60006120D2060CD51DB15A7D521E954207D1A8
:10EA70001CB11A7D521E944202D1012280F83B2023
:10EA8000524665E040F6FF7E0C4618E0002A14DB93
:10EA900093F815C0944510DD002C0EDB93F814C0DC
:10EAA000A4450ADD02F1010808FB0C48DDF800C0AE
:10EAB0003CF918C0F44500DAE646641C24B2B442BE
:10EAC000E4DDB3F868C07446F44500DB0024A646D4
:10EAD000954200D1F3460C4636E0002A2EDB93F82F
:10EAE00015C094452ADD002C28DB93F814C0A445FA
:10EAF00024DD02F1010808FB0C48DDF800C03CF9F8
:10EB000018C0B3F86880E04501DB4FF0000CCDF889
:10EB100004C093F8F1C7BCF10F0F07D1DFF838C379
:10EB20004FF00008ACF81A80ACF81C80DDF804C087
:10EB3000ACEB0E0CCC440FFA8CF903E04FF0010C57
:10EB400080F83AC0641C24B2B442C6DD521C12B232
:10EB5000BA4297DD93F8F1270F2A0ED1BE4A0F2350
:10EB60001380A2F802A09780D1801681A2F80A90A3
:10EB700090F83A009081A2F80EB04846BDE8FC8FAC
:10EB800070B50646B54814460D460278B1480021D6
:10EB9000012A006801D190F87F10227E042A01D05A
:10EBA000022A1CD190F86630628919448A4216D92B
:10EBB00090F881104B064FF003010FD5A84B1B783E
:10EBC000012B0CD1A74B9B78012B03D0A64B9B7834
:10EBD000012B03D190F89606824200D921760422B7
:10EBE000294604F11400F5F7E1FC012229463046DC
:10EBF000FFF74BF9224629463046FFF7D6FC204660
:10EC0000BDE870400AF0BCBB2DE9F041C0B01C4625
:10EC100090466B46FFF711F9224641466846FFF7DA
:10EC2000C3FE924D8B4E924F2878E0B9306890F831
:10EC30002002800717D53878A8B9207E022801D095
:10EC4000012810D18022694620A8F5F7AFFC0122E7
:10EC5000414620A8FFF719F9414620A8226905F08E
:10EC60009AFA012822D0306890F82002000618D5C0
:10EC700080480078A8B9387898B9287888B97E484B
:10EC8000007870B97D487E4900780978084308D13A
:10EC90007C48007828B94146684605F02FFA0028DC
:10ECA00004D0224641466846FFF76AFF40B079E645
:10ECB0002DE9FF4F86468B4600204FF6FF755378AF
:10ECC000D67828E003EB03140EEB440101F122098E
:10ECD000604914789778D1F800A018E009EB040196
:10ECE00091F801C0DC4510D10E999AF81480D1F842
:10ECF0002CC0591C01FB08410CEB410109888842DA
:10ED000000D208468D4200D90D46641C24B2A742A9
:10ED1000E4DA5B1C1BB29E42D4DA039908800D9999
:10ED20000D8004B06CE62DE9F04F9B468246537887
:10ED3000DDF824E02CE000BF534D03EB03100AEB99
:10ED40004004AD68223405EB400522351078414F70
:10ED50004FF0010917E0261876788E4211D13E68EF
:10ED6000DEF82CC096F814805E1C06FB08060CEB3F
:10ED70004606B6F900605E4503DD05EB000C8CF835
:10ED80000190401C00B296788642E4DA5B1C1BB20C
:10ED9000D0789842D0DA33E62DE9F0472D4F8146FE
:10EDA000C8B038681D46884690F8706047A8CDE91D
:10EDB0000005144646AB4846FFF77AFF287E48B95F
:10EDC0002D4800780028386802D090F8EC6601E001
:10EDD00090F8CE61BDF81811BDF81C016422091A23
:10EDE0007143B1FBF2F1284F0E184FF48861B868F7
:10EDF0000EF039FDB3B22246414648460095FFF772
:10EE000092FF2068029002AB2FAA0121B868FEF79A
:10EE100020FF064601283BD901240DF1BC0A0DF163
:10EE20000809B84612E000BF3AF81400688109EBFF
:10EE300084072946384602F05BF82B463A462146BD
:10EE4000D8F80800FFF7E0FE641CE4B2B442EBD946
:10EE500048B01BE03C02100018D801206F021000DF
:10EE6000FC05100064271000F8261000670210004F
:10EE7000680210001A051000720210006A021000E9
:10EE80006B02100073021000A0041000BDE8F087B0
:10EE90002B46224641464846FFF7B6FED8E72DE905
:10EEA000FC4FDDE90B8914789678FE4DDFF8F8B356
:10EEB0002D78DBF80070012D1AD097F87150DFF82B
:10EEC000ECC3AA4603EB031500EB4500DCF808C0D1
:10EED00022300CEB45052235D8F82CC03F7D5B1C59
:10EEE000D8465F430CEB47034FF0010B1CB10CE01D
:10EEF00097F8C950E3E744788C4205D1B3F9007024
:10EF00004F4501DD85F801B00124D8F800C097789D
:10EF10009CF814C0ACF1010C674562D1461CBE5D83
:10EF20008E4207D133F917C0CC4503DD05F1010C42
:10EF300007F80CB09278521ED6B252E002195278FD
:10EF40008A424CD133F914204A4548DD02EB0A0EBF
:10EF5000002703EB4402CDE9002732F9022C964545
:10EF600005DADDF800C0BCF902C0E64537DB012C4C
:10EF700010D0D8F800703F7DBF1EA74217D1009F68
:10EF800037F9047CBE4527DA009FB7F90270BE4509
:10EF900025DB21E0B3F9027007EB0A02B3F9007038
:10EFA000BA4219DAB3F90670BA4218DB14E0964592
:10EFB00006DA009FB7F90470BE4501DA012201921A
:10EFC000009F37F9047CBE4504DA009FB7F9027050
:10EFD000BE4504DB019A12B92F1987F801B0641CF1
:10EFE000E4B2B442AAD9C9E52DE9FF4F9AB092F82C
:10EFF0000180D7780020ADF84800ADF84C0015909E
:10F00000A848A94D1E4601782868144601291FD03A
:10F0100010F1710012AB90F8009090F801A013A8C5
:10F02000CDE90006DDE91A01FFF742FE2868A04994
:10F0300090F8760070B1BDF84820BDF84C300988D2
:10F04000D21A42436420B2FBF0F0084405B203E058
:10F05000C930DFE7B1F90050607848B9CDE9006503
:10F06000DDE91A014FF0010800232246FFF717FFE0
:10F070008D49E0780968497D491E884209D1CDE96A
:10F080000065401EC7B2CBB2DDE91A012246FFF788
:10F0900006FF4146ECE000BF844B1A9A01EB0110D9
:10F0A00002EB40029B68223203EB400022300790C3
:10F0B0007D48F36AA1F1010C0068007D00FB0CFCA7
:10F0C00003EB4C0CCDF830C000FB01FC03EB4C0C07
:10F0D000CDF814C001F1010CCDF85CC000FB0CFCB4
:10F0E00003EB4C0B01F1020C00FB0CFC03EB4C0E90
:10F0F00001F1030C00FB0CF003EB400006902078BC
:10F10000B0E0131893F801C01B9B9C457ED13BF9DE
:10F1100010300393AB4279DD00230D93039BDDF8A0
:10F1200014C04B4401933CF910C0CDF850C0634566
:10F1300006DA9C463EF910309C4501DA01230D9316
:10F14000F0B3594B1B6819931B7D18935B1E8342C8
:10F1500072D00BEB4008DDF804C038F9023C0B9389
:10F160009C4506DA6346B8F902C0634501DA01231B
:10F170000D93DDF814C0039B0CEB400CCDF838C0A8
:10F180003CF902CC5344634509DA0EEB400CBCF960
:10F1900002C0634503DA4FF0010CCDF834C0DDF84E
:10F1A00038C0BCF902C0634505DA0EEB400C3CF9EF
:10F1B00002CC634554DB0D9B43BB199B5B7D00E098
:10F1C0003AE09B1E8B420CD0DDF850C0019B63459A
:10F1D00007DADDF818C03CF910C0634501DA0123F5
:10F1E0000D9301290CD0DDF830C0019B3CF910C013
:10F1F000634505DA3EF910C0634501DA01230D933A
:10F2000001281CD0189B9B1E834200E016E00AD008
:10F21000DDF82CC0019B634505DAB8F904C06345ED
:10F2200001DA01230D9338F904CC019B634503DA1D
:10F23000B8F902C0634513DB0D9B5BB110E0BBF96D
:10F2400002C00CEB0903BBF900C06345F4DABBF95B
:10F2500006C0EFE7079B4FF0010C034483F801C0A1
:10F26000401CC0B2A3788342BFF44BAF1798C1B221
:10F27000B9427FF611AF15981EB08CE52DE9FF4F0E
:10F280000A4CC5B000264FF48861A0680EF0EBFA76
:10F2900045AD0FCDFFF7A8FE479909680091A8BBBF
:10F2A0006B4607E06F0210003C021000A004100043
:10F2B000440510002DAA0021A046A068FEF7C9FC55
:10F2C0000546012837D90AF057F90124F74F0DF107
:10F2D000B409EA4623E000BF396839F8140091F810
:10F2E0007510884213D9012688F800604899488132
:10F2F0000AEB84008346489901F0FAFDE1B25A46D0
:10F30000489BD8F80800FFF77FFC07E013E0E848C7
:10F31000007818B90AEB840004F01CFF641CAC42AE
:10F32000DADD386890F84004800702D400200AF043
:10F3300028F9002E03D145AC0FCCFFF765FC49B08E
:10F3400029E52DE9F04F8A46D84900259946864699
:10F35000D1F8006028462B4609EB0301491E1FD453
:10F36000747D8C421CDD377D01F1010107FB01F149
:10F370000EEB410803EB430C4FF000010AEB4C0B82
:10F3800002EB0104641E08D4A74206DD3BF911C05C
:10F3900038F91440604404FB0C55491C0329EFDB89
:10F3A0005B1C032BD8DB00B9012095FBF0F0F2E4E5
:10F3B0002DE9FF4F82B00C464178DDF83CB001B139
:10F3C000491EBA4A01F0FF09C1781668737D5D1EB7
:10F3D000A94201DA491C00E02946CDB2017801B109
:10F3E000491E01F0FF0A8178307D431E994201DAFF
:10F3F000481C00E0401EC6B2B4F9120009F1010138
:10F40000019064E0A94B4A1C1868007D00FB02F7DC
:10F41000484305990BEB470E01EB400000900AF1C1
:10F42000010051E0A14909680B7D059902FB030722
:10F4300001EB4701049FB1F90210B94240DD009988
:10F44000B4F9008001EB40010027B1F900C00CFBCA
:10F450000877B1F902C0B4F902800CFB0877B1F962
:10F4600004C0B4F9048001EB43010CFB0877B1F947
:10F4700000C0B4F9068001EB43030CFB0877B1F937
:10F4800002C0B4F908800CFB0877B1F904C0B4F9E4
:10F490000A80B3F900100CFB0877B4F90CC001FB2B
:10F4A0000C71B3F90270B4F90EC0B3F9043007FB64
:10F4B0000C11B4F9107003FB0711019B91FBF3F1E0
:10F4C0002EF81010401C00B2B042ABDB11B2A942C2
:10F4D00098DB4F4617E0017D781C41430BEB410858
:10F4E00000903B46524621460598FFF72AFF28F830
:10F4F0001A003B46324621460598FFF722FF28F8BE
:10F500001600009807B26948AF420068E3DD007D4D
:10F51000691C41430BEB4101009109F10101484392
:10F520000BEB4008574612E04B463A4621460598F9
:10F53000FFF707FF28F817002B463A4621460598A3
:10F54000FFF7FFFE009921F817007F1C3FB2B7427A
:10F55000EADD06B01FE4F8B556491046069A097868
:10F560001D46022914D2544C50492E7E2368096846
:10F570007EB191F84060B6060AD5012A08D1009301
:10F58000B1F958204D4B4E49FFF712FF2068E86251
:10F59000F8BD91F8C061F706FAD5B60609D5009313
:10F5A000B1F9C421454B4749FFF702FF2068A86223
:10F5B000F8BD012AFCD10093B1F9C421E2E72DE99D
:10F5C000FF5F3A4E8346404D3468A07E80070AD5DF
:10F5D00045F6BA50ADF80000ADF80200ADF80400F1
:10F5E00044F6121009E046F6B650ADF80000ADF84A
:10F5F0000200ADF8040045F28A00ADF806001021C3
:10F6000032480EF030F9324B1421304A4FF00109E4
:10F61000B3F900701DE0002016E000BF94F81480DC
:10F62000431C9C4603FB081335F91330BB4209DD2C
:10F6300002EB410A09FA00F33AF8288C48EA030879
:10F640002AF8288C0FFA8CF0637D8342E6DC491C93
:10F6500009B2207D8842DEDC0024EA46904602AFF3
:10F6600008EB840138F8240049884FF0000540EA8F
:10F67000010027F814003AF8141000EA010027F8F6
:10F68000140043E037F8143009FA05F213423BD076
:10F69000827E008B92071FD5B0FBF1F10D484057D9
:10F6A00005FB110000F273501DE000003C02100049
:10F6B000680210006D0210009802100018D8012096
:10F6C00086DC010072DC010038430120285810005C
:10F6D00044051000AC041000B0FBF1F0FE4949579E
:10F6E00005FB00102D30ABF802003068C18A007DA8
:10F6F000B1FBF0F060434FF4F06101EB4000ABF878
:10F700000000584609F03CFE6D1C2DB23068417D6A
:10F71000A942B7DC641C24B2042CA1DBBDE8FF9F26
:10F72000F0B4EE4C2678EE4C256816B1B5F80241DF
:10F7300001E0B5F800411E7E64431EB195F86050AB
:10F74000EE0702D0F0BCFFF727BBAD0705D5E54DAE
:10F750002D68A54201DAF0BC90E5F0BCFFF754BA81
:10F760002DE9F0478146DE488A46002301681846A5
:10F7700001250E7D4F7D1DE000EB001409EB4404D4
:10F780002234194612E000BF52F8208005FA01FC2D
:10F7900018EA0C0F08D004EB010898F801C0BCF17E
:10F7A000000F01D188F801A0491CC9B2B142EBD3C6
:10F7B000401CC0B2B842DFD3BDE8F087C74A10B5DD
:10F7C000127801243AB9C64A126892F860201207EA
:10F7D00018D5012916D181780278891A01D5C1F18D
:10F7E000000101F10101CAB2C1784078081A00D5C0
:10F7F0004042401CC1B21046F4F76BF8C0B2012879
:10F8000000D10024204610BD2DE9F04F8A46B449AE
:10F8100083469E464FF001095078D6780C6824E064
:10F8200000EB00130BEB430322331178957818E0BB
:10F830005F1897F801C0D44511D194F81480471C83
:10F8400007FB0817DEF828C00CEB4707B4F8D2C155
:10F85000B7F90070BC4502DA4FF0000903E0491C1B
:10F8600009B28D42E4DA401C00B28642D8DA48463A
:10F870009DE52DE9F0439946994B01261C6894F8C3
:10F8800008319D0748D51578B5EB531F01D80025E1
:10F8900001E0A5EB5315EFB2257D92F802C0A5EB70
:10F8A000531808F10108E04501DA6D1E01E00CEB88
:10F8B000531505F0FF0C5578B5EB531F01D8002503
:10F8C00001E0A5EB5315647DD278A4EB531808F141
:10F8D0000108EDB2904501DA641E01E002EB531419
:10F8E00004F0FF0811E000BF05EB051200EB420336
:10F8F00022333C4606E01A19527812B18A4200D0EF
:10F900000026641C6445F6DD6D1C4545ECDD002ECB
:10F9100002D1022189F81810BDE8F08330B5704C8F
:10F92000714A2468B2F90030704A34F9A85FB2F91C
:10F930000020B4F9024029B96D49B1F900306D4990
:10F94000B1F90020A04201DD104630BDA84201DA25
:10F95000184630BD201AD11A4843611B90FBF1F0C4
:10F96000101A00B230BD2DE9FF4F83B04FF0FF36C3
:10F97000DDE9105489460746019693464FF0640A24
:10F98000B04610460699F3F7ACFF01B24FEA6900A2
:10F99000009188427DDA52480068B0F8A1204A45BB
:10F9A00077DD129931B1012918D0022927D0032916
:10F9B00070D13DE0A11E05D4027D611E01FB025104
:10F9C00037F91160427DA11C8A424DDD007D04F1B2
:10F9D000030404FB005037F9100044E0A91E07D4CB
:10F9E000027D611C01FB025107EB410131F9046CFE
:10F9F000007DA91C884237DD04F1010415E0A91E31
:10FA00000BD4427DA11C8A4207DD027DE11C01FB73
:10FA1000025107EB410131F9046C007DA91C8842B9
:10FA200022DDA11E20D4A4F1010404FB005016E045
:10FA3000A91E09D4A11E07D4027D611E01FB02513B
:10FA400007EB410131F9046C017DAA1C91420BDDE9
:10FA5000427DA01C824207DDE41C04FB015007EB41
:10FA60004000B0F904008046701C48D018F1010035
:10FA700045D058460699F3F72CFF009902B2A9EB3E
:10FA80000100069B01B2ABEB030064235843009CCA
:10FA900001E054E033E009EB0403544203EB440378
:10FAA00090FBF3F0002800DA4042414391FBFAF169
:10FAB000A9EB010109B25A4524D1069A64235A439D
:10FAC000069BF31A03FB002393FBFAF2642412B2A1
:10FAD0000BFB04F310E00000AC0410006D021000FA
:10FAE0003C0210004C0510004405100046051000B3
:10FAF0003C0510003E051000A9EB0B0412E0019834
:10FB000007B054E464230BFB03F2A8EB0B0303FBE5
:10FB1000002393FBFAF2069B6424069D634312B212
:10FB2000A9EB050404FB003494FBFAF3484390FB73
:10FB3000FAF01BB21A440844C2EB400006B2304649
:10FB4000DEE72DE9FE4F9946F94B571C0646D3F8E0
:10FB500000C04FF0FF3004469CF81430054607FB08
:10FB6000031B5FEA090836F91BA009D0B8F1010FA1
:10FB700018D0B8F1020F21D0B9F1030F52D133E000
:10FB8000B2F1010803D402FB031536F915509CF8B5
:10FB90001580B84544DD02F1020404FB031336F975
:10FBA00013403DE04F1E03D406EB4B0535F9025CD4
:10FBB0004F1CBB4234DD06EB4B032FE0B1F10108D3
:10FBC0000AD49CF81580B84506DD951C05FB031585
:10FBD00006EB450535F9025C4F1CBB4220DD571E84
:10FBE0001ED402FB031317E0B1F1010808D4B2F1EF
:10FBF000010805D402FB031506EB450535F9025C47
:10FC000001F1010843450BDD9CF81580B84507DD7F
:10FC100002F1020404FB031306EB4303B3F90240B1
:10FC20006B1C01D1631C0ED09CF8A0309B0607D53D
:10FC30008DE806022B46224651463046FFF793FEDA
:10FC4000691C03D003E047F6FF710AE02546611CFA
:10FC500000D12C466219C2EB4A0109B2884200DD8C
:10FC60000146B348006890F8F107022808D1B1486E
:10FC700020F8395000EBC900A0F802A08480C180B0
:10FC80000846BDE8FE8F2DE9FF4F1E46A84B4FF0FA
:10FC9000000A1178186883B0554654465FEA010E91
:10FCA00006D15178B9B1417DD778491E8F4212D023
:10FCB000017D97788B46491E8F4204D192F801C08E
:10FCC000BCF1000F07D08F420BD1417D92F803C0E9
:10FCD000491E8C4505D1B0F8AA00801CA6F8230067
:10FCE000AAE0517892F803C0B06A24E04B1C0BFBE9
:10FCF00003F200EB42020192039A01EB011302EBC3
:10FD0000430202F122090BB27246009310E000BFD9
:10FD100009EB020393F80180049B984507D1019BEE
:10FD200033F91230534502DD009C9A4615B2521C3D
:10FD30009742EDDA491C8C45D8DA01232246294640
:10FD4000FFF7FFFE0746002322462946B06AFFF769
:10FD5000F8FE8046022322462946B06AFFF7F1FEEC
:10FD60008346032322462946B06AFFF7EAFEDFF8FE
:10FD7000C0A18146DAF8000090F8A01049061ED50F
:10FD8000B5B1017D491EA94212D01CB1407D401E73
:10FD9000A04201D1B8460BE041463846F3F799FD41
:10FDA00002B249465846F3F7A4FD00BF0FFA80F8A7
:10FDB0000027601ED446641CDAF800901FE008EBB0
:10FDC0000700F3E7002819DB99F81510814215DDCB
:10FDD00099F814A0431CB26A0AFB03F102EB410B31
:10FDE000691E6A1C08E0002905DB8A4503DD3BF833
:10FDF00011303B441FB2491C9142F4DD401CA0422B
:10FE0000E0DDFA2008FB00F898FBF7F004B2A6F852
:10FE1000234001212046FFF781FD47490C80DCF893
:10FE2000001091F8F117022903D142490C844F8444
:10FE30008884318C814201DD012061E600205FE68B
:10FE40002DE9FF4FB0F92050A3F10103002403EB8B
:10FE5000D37040F34F0316B22146F01A00D50020AC
:10FE60000FFA80FB3248F7180068467DA6F1010CB6
:10FE7000674501DD664600E03E464FEA224736B25E
:10FE8000FA1A00D500220FFA82F9027D3B44571E70
:10FE9000BB4201DD521E00E01A4617B25B462EE05F
:10FEA0004A4603F1010A26E0037D0AFB032C9E4625
:10FEB000019B33F91C30B0F868C09C4500DB00237F
:10FEC0004FF47A7C03FB0CFC9CFBF5FC644490F83B
:10FED000F1C724B2BCF1100F09D190F81580DFF8FA
:10FEE00054C008F1010808FB0E182CF81830491C02
:10FEF000521C09B212B2BA42D6DD0FFA8AF3B342EB
:10FF0000CEDD90F8F127102A0ED10A481023038085
:10FF100043885B1C43808480C180A0F80A9087815D
:10FF2000A0F80EB006824582012907DA002008E019
:10FF30003C02100018D80120E226100094FBF1F0DA
:10FF400000B2102A01D1FE49088104B090E42DE9E5
:10FF5000FF4F8146B0F93860581E00EBD07040105A
:10FF600011B20D1A0FFA85FB0D184FEA224CACEBBB
:10FF700000020FFA85FA604405B25B4396FBF3F08A
:10FF800006B281B0EF4812B2009202680024DFF896
:10FF9000B0E392F8F177092F15D14FF00108AEF8D0
:10FFA0001280AEF8143092F81480491C01FB08CC82
:10FFB000029931F81C10AEF81610B9F83810AEF8E6
:10FFC0001810AEF81A60584657E000BF40F6FF7BA5
:10FFD000009918E0002814DB92F815C0844510DD64
:10FFE00000290EDB92F814C08C450ADD00F10108EF
:10FFF00008FB0C18DDF808C03CF918C0DC4500DA35
:020000021000EC
:10000000E346491C09B2A942E4DD009931E0002829
:1000100012DB92F815C084450EDD00290CDB92F846
:1000200014C08C4508DD00F1010808FB0C18DDF850
:1000300008C03CF918C001E04FF0000CE146092F60
:1000400005D14FF00008AEF80280AEF80480A9EBAD
:100050000B0CB2F868800FFA8CFCE04501DB4FF026
:10006000000CBCEB060C01D5CCF1000C491C64441F
:1000700009B2A942CBDD401C00B25045A6DD092FD4
:1000800001D1AEF81C4094FBF3F001D1AEF81E0094
:1000900005B0BDE8F08F2DE9FF4F8346DDE90DE7A0
:1000A000002038608A465378A64E33E003EB0314F1
:1000B00031680BEB4405DEF828C00C7D03F1010923
:1000C00004FB09F422350CEB440411781CE000BF5A
:1000D00005EB010C9CF80180D04513D134F9118057
:1000E000D7F800C0C444C7F800C034F911C0844533
:1000F00008DD6046DDF80CC0ACF80210DDF80CC07D
:10010000ACF80030491CC9B292F802C08C45DFD26D
:1001100009F0FF03D1789942C8D28B49B1F9001098
:10012000884252DAD178537899424ED101210F2B6F
:1001300024D11378854CD6F800801CE0A56801FA1C
:1001400003F73D4216D13D438946A560002B05DDEE
:100150005F1E09FA07FC45EA0C05A56098F81450E3
:100160006D1E9D4206DD5D1CA76801FA05F947EA90
:100170000907A7605B1C95789D42DFDA5378002B56
:1001800023D11378724C37681CE000BFA56801FAD0
:1001900003F6354215D135438C46A560002B05DDAD
:1001A0005E1E0CFA06F845EA0805A5603D7D6D1E49
:1001B0009D4206DD5E1CA5680CFA06FC45EA0C05AE
:1001C000A5605B1C95789D42E0DABEE62DE9FF4F05
:1001D00083B01878109C92461E46A07098782070C4
:1001E0005878E070D87860704FF000085F784CE085
:1001F000039907EB071001EB400101F12209049973
:1002000001EB400000F1220B1298826A4D48006811
:10021000017D781C4143019002EB4100009035784C
:100220002EE000BF09EB05004178514526D100982A
:1002300030F91510119881421CDD08F101001FFAF8
:1002400080F821782846F3F744FB2070617838461F
:10025000F3F73FFB6070A1782846F3F742FBA070EC
:10026000E1783846F3F73DFBE0700BEB050080F8D2
:1002700001A003E00BEB0500002141706D1C2DB2C5
:10028000B078A842CEDA019807B2F078B842AFDA77
:100290000FFA88F034E42B490278096822B10A7D0C
:1002A0008378521E934208D1427822B1C278487DA9
:1002B000401E824201D1012070470020704730B5B6
:1002C0000546A1B01F4800238DF8803002680C4617
:1002D000107D401E8DF882008DF88130507D6B4678
:1002E000401E8DF8830020AA2846FDF7A6FD0022B7
:1002F00020A96846FDF7C9FD6A4621462846FFF752
:100300002FFA21B030BD2DE9F14FE2B00026CDE942
:1003100058661048104D5C9600686860094C00F5FE
:100320008860A8602168B346B1F90E125A914FF463
:1003300088610DF098FA206890F86010CA070DE007
:1003400018D801203C0210003C0510006427100062
:10035000F826100094021000A004100001D18907B3
:1003600001D501215991FE49097821B190F8E006A3
:10037000C0F3400003E090F8C001C0F3C0005E90FD
:100380000020149014AB41AA01216868FDF761FCBC
:10039000F44907460873236801201A7D15E00121FE
:1003A00000EB0016F04DDFF8C49309E0D9F804C063
:1003B00001EB46081CF808C005F802C0521C491C95
:1003C00093F814C08C45F1DA401C597D8142E6DA7D
:1003D0000125D1E23C2103A80DF067FADFF89083F4
:1003E000E9B241A8CDF83480CDF838808DF82E10D0
:1003F00030F81500ADF8160058AA03A8CDE90002A0
:1004000014A8DFF8689300EB850212925DABD9F86F
:100410000400FFF740FE0646206890F8F1071D280B
:100420000DD11D21A8F8001005EB450108EB410096
:1004300028F81160BDF81620428063218180ADF854
:100440002C60052203A85D99FEF7DCFAADF84400A4
:100450000523C84903A85D9AFFF7F2FC014620680E
:1004600090F8F1270C2A0AD10C23A8F80030B8F82C
:1004700002305B1CA8F80230589BA8F80430ADF895
:10048000421090F8F1170C2925D0152923D000210E
:10049000ADF82F10DFF8D4C28DF83C10BDF97621ED
:1004A000BDF97431ADF84020ADF83E308CF8001045
:1004B00042B13BB1017D491E8A4203D0417D491EB4
:1004C0008B4219D101215B919DF83D1041F0010152
:1004D0008DF83D1012E0BDF84220A8F80620BDF8C6
:1004E0004420A8F808209DF84620A8F80A209DF886
:1004F0004720A8F80C20CAE700215B9100215F91FA
:100500009D49097801291AD190F85E148A4216DBB8
:10051000017D491E8A4212DC9849994BB0F95B244F
:100520000A801B78012B03D190F88F311A440A807E
:1005300090F85D0491B2081A924908801BE26FF0AE
:100540000101619102216091017D5B1C03FB01228D
:100550004FEA011C0FFA82FA8B4BCDE9001C0022F6
:100560000292D3E903C242EA0C02D3F804C01B781A
:1005700042EA0C09854A012BD2E9038C4CEA080CAB
:10058000D2F804804CEA080E02D01278012A20D159
:1005900000221CE00123934013EA090F09D0DDF883
:1005A00004C00CEB0208DDF884C101FB0C88D045C7
:1005B00009D013EA0E0F09D0609B01EB020C01FB7E
:1005C00003CCD44502D10121029102E0521C914298
:1005D000E0DC6F490978890740D561490978E9BBB2
:1005E0006C4A90F8A710128891426549097801D2A7
:1005F00011B179E0022977D2589A5A998A4273DA6E
:10060000029959BB01218DF824105D4990F8A4800E
:100610000978012905D190F8BC2002EB08011FFAE6
:1006200081F85B9901293ED090F8A51090F8CE0092
:1006300008445949814603A8B1F9002013A9009143
:10064000CDE90120DFF824A1129BEAB2DAE9010129
:10065000FFF7BCFD80B2ADF8160000E022E0424991
:100660004045485540D948453ED84B49B1F900105E
:100670008E4239DD012819D036D9206890F8A010B3
:1006800089071BD54549B0F8FD00096840438842F9
:1006900014DBE9B203AB13AADAF80800FFF7F3FAA8
:1006A00001280BD020E090F8A600C2E73C48B0F942
:1006B000000086421FDC5F98B0B15CE1206890F8D2
:1006C000A000000617D501219DF84700CDE90001E3
:1006D0009DF84630BDF82C20BDF84210BDF844000E
:1006E000FEF70AF9012806D05B991298FFF766F821
:1006F000012817D03FE10220ADF82600ADF8280010
:1007000000208DF825004FF0010BE9B203AB5646EF
:10071000129ADAF80400FFF7ACF8E9B203AB13AAB7
:10072000B06891E01748B0F9000086427EDD1D49AF
:100730000DF58278B1F9001038F81590814238DA59
:1007400013AACDE90020094803A902914168EAB241
:10075000129B0846FFF73AFD28F8150024E0000038
:1007600072021000E2261000D0A70120A0041000A1
:1007700018D8012038430120730210003C051000F6
:100780006D0210004405100064271000F8261000C8
:10079000E0021000D4041000460510004C051000C3
:1007A000480510003A051000DDE912120A60ADF8A4
:1007B0001600206890F865608648007848B1129865
:1007C000FFF769FD0128206837D090F8BD0030445C
:1007D00086B238F81500B04238D903A87E4E4FF0E3
:1007E000010B0090CDF870B1EBB2129A0D987168C0
:1007F00000F09AFB206838F8151090F867209142B5
:100800001ED202218DF82410744BBDF82A10599A7B
:100810009982B0F86E00814200D20022B9F1030F34
:1008200011D3002A0FD0E9B203AB00E00FE0009231
:10083000129A7068FEF78FFE97E090F8C300C6E743
:1008400004208DF824009FE0FEF7DEF993E0206895
:1008500090F8C011C90733D06149096881B3614973
:10086000097869BB00218DF8241090F8C001400779
:1008700005D55948E9B214AA4068FFF720FD5A4847
:1008800047F6FF78007818B1206890F8E16609E033
:100890005B9801285548007809D00128206810D0BD
:1008A00090F8CB614B48007801280DD011E0012869
:1008B000206802D090F8CD61F4E790F8CC61F1E7C0
:1008C00059E090F8CA61EDE7206890F829043044B7
:1008D00086B247480DF58279B0F900104548B0F965
:1008E0000000814212DA13AACDE900203A4803A998
:1008F00002914168EAB2129B0846FFF767FC29F8AB
:100900001500DDE912120A60ADF8160039F815007D
:10091000B04230D940452ED8629902202E4E087040
:1009200003A80090EBB2129A0D98716800F0FCFADF
:100930005E980090E9B203AB129A7068FEF70BFE66
:10094000206890F8C00180070DD52848007801285C
:1009500009D1E9B203AB129A7068FEF755FF01287E
:1009600001D1254908705E9870B1E9B203AB129AC3
:100970007068FEF7D5FE6D1CBD427FF62BAD1F489B
:100980000078012805D016E0E9B203AB129A70682E
:100990005AE70420ADF81600ADF814001848642199
:1009A00007910088401CADF82C0002208DF824002F
:1009B00003A8FEF704FE1349134881F800B05C99C0
:1009C000017063B0BDE8F08F04480021017301801D
:1009D000704700006D021000A0041000E226100015
:1009E0009C010022590210007202100061021000E6
:1009F0003A0510004A051000380510007302100077
:100A00003C0510005F02100060021000704770B5D6
:100A10000346AF48154600240268107D527D03EB63
:100A20004003504300B20AB201461846F3F758FAA1
:100A3000A84200DD0124204670BD2DE9F047A44CFA
:100A40000F460646216800259146B1F81C04012B8B
:100A500003D1B1F81E14084480B201B2304600F050
:100A60006FFF80462068B0F82424B0F82214304686
:100A7000FFF7CDFF06462068964B427DB0F9201463
:100A8000384602F008FC07462068934B027DB0F917
:100A90002014484602F0FFFB012F15D1012813D185
:100AA000B8F1000F10D1012E0ED120688C4B417D82
:100AB000007D41434A008949096801EB400103EB8D
:100AC0004000F3F773FD01252846BDE8F08737B5F0
:100AD000144601A96846F3F745FE00986080019826
:100AE000208002206083A083204608F049FC3EBDA0
:100AF0002DE9F04700271446054689463E464FF04B
:100B00000108DFF8CCA102F0B8FC00B24FF4FA4CB7
:100B100035F91010DAF80000B0F8460241434FF4FE
:100B20007A7091FBF0F001B20020034604EB400222
:100B3000401C9380A2F80EC00328F7DB012020752B
:100B4000002031E0B8F1010F31D004EB460235F955
:100B500010C0D389634504DD35F81030D381A31963
:100B60009872D28935F910300A4493421BDD7F1CFC
:100B7000FFB24FF00108022F00D90227227D521C3C
:100B8000227504EB470235F91030B2F804C0634512
:100B900009DDDAF800C0BCF85EC1634503DD35F855
:100BA00010309380E055401C4845CBDB8DE704EBCB
:100BB000470235F91030B2F804C0634509DDDAF8B0
:100BC00000C0BCF826C4634503DD35F810309380BF
:100BD000E055928835F91030521A9342E3DA761CC8
:100BE000F6B24FF00008022E00D9022604EB4602AE
:100BF000B2F80EC09C45D6DD35F81030D381A2196D
:100C00009072D0E72DE9FF4FDFF8C4908B468FB08C
:100C1000D9F800009A464C46017D08AA5846FFF7CD
:100C200067FF206802AA417D0F98FFF761FF9DF8DA
:100C30001C709DF83460B74202D90126002529E0D6
:100C400001270025002422E0D9F8000090F81B14A9
:100C500001F00F01009108A9C38A0A5D017D584681
:100C600002F01CFC8046D9F8000090F81B1401F03B
:100C70000F01009102A9038B4A5D417D0F9802F09C
:100C80000DFC014652464046FFF721FF641CB4426A
:100C9000DADB6D1CBD42D5DB13B0BDE8F08F00B5CB
:100CA0008FB002238DF818300523ADF80A3041F6D5
:100CB000583303930723ADF808300A4B1B885B1C9D
:100CC000ADF820306B46FFF79DFF0FB000BD000070
:100CD0003C021000BC021000B80210009402100088
:100CE00018D801203C051000F0B5B2F900400568A5
:100CF000AC4202DDB3F900102EE002EB410434F9FE
:100D0000026CAE4204DA03EB410131F9021C23E02C
:100D10000024491E0BE000BF32F91470AF4205DC1D
:100D200002EB4406B6F90270AF4202DA641C8C4250
:100D3000F2DB32F9146003EB440133F91430B1F9FA
:100D4000021002EB4402AD1BC91AB2F9022069433A
:100D5000921B91FBF2F119440160F0BDF0B50E4613
:100D60002B49096801F275433AB3012A2ED0022AB1
:100D700035D0032A40D0042A49D191F86EC491F8A5
:100D80006D441A4691F8741403EB4C0303EB4107CE
:100D900007EB44050CEB04013E2938DCBCF1010FE4
:100DA00002DD6146FFF7A0FF012C30DD2B463A46FD
:100DB00021463046BDE8F04096E791F86FC491F8BF
:100DC000704403EB4C0591F8711410E091F86FC476
:100DD00091F8704403EB4C0591F8721407E091F818
:100DE0006FC491F8704491F8731403EB4C0503EB56
:100DF000410202EB4C07CDE791F811C601F21262F5
:100E000002EB4C0391F8104603EB4C07C0E7F0BD32
:100E10003C0210004FF47A72504390FBF1F1744899
:100E200010B5814201DAC01110BD42F6A6408142E0
:100E300001DD5A2010BD6F4A002000BF32F910308A
:100E40008B4205DC02EB4003B3F902308B4202DA3D
:100E5000401C4528F2D332F9104000EB800302EB2E
:100E60004000091BB0F90200553B001B01EB81015A
:100E700091FBF0F0184410BD30B50D460446FFF765
:100E8000C9FF00EBD0704010002D02D00DDD34B151
:100E900030BD002C03D005DD4FF02D0030BD4FF0EC
:100EA000000030BD4FF05A0030BD002C03D005DDEE
:100EB00000F15A0030BD6FF0590030BDA0F15A006A
:100EC00030BD10B58C1A00D56442002800DA4042CB
:100ED00004EB400011440A18081A521040104FF455
:100EE0007A71484390FBF2F0C0F57A70D88310BD58
:100EF00030B5827803784D89D21AC3784078521C75
:100F00001B1A5B1C05FB02F0D4185D4340006A000D
:100F1000B0FBF4F0B2FBF4F2904202D948838A832A
:100F200030BD4A83888330BD2DE9FF4F0027164628
:100F300082B03A463C46BC46BB46BA46707896F804
:100F4000039025E0039900EB001301EB43012231EC
:100F500001913178009196F8028016E0019B0B44D4
:100F60005D78059B9D420FD1A9EB000303F1010EB3
:100F7000009B0EFB0EAACD1A6D1C05FB05BB05FBE5
:100F80000ECC7F1C2A447444491C8845E6DA401C78
:100F90008145D7DA4FF47A70504390FBF7F101FBAB
:100FA00004F54FF47A734FF47A70604390FBF7F0D6
:100FB000514391FBF3F2604390FBF3F195FBF3F5A2
:100FC000ACEB0505ABEB0207AAEB01046800391B8B
:100FD000FFF752FF0F9922464876394628460F9B65
:100FE000FFF76FFF0F9906B03046BDE8F04F7FE77F
:100FF0005AD3FFFF2CDC0100F94900200870F949A1
:101000000870F9490870704710B5F84A00206FF071
:10101000004100BF42F82010401C1428FADB3C219C
:10102000F3480CF020FC4021F2480CF01CFCF24983
:10103000002048618861487010BD10B5044600204A
:101040002070A070E07061706060E060206160619D
:10105000206684F85800A4F85A00A4F85C00A4F8AC
:101060006600A4F8640084F86800202104F11800E8
:101070000CF01BFC04F13800BDE8104020210CF0FE
:1010800014BC70B5DD49002001220870DC49E54B35
:10109000E54D0A70DB49E54E0870DB490870DB4915
:1010A0000870DB490870DB490870DB490A70DB49CE
:1010B0000870D1498871486288620871C861086205
:1010C0004A71D74A1268B2F862401C80B2F8A13067
:1010D0002B80B2F80C523580D54EB2F8C621328042
:1010E000D44E3480D44C2380D44B1D80D44B1A80F2
:1010F000D44A10800861FFF789FCFFF77DFF0121CA
:10110000D148FFF79AFF0021D048FFF796FFBDE8CE
:10111000704079E72DE9FF4FC14A9B4681B01268C4
:10112000012592F815C0137D0CF1010C69E000BF98
:101130004FF0000A47F6F8724FF001095442D646C4
:101140005646CDF8009019E005FB036730F817808C
:1011500031F81770A7EB08073FB2BA4200DD3A46F4
:10116000BC4200DA3C46002F02DA4FF0000903E0EF
:1011700002DD4FF00007009706F101069E42E3DB17
:10118000009E59EA060709D0B9F1010F03D0B9F161
:10119000000F05D008E0009C012C05D1002203E0DF
:1011A000009E012E00D12246002412E005FB0346DA
:1011B00030F8167031F816601744F61B36B25E45EB
:1011C00006DACBF10007BE4202DDB2440EF1010E99
:1011D000641C9C42EADBBEF1000F01DD9AFBFEFAC3
:1011E0000AEB0204002209E005FB0326DDF80C806F
:1011F00030F81670521C274428F816709A42F3DB18
:101200006D1C654594DB05B0BDE8F08F2DE9F00F4E
:10121000834C9B46266896F8E036DD088C4B1B789D
:10122000022B02D0032B04D004E096F8ED56ED0813
:1012300000E00025C2F11007BBF1010F07D0DFF875
:101240001492042B07D0EBB30023A24657E0BDE86D
:10125000F00FF3F7D0B9002530E0002329E000BFFC
:1012600005FB063631F916C030F916800CFB02FC7E
:1012700008FB07CC4CF30F1C21F816C0D4F800C0B3
:101280009CF8408698450FDC9CF8418698450BDB1E
:101290009CF8428608F10108A84505DC9CF843C685
:1012A0000CF1010CAC4503DA39F816C021F816C070
:1012B0005B1C2668367D9E42D2DA6D1C23685B7DFE
:1012C0005B1C00E03AE0AB42C7DABDE8F00F7047C4
:1012D000002611E0DAF80040247D03FB0464761C4C
:1012E00031F914C030F914800CFB02FC08FB07CC68
:1012F0004CF30F1C21F814C0AE42EBD95B1CDAF89A
:1013000000605446767D761C9E42E1DA00204A4613
:101310000EE02B4607E000BF00FB06365B1C32F8F0
:10132000167021F816702668367D9E42F4DC401C4B
:1013300023685B7D5B1C8342EBDAC6E7464B1B7878
:10134000012B01D0002343E00125A24627E0002421
:101350001FE000BF414EC4F11F0806EB850605FBE8
:10136000034356F804CC012606FA08F61CEA060FD9
:101370001FD0BBF1010F19D031F9136030F913C040
:1013800056430CFB076646F30F1600BF21F81360A7
:10139000641CDAF800301B7DA342DBDA6D1CDAF83E
:1013A0000040647D641CAC42D1DC8EE730F81360F1
:1013B000ECE739F81360E9E731F9135030F91360BD
:1013C000554306FB075545F30F1521F813505B1CD9
:1013D0002668757D367D6D1C75439D42ECDC74E797
:1013E0006102100038051000590210003858100032
:1013F000C02B0120FC2B0120CC0410005D0210004A
:10140000560210005E0210005F0210006002100021
:101410005B0210005C021000AD021000D902100047
:101420003C0210003C0510003E0510004005100075
:101430004205100044051000460510004805100044
:101440004A0510003A05100064271000F826100025
:1014500072021000A800012005031000E42810000B
:101460002DE9FC5F984693460C46074600264FF050
:101470000109FE4D2868007D420001EB80003946DD
:10148000F3F794F82868417D007D491C41434200F0
:1014900000EB400007EB410104EB4000F3F786F856
:1014A00002274FF0300A28683023007DCDE900A0E4
:1014B00000FB07F104EB410002462146F3F7D5F9A2
:1014C0007F1C042FEFDB00202DE000BF00EB420368
:1014D00034F9101034F91330C91A01D5C1F10001E3
:1014E00000EB820224F812102A6834F91010127DE1
:1014F00002EB4203034434F91330C91A00D54942C0
:1015000002EB8202024409B224F812102A68127D0A
:1015100000EB820234F91230434500DD761C414570
:1015200000DD761C401C29680A7D8242CEDCD1B2E7
:1015300001EB410145F2AA5024F8210028685E45DC
:10154000007D00EB400004EB800046802968097DA7
:1015500001EB410104EB8101A1F8048001DD4FF0B2
:1015600000094846BDE8FC9F2DE9F0438946C04983
:1015700000252C460A78BD490B6812B1B3F8EE6617
:1015800001E0B3F8F6625A7D197D521C4A430EE021
:1015900039F9117030F911C007EB0608C44505DDB3
:1015A000BCEB070700D57F423D44641C491C8A42BE
:1015B000EEDCB04865B193F83610A14208D2816ADA
:1015C00011B10120BDE8F083012181620020F9E71B
:1015D0000021FAE72DE9FF5F8B46A548A34916468F
:1015E0000025027808680124A84612B190F8F12677
:1015F00001E090F837208A4602F00F0290F82010A0
:1016000002EB82024FEA420709071FD5B0F9789032
:101610009A48994A01680098F2F766FE98489649F8
:1016200002680B68D1F804C0D21A4368A3EB0C031C
:101630001A448368D1F808C0C068C968A3EB0C03DA
:101640001A44401A8118494500DD0024DAF80000E8
:10165000D14690F82000800713D58A48007880B9D9
:101660008948007868B989480078012809D18848F4
:10167000007830B959460098FFF776FF08B100248A
:1016800000E00CB94FF005087A480021C0F810803E
:101690008279A2B13170426A521C4262D9F800309C
:1016A00093F837301B0903EB8303B2EB430F02DDE2
:1016B00041628171012504B02846BDE8F09F0123F5
:1016C00014B141623370F6E7426A541C4462BA4274
:1016D00009DD83714162D9F8002092F837201209A0
:1016E00001D1817101253170E5E72DE9FC5F5F488B
:1016F000684900688979B0F9A130B0F90C42012934
:1017000006D190F83116490702D5B0F9602601E0FC
:10171000B0F9622056490978019111B1B0F9E21689
:1017200001E0B0F9C6115C4D2E78504D012E2D68A8
:1017300095F8C05100950FD1584D2D6865B1009DA9
:10174000B0F9AD30B0F96C20AD0705D5544D2D780A
:10175000012D01D1B0F96A204A4D2D78012D36D0E6
:10176000022D07D3B0F8BE1009B1B0F9BE20134660
:101770001C4621464B4DA2462B804B4D2C804B4D99
:101780002A804B4D298090F8A36090F864509F1BED
:101790000FFA87FC474FA41B90F8C361A7F800C05D
:1017A000E146DFF814C124B2A346ACF80040434C34
:1017B000551B2DB22580DFF808C18E1B414C36B277
:1017C000ACF800602478AE46012C0FD090E090F881
:1017D000BA502B442C4490F8BB501BB22A4490F8CA
:1017E0002A5424B2294412B209B2C3E790F8CC407B
:1017F000642504FB02F8B8FBF5F84244DFF8AC803E
:10180000A8F8002004FB03F8B8FBF5F21A44254BB6
:10181000DFF8A4801A8004FB0BF2B2FBF5F303EBB4
:101820000B02A8F80020019A002A05D090F8CF30CA
:101830001F4A03FB01F302E01D4A04FB01F3B3FB63
:10184000F5F31944118004FB0EF2B2FBF5F31B49CA
:1018500003EB0E020A8004FB0AF2B2FBF5F3124915
:1018600003EB0A020A8004FB09F12DE03C021000A0
:1018700072021000CC04100048261000A0021000D4
:10188000382610006D02100067021000730210006D
:101890005D021000E4021000610210009C010022B1
:1018A000380510003E051000480510003C051000EA
:1018B00042051000460510004005100044051000C8
:1018C0004A0510006F021000B1FBF5F202EB0901AE
:1018D000398006D090F8CF0000FB06F0B0FBF5F0A1
:1018E00003E004FB06F4B4FBF5F03044ACF8000070
:1018F000FE48007880070AD4FD48FE490088088029
:10190000FD490880FD48FE4900883880088000981D
:10191000C00702D0FB48006830B9F6480188FA4891
:1019200001803888ACF80000F448BCF90020B0F918
:101930000010B7F90000F1F7DCFFF449088011E668
:10194000F34A10B51268537D127D5B1C534306E0C9
:1019500030F912408C4201DD012010BD521C9A4228
:10196000F6DB002010BD30B5E94A1268537D127DC8
:101970005B1C53430AE000BF30F912408C4202DC8A
:101980004D42AC4201DA012030BD521C9A42F3DBD9
:10199000002030BD2DE9F05F8346DE488A461546BB
:1019A0000068002406464FF408610BF05CFFD8493C
:1019B00000202860086801229446037D19E000BFDA
:1019C00002EB021006EB400901200DE03AF913701A
:1019D0005B1C5F4507DD09F800C0D5F80080641C7A
:1019E0004744A4B22F60401C0F683F7D8742EDDA68
:1019F000521C0868407D9042E2DA20465DE6F0B570
:101A0000C34E33685D7D1B7D6D1C5D4300242746FE
:101A100009E000BF30F913C0944502DA21F81370D1
:101A200000E0641C5B1CAB42F4DB3068B0F89A0049
:101A3000A04201DD0020F0BD0120F0BDF0B5002581
:101A4000B34C26E000220123767D0EE003FB075C09
:101A500030F91CC0BCF1000F04DD0AB1944503DA73
:101A6000624601E00022731C5B1C9E42EEDA002AF3
:101A70000EDD012308E0367D03FB065630F81670B4
:101A8000BF1A21F816705B1C2668777D9F42F2DA38
:101A90006D1C2668377DAF42D4DCF0BD2DE9F043E4
:101AA0009B4B81461868467D057D761C002028E00A
:101AB0001A6892F85C20642A05D9C2F16402424394
:101AC00092FBF5F405E0643A02FB00F494FBF5F4B4
:101AD000141B643401224FF064080FE01F683F7D3F
:101AE00002FB070739F917C0BCF1000F05DD0CFB3D
:101AF00004FC9CFBF8FC21F817C0521CB242EDDB41
:101B0000401CA842D4DB5DE52DE9F047804B8146BF
:101B10008A461868447D057D641C01202DE01E68FE
:101B200096F85D10642907D9C1F16401421E514342
:101B3000727D91FBF2F206E06439421E777D4A43E2
:101B400092FBF7F28A1A317D6432414309EB410678
:101B50000AEB410700214FF064080BE036F911C091
:101B6000BCF1000F05DD0CFB02FC9CFBF8FC27F828
:101B700011C0491CA942F1DB401CA042CFDBBDE8EB
:101B8000F0872DE9F04F9146DDE909B7012547F6C9
:101B9000F87256429A46AC46002416E030F81430EB
:101BA00031F81480A8EB03031BB29A4200DD1A46F9
:101BB0009E4200DA1E46002B02DA4FF0000502E0DA
:101BC00001DD4FF0000C04F10104BC42E6DB55EAF4
:101BD0000C0306D0012D01D02DB108E0BCF1010F9E
:101BE00005D1002203E0BCF1010F00D132460025EF
:101BF0002C462B4611E000BF30F8136031F813C0BB
:101C00001644ACEB060636B2564505DACBF1000CAD
